:1000000010A904000000000004A8000008A80000D7
:100010000CA8000010A8000014A800000CA9000003
:100020000CA900000CA9000018A800001CA80000E2
:1000300020A8000024A800000CA9000028A80000A7
:100040002CA8000030A8000034A8000038A8000048
:100050003CA8000040A8000044A8000048A80000F8
:100060000CA900000CA900004CA8000050A800003A
:1000700054A8000058A800005CA800000CA90000CB
:1000800060A8000064A800000CA9000068A8000097
:100090006CA8000070A8000074A8000078A80000F8
:1000A0007CA8000080A8000084A8000088A80000A8
:1000B0000CA900000CA900000CA900008CA80000ED
:1000C00090A8000094A8000098A800009CA8000038
:1000D000A0A80000A4A80000A8A80000ACA80000E8
:1000E0000CA900000CA900000CA90000B0A8000099
:1000F000B4A800000CA900000CA90000B8A80000DA
:10010000BCA800000CA900000CA900000CA900006C
:100110000CA900000CA900000CA900000CA900000B
:10012000C0A800000CA900000CA90000C4A8000091
:10013000C8A80000CCA800000CA900000CA9000071
:100140000CA900000CA90000D0A800000CA9000018
:100150000CA900000CA900000CA90000D4A8000004
:100160000CA900000CA900000CA90000D8A80000F0
:10017000DCA80000E0A80000E4A80000E8A8000057
:10018000ECA80000F0A80000F4A80000F8A8000007
:10019000FCA8000000A9000004A9000008A90000B4
:1001A0000CA900000CA900000CA900000CA900007B
:1001B0000CA900000CA900000CA900000CA900006B
:1001C0000CA900000CA900000CA900000CA900005B
:1001D0000CA900000CA900000CA900000CA900004B
:1001E0000CA900000CA900000CA900000CA900003B
:1001F0000CA900000CA900000CA900000CA900002B
:10020800D2890200D2890200D2890200D289020072
:10021800D2890200D2890200D2890200D289020062
:10022800D2890200D2890200D2890200D289020052
:10023800D2890200D2890200D2890200D289020042
:10024800D2890200D2890200D2890200D289020032
:10025800D2890200D2890200D2890200D289020022
:10026800D2890200D2890200D2890200D289020012
:10027800D2890200D2890200D2890200D289020002
:10028800D2890200D2890200D2890200D2890200F2
:10029800D2890200D2890200D2890200D2890200E2
:1002A800D2890200D2890200D2890200D2890200D2
:1002B800D2890200D2890200D2890200D2890200C2
:1002C800D2890200D2890200D2890200D2890200B2
:1002D800D2890200D2890200D2890200D2890200A2
:1002E800D2890200D2890200D2890200D289020092
:1002F800D2890200D2890200D2890200D289020082
:10030800D2890200D2890200D2890200D289020071
:10031800D2890200D2890200D2890200D289020061
:10032800D2890200D2890200D2890200D289020051
:10033800D2890200D2890200D2890200D289020041
:10034800D2890200D2890200D2890200D289020031
:10035800D2890200D2890200D2890200D289020021
:10036800D2890200D2890200D2890200D289020011
:10037800D2890200D2890200D2890200D289020001
:10038800D2890200D2890200D2890200D2890200F1
:08039800D2890200D2890200A3
:020000040001F9
:1050000010A9040000000000D28904000200000082
:10501000D289040002000000D289040002000000CE
:10502000D289040002000000D289040002000000BE
:10503000D289040002000000D289040002000000AE
:10504000D289040002000000D2890400020000009E
:10505000D289040002000000D2890400020000008E
:10506000D289040002000000D2890400020000007E
:10507000D289040002000000D2890400020000006E
:10508000D289040002000000D2890400020000005E
:10509000D289040002000000D2890400020000004E
:1050A000D289040002000000D2890400020000003E
:1050B00096A8040001000000D2890400020000004C
:1050C000D289040002000000D2890400020000001E
:1050D000D289040002000000D2890400020000000E
:1050E000D289040002000000D289040002000000FE
:1050F000D289040002000000D289040002000000EE
:10510000D289040002000000D289040002000000DD
:10511000D289040002000000D289040002000000CD
:10512000D289040002000000D289040002000000BD
:10513000D289040002000000D289040002000000AD
:10514000D289040002000000D2890400020000009D
:10515000D289040002000000D2890400020000008D
:10516000D289040002000000D2890400020000007D
:10517000D289040002000000D2890400020000006D
:10518000D289040002000000D2890400020000005D
:10519000D289040002000000D2890400020000004D
:1051A000D289040002000000D2890400020000003D
:1051B000D289040002000000D2890400020000002D
:1051C000D289040002000000D2890400020000001D
:1051D000D289040002000000F6680400020000000A
:1051E000D289040002000000D289040002000000FD
:1051F000D289040002000000D289040002000000ED
:10520000D289040002000000D289040002000000DC
:10521000D289040002000000D289040002000000CC
:105220002FA821000EFF27000E01880000000000BB
:10523000000020000000E000020032000001200019
:10524000200288000C0007004058280021002000A0
:105250000F000700000020000000E0000200320004
:10526000000002000000000046B60200000000003E
:105270000040DA000000FE00801020000000E00086
:10528000020032001020200090018800000006007B
:10529000A1028800800078000000EB001A003700AF
:1052A000E280400054A0B4009101BA00E2804000C6
:1052B00054A0B4009102BA00E280400054A0B400AF
:1052C0000002EB00472BDE00F507B200A6018800C4
:1052D000602CE10008003A000049EB000201E80000
:1052E000020039003420EC0002F0A0008301E90044
:1052F000F9FF3E00040037006128E10001003200A0
:105300000082EB000B00070011C3BA001101BA00C4
:105310000604E00003003A000200E000E0FF3A006B
:1053200000000600F607B200A6028800820078009E
:10533000F5FF370004D0A300E20F49001C0039003C
:10534000810278003549BA000201E8000200390004
:105350003420EC0002F0A0008301E9000F003200CD
:105360002549BA000201E800020039003420EC00AF
:1053700002F0A0008301E900080032000400E00010
:105380000600320015C9BA000201E8000200390027
:105390003420EC0002F0A0008301E9008180E800E5
:1053A00054A0B4000300E000E2FF3A000000060051
:1053B0009102BA00055978008301E900F7FF320035
:1053C000C82ADE00055978008301E900F3FF3200A6
:1053D0000400E000F1FF320011D9BA00EEFF3700FF
:1053E0001C3B0400010000002800FA00889FBE005A
:1053F0008A9FBE008C9FBE000706780087866900E2
:105400000C003B00030478008704780008F0A1003A
:1054100009F0A100840F5000858F5800860F5900B5
:10542000890F5C00030033000CF0A20001003A0079
:105430000CF0A100A80107006400E1005F00320049
:10544000780147006408E100610032006C01470008
:10545000748557003200BE001201BE003A04BE003F
:105460001A05BE001E039000BE0A9000850353007B
:1054700006003D000004FD008104FD000205FD0062
:105480008305FD008703EA00050378000DF8A300FB
:105490000400320060041400E0841C0060051D005C
:1054A000E0851D006022B8007D0320000D38E1007A
:1054B0008006EB000B0039004433DD00F300B2003E
:1054C0008301730039003700848272000D02780076
:1054D000E10664008B85D1000A85D3008984D3005E
:1054E0000884D3008703E900F7FF3B000800400071
:1054F000898048000A0149008B81490004003B0073
:1055000060001000E080180060011900E0811900BF
:105510000358A300090032008D8272008482720059
:10552000610260008301D1000281D3008180D30039
:105530000080D3000603E8001B0037000348A300E7
:1055400017003A000600E000170034000603E900E7
:105550000D00A300000048008180480002014900BE
:10556000838149000348A3000F003A000600E000D1
:10557000090034000603E900000040008180480073
:10558000020149008381490001003A000003EB0059
:105590000348A300F5FF32006022B8000200370084
:1055A00084827200618266001F01070003F0A1007F
:1055B0000CF0A70003F0A0005B0137006401470076
:1055C0006408E10002003A000DF8A30053013A001C
:1055D0003200BE001201BE005301370003F0A200EA
:1055E000889FBE008A9FBE008C1F7800C5020700FE
:1055F000CC0233006450E1004F0032006420E1002F
:105600005200320003826C0007003B000905D00005
:105610000306D000820F54000C065D000200390022
:105620000200320089017800030678008582550067
:1056300004003D000003FD008103FD008502EA0037
:105640008B854200840F720002003B006000100056
:10565000E08018006011B8000005EB007A28E10036
:105660000A00390006007800C75DDD00F707B200C8
:10567000878075002D003700828171000A01780053
:10568000610560008180D1000080D3008502E900BF
:10569000F9FF3B00060440008784480002003B00FD
:1056A00060041400E0841C000988A3000700320095
:1056B0008A81710082817100610164008904D100D6
:1056C0000884D3008B05E800170037000978A30091
:1056D00013003A000B00E000130034008B05E900D2
:1056E0000804440089844C000A4474000978A3002B
:1056F0000D003A000B00E000070034008B05E900C4
:105700000804440089844C0001003A000B0020008A
:105710000978A300F7FF32000001EB000200370018
:10572000828171000A0178003B0207000CF0A7009B
:1057300001F0A000840237006420E10002003A007A
:10574000838F6C00840233000801BE000200BE009B
:105750007D0237008F1FD100D50307008F87E90036
:105760000000E00000000600809FEB00D00307006F
:105770008F87E9000000E000000006002800FA0022
:10578000889FBE008A9FBE008C9FBE0003866B0070
:10579000D10007006400E100440032006408E10029
:1057A0004A0032006100E100460032006108E10079
:1057B00049003200EC0647006000B8003D02BE0020
:1057C0003D03BE00F48657006011B8003D04BE00E2
:1057D0003D05BE007D0320000B0037000000A00047
:1057E0008D06E900130032000402420085824A005F
:1057F00006034B0087834B00000040008180480077
:1058000002014900838149000802520089825A003E
:105810000A035B008B835B00F0FF3B000802420041
:1058200089824A000A034B008B834B008D06E900F6
:10583000EDFF3A008482720086827200F707B200A0
:105840008782720001003200150020001E049000C3
:105850003E0B900006035400E63FB0000368A3002F
:10586000070032000000A7000500A0008301D1005E
:105870000281D3008180D3000080D3000603E800BA
:105880008301D1000281D3008180D3000080D30046
:105890000002EB000482D2006300070003F0A100C5
:1058A0000CF0A70003F0A0009F003700640247003F
:1058B0006408E100990032003400BE003401BE00EB
:1058C000F6FF37006108E100940032006011B80073
:1058D0006000B800F1FF370003FF2700020020003E
:1058E000FBFF3700889FBE008A9FBE008C1F780098
:1058F000040207000B02330003866C006450E100D1
:105900002E0032006420E100330032006150E100DB
:105910002F0032006120E100310032008585550002
:10592000EB07B00009002000080420000500370044
:105930000804440089844C000A0031000603430037
:1059400087834B000001530081815B00F8FF330027
:105950000203BE000800A0000804440089844C0033
:10596000F6FF3900C639DD00830173000100320003
:10597000130020008904D1000884D3000998A300F3
:10598000050032000800A7000300A0008904D10030
:105990000884D3008B05E8008904D1000884D30073
:1059A0000001EB000281D2009B01070001F0A10081
:1059B0000CF0A70001F0A000E30137006420E10033
:1059C000E50132000801BE000200BE00F7FF37000B
:1059D0006120E100E00132006000B800F3FF370011
:1059E0000000200001F82700F0FF3700839F6800C7
:1059F0000100E00002003D0060001000E08018009F
:105A00000300E00002003D0060011100E081190088
:105A1000AA0207004F00E00002003B0060001000F7
:105A2000E080180000000600180020005700200049
:105A3000080453000D003D000600200097FC2F00D5
:105A40000740E1001E0034008482720061026000A1
:105A50008301D1000281D3008180D3000080D30074
:105A60000804E800F8FF3A004700200061046000E5
:105A700005047400040464000D003200610040005D
:105A8000E080480060014900E081490003B8A500BA
:105A9000070032000603E8006538E10004003A0020
:105AA0008301D1000281D3008180D3000080D30024
:105AB000F87F20000830E10003003500080378007B
:105AC0006000B8006011B8004433DD00F300B2009C
:105AD0008301730000000600680447000294BE00C2
:105AE0000094BE00FC0447008694BE008494BE006F
:105AF0000900780037030700080078003503070025
:105B000099007800814F70000B003B000800BE0038
:105B1000100307004F00B10003003700F3FF270018
:105B2000F2FF2F006110B9004F06BE004F05BE0006
:105B30004F04BE000080FA000000060081037800D8
:105B40005B0107000001BE006000B8000478A300FC
:105B500013003A006220E10015003E000D003900FC
:105B60008301D1000281D3008180D3008301D10061
:105B70000281D3008180D3008301D1000281D30050
:105B80008180D3000538B000C42ADD00F300B200E4
:105B90008381720007F0A70003F0A0000000060058
:105BA000F3FF2700F2FF2F006110B900FBFF370061
:105BB00003FF2700F7FF3700140020002C033700F5
:105BC000F4FF2F002A0337001400FA00889FBE005C
:105BD0008A9FBE008C9FBE000004BE000205BE006E
:105BE000680047000A90BE000890BE00F902070056
:105BF0000070A7000BF0A1009E0990000E09900014
:105C0000FE0090006E0090009E0290003443200041
:105C1000848252000A00320010003C00B4FC2F00C5
:105C20000428E1001F0034008301D1000281D30069
:105C30008180D3000080D3008502E800FAFF3A009B
:105C40000B00E000B8FF3B0060001000E08018008F
:105C500060011900E0811900B3FF3700B400200093
:105C60000428E10007003D0000004000818048005A
:105C700002014900838149008502E900FAFF3A00E8
:105C8000EFFF3700F3FF2700F2FF2F006110B9008C
:105C90000B00E000A4FF3B000300280002002000EE
:105CA000010037006011B8006000B8009EFF3700A7
:105CB0001400FA00889FBE008A9FBE008C9FBE0021
:105CC0000004BE000205BE00680047000A90BE0046
:105CD0000890BE00BF0207000070A7000BF0A100F3
:105CE000304320009E02900080825200B0FE2F00C0
:105CF0000028E10011003D00B0FC2F000028E10069
:105D0000150034001E0990008E0890007E0090005F
:105D10000501B0000201D1008180D3000080D300D2
:105D20008502E800FBFF3A000B00E0007EFF3B002D
:105D300060001000E08018007BFF3700F0FF2F00AC
:105D4000F1FF27000B00E00077FF3B000100280077
:105D50000000200074FF37006000B80072FF3700B9
:105D60000001BE00D20007000470A70003F0A100EC
:105D70006509B100160032000D0035006828E10009
:105D800006003500F0FF2F00F1FF27000300E000C0
:105D900013003B0001002800000005000000400047
:105DA000818048008502E900FCFF3A0008003700C6
:105DB000F88F420002003C008000EB00000005006C
:105DC0008100D1000080D3008502E800FCFF3A008A
:105DD0000300E00002003B0060001000E0801800BB
:105DE000000006001400FA00889FBE008A9FBE00D3
:105DF0008C9FBE000004BE000205BE006800470084
:105E00000A90BE000890BE00720207000070A70052
:105E10000BF0A1000BF8A30016003A009E029000C0
:105E20003043200080825200B0FE2F000028E100A5
:105E30000D003C00B0FC2F000028E1000D003400F4
:105E40001E0990008E0890007E0090000501B000B1
:105E50000201D1008180D3000080D3008502E800D8
:105E6000FBFF3A0030FF370001002800000020004F
:105E70002DFF37006000B8002BFF37000001BE0087
:105E80008B0007000470A70003F0A10003F8A30033
:105E900013003A006509B100100032000900350016
:105EA0006928E1000200350001002800000005001B
:105EB00000004000818048008502E900FCFF3A00B4
:105EC00000000600F88F4200050035008100D10077
:105ED0000080D3008502E800FCFF3A0000000600C5
:105EE0008000EB0000000500881F780003047800A4
:105EF0000300E00007003D0060001000E080180093
:105F000060011900E081190002003B0001F02D0042
:105F1000030037000A00070008F0A70003F0A00004
:105F20004F047800000006004F89DE0082017800EF
:105F3000EDFF37004F89DE008201780067023700ED
:105F4000889FBE000082700004027100048271000C
:105F50002400320036432000C50020008383CF0098
:105F60000A0039000541B1008283CF0007003900E3
:105F70000541B1008183CF00040039000541B10023
:105F80008083CF00010039000541B10085C3530073
:105F90006022B800120032000A003B0084827200C6
:105FA000610260008301D1000281D3008180D300AF
:105FB0000080D3000603E8008743E800F7FF3A00BB
:105FC00007003700000040008180480002014900BE
:105FD000838149000603E9008743E900F9FF3A009D
:105FE00091FE07004F04BE00000006000002EB0017
:105FF0006B0107000500320007FF230006002000A8
:106000006022B80003F0A700FF00070000000600B0
:106010000400200016023700810020006180550036
:106020000B003D000B00200061FE2F000100E1008D
:106030001D00340082817100610164008904D10077
:106040000884D3000000E800FAFF3A007100200045
:10605000610064000300700002006000090032006B
:1060600061044400E0844C000988A500050032006A
:106070008B05E8006808E10002003A008904D100BD
:106080000884D300F20F20000258E10005003D0013
:10609000C75DDD00F907B20089807500080078004F
:1060A000000006000BF827008B00780000000500B8
:1060B000C70ADE00F107B200F50FB2000800320097
:1060C000E1CF4200020032000170A0002400050070
:1060D000810F700001003200040805004400050033
:1060E000810F700002003A00140005008502E900EB
:1060F0000000400081C04800FCFF3B000170A00090
:10610000240005000004BE00E9FF07000003BE00F4
:106110000405BE000200BE00E5FF0700844F7500C5
:10612000000006000200BE006450E10005003600D9
:106130006420E100020036000968A30001003A0073
:106140000800BE000160A0004F0678004F05BE00A9
:106150004F04BE0000000600F0FF2F00F1FF2700F3
:10616000F9FF37002800FA00889FBE008A9FBE0012
:106170008C9FBE0003866B0057FE07000028A3001B
:1061800064003A000128A30067003A000008A30059
:1061900062003A000108A30065003A001E0090006A
:1061A000BE08900081064000ED3FB100F48057002A
:1061B000EE019000111AB8008E099000311BB80052
:1061C0009E099000311CB800511DB800F48557009D
:1061D00046000700FE0190003A0007008B85E800AA
:1061E0003E0007008E09900040000700EE0190007D
:1061F000340007008B85E800380007008E09900006
:10620000400007009E0990001B18B8008904400058
:106210000A854800FE019000340007008B85E800E5
:1062200038000700EE019000300007008E09900052
:106230001B18B800890440000A8548000A98A3008A
:1062400008003A000402420085824A0006034B001F
:1062500087834B0008044C0089844C000A054D00DC
:106260008D06E90084827200850273004C3ADD00DD
:10627000850272000100320015002000443ADE0061
:106280001400B2004538DE00CB45DD000B00700085
:10629000C540DE00CB4DDD008B8070004549DE003F
:1062A000CB55DD000B017100C551DE000D037800F8
:1062B000DDFD070003F0A1000CF0A70003F0A00033
:1062C00019FE37001B18B8008502400006834800FD
:1062D000E0834B0060044C00070037001B18B80037
:1062E0000603400087834800FAFF37001B18B800F8
:1062F0008703400008844800E0844C0060054D009E
:10630000000006001B18B8000804400089844800FB
:10631000FAFF37000108A30000FE3A005800BE0053
:106320005801BE00E3FF37000008A300FBFD3A0060
:1063300009047800F9FF3700889FBE008A9FBE00DD
:106340008C1F78006FFF070076FF330003866C0018
:106350006450E100240032006420E1002700320094
:106360006150E100220032006120E1002100320092
:106370008B854200EB07B1000134B800003AB80049
:106380000804420089844A00013AB8000030B8008D
:106390008880400009014A000400330000004000EA
:1063A00081804800020149008B05E900C909DD0030
:1063B000830170000100320013002000C814DE00C9
:1063C0004814DD004709DE001200B200C808DE00F4
:1063D0000884700010FF070001F0A1000CF0A70076
:1063E00001F0A00058FF37006120E1005AFF3200A1
:1063F0000801BE000200BE00F7FF37006150E10057
:10640000FCFF3A0054FF370007F0A200F6FB37000C
:106410001400FA00889FBE008A9FBE008C9FBE00B9
:106420000005BE000206BE00680047000C90BE00DA
:106430000A90BE00E70007006400E1001A00320085
:1064400016003E006100E1001A0032006E04900068
:10645000FE0490000E0B90009E0B90006011B8009F
:106460009E0590000B38B100D5012000828171009B
:10647000610164008703D1000683D3008984D300BF
:106480000884D3008502E900F8FF3A00E2FE070025
:106490000DF0A70001F0A000A3FD3700F1FF2700D9
:1064A000F0FF2F00A0FD370001F8270000002000BA
:1064B000F7FF37006000B800F5FF37006022B80032
:1064C000060220000000D0008180D2000482D200A9
:1064D0008582D2000000A0000202520083825A008E
:1064E000030031000202420083824A000000A10042
:1064F0000603E900F3FF3A0000000600889FBE0093
:106500008A9FBE008C1F78000006EB00E00F500051
:10651000E08F5800E00F5900E08F590007003D0060
:106520006044B8006055B8000000540081805C00F1
:1065300002015D0083815D001C002000E00F52001D
:10654000E08F5A00E00F5B00E08F5B0007003D002A
:106550006044B8006055B8000402540085825C00B5
:1065600006035D0087835D000C00A2001A0107008E
:106570000C00E000060032006022B8006033B80072
:106580000000520081805A0002015B0083815B00A1
:106590004F0678004F05BE004F04BE000000060005
:1065A0001400FA00889FBE008A9FBE008C9FBE0028
:1065B00004067800E80247008292BE008092BE0086
:1065C00005007800830007006200E10033003A0014
:1065D0006000B8006011B8001E0390000C03530067
:1065E000F63FB100220035004B0320000B30E100E4
:1065F0002A003D00FB012000FAFF2F006154B90082
:106600006C0147008B05D1000A85D3008984D30033
:106610000884D3000603E900FAFF3B003200BE0005
:106620001201BE0000026400818264000203650062
:106630008383650005027200060272000702720081
:10664000160032000884EA008984EA000A85EA001C
:106650008B85EA000000640081806400020165000F
:10666000838165006022B8001E039000EEFC0700E5
:10667000DE03900007F0A70003F0A0000082EB000B
:106680000400E0008E0290004F06BE004F05BE00E1
:106690004F04BE000080FA000000060064014700BD
:1066A000040020003200BE001201BE00F4FF3700DB
:1066B000889FBE008A9FBE008C9FBE000404BE005F
:1066C0000605BE00809FBE00829FBE002F0007000F
:1066D000040678000800BE000A01BE002B00070077
:1066E000840678004F03BE004F02BE008D4F760037
:1066F0007FB0970013003300F0FF2F008B8F6B00EB
:1067000006003B000D0666000C00A7000A003700DB
:1067100007F0A600100020000A003700880F520082
:10672000898F5A008A0F5B008B8F5B000300390052
:106730001000200001003E000000200007F0A7002C
:106740000000EA004F06BE004F05BE004F04BE0029
:1067500000000600E48240001078A3000700320029
:10676000640240001178A3003400BE001401BE0092
:10677000040032000330A700000006003500BE0010
:106780001501BE000330A0000000060005FF270031
:1067900005826100070032000428E1000100320098
:1067A000240005000600070001003A00440005002F
:1067B0000408050002000700F9FF3A001400050074
:1067C0006F82610081027000850271008502720093
:1067D00000000600800078005002BE005003BE009A
:1067E0004439DE00F700B200F37F200003016100AE
:1067F000090032000218E10016003A00850172001B
:1068000083017300838173000008200015003A00A3
:1068100040002000130037008501720083017300DF
:106820008381730005003A0004A8BE0006A8BE00DC
:10683000100020000B0037000201E90004024200B2
:1068400085824A0006034B0087834B000748A3005C
:10685000F9FF32000740A00004A8BE0006A8BE0051
:1068600020002000800098009200980000000600A0
:10687000889FBE008A9FBE00841F780021FE07000B
:106880004F00780011003300F0FF2F00838F6C0061
:1068900006003B00040565000A00A7000800370059
:1068A00009F0A6001000200008003700820F5400F5
:1068B000838F5C00030039001000200001003E00BF
:1068C0000000200009F0A7000000EA004F05BE000C
:1068D0004F04BE000000E00000000600881F7800A2
:1068E000030478000300E00007003D006000100092
:1068F000E080180060011900E081190002003B00EF
:1069000001F02D00030037000400070008F0A70085
:1069100001F0A0004F04780000000600889FBE0030
:106920008A9FBE0000827000040271000482710020
:10693000260032000004BE000200BE006011B80054
:106940006B092000950220000182CF000A00390067
:106950000541B1000082CF00070039000541B100B8
:106960000982CF00040039000541B1000882CF0040
:10697000010039000541B100054252001200320009
:106980000A003B0082817100610164008100D10036
:106990000080D3008984D3000884D3008B05E800ED
:1069A0000442E800F7FF3A000700370008044400FB
:1069B00089844C0000004800818048008B05E90074
:1069C0000442E900F9FF3A0093FD07004F05BE00BD
:1069D0004F04BE0000000600889FBE008A9FBE00D4
:1069E0008C9FBE000404B8000506B8008904460068
:1069F00060854E000606B8000A054600E0854E0098
:106A00000706B8008B054600040EB800890446004E
:106A10000A854E00E0854D00050EB8000A054600C7
:106A20008B854E00060EB8008B0546000416B80094
:106A30000A0546008B854E000516B8008B054600FA
:106A4000041EB8008B0546000800BE000A01BE0007
:106A50004F06BE004F05BE004F04BE0000000600FA
:106A60008001780002003700815978000201E900B6
:106A70000200E000FCFF3A000000060012010000E6
:106A8000000200000200000000080000D80400001E
:106A90000A000000000100000102000003010000E4
:106AA00009020000430000000201000000C00000D5
:106AB0003209000004000000000100000202000092
:106AC0000100000005240000001000000104000087
:106AD000240200000205000024060000000100005E
:106AE00005240000010000000107000005810000EE
:106AF000030A00000001000009040000010000007A
:106B0000020A00000000000000070000050200006B
:106B100002400000000000000705000082020000A3
:106B20004000000000000000040300000904000011
:106B300028030000520000006F00000074000000F5
:106B4000720000006F0000006E000000690000008D
:106B5000630000002000000041000000470000002A
:106B60002F00000056000000430000005400000009
:106B7000200000004C0000007400000064000000D1
:106B80001A030000410000007700000054000000DC
:106B90006800000065000000720000006D00000049
:106BA0002000000076000000310000002E000000F0
:106BB00030000000140300004100000077000000D6
:106BC0002D000000760000003000000030000000C2
:106BD0002E000000330000003300000050B500001C
:106BE00094B5000098B50000C0B50000DAB500000B
:106BF0007B4600003939000052440000447D00000B
:106C00000D00000008000000000000000F00000060
:106C10001000000015000000900000002800000097
:106C20000200000058000000080000000000000002
:106C30000F00000010000000150000009000000090
:106C400028000000020000005C000000303100005D
:106C50003233000034350000363700003839000088
:106C6000414200004344000045460000303100002E
:106C70003233000034350000363700003839000068
:106C80004142000043440000454600000200FA0073
:106C90000060FE00A4790700417A0700B86C02008A
:106CA0000200000003003700000000000100370070
:106CB000000000000060FE009E7A0700000E210028
:106CC00010407800E14F500001003A00C17C0700FD
:106CD00080802000104078000004E00014003A009A
:106CE000014307000080200010407800E14F500071
:106CF00001003A00607C070090802000104078007E
:106D00008040E800908020000148780090802000BA
:106D10009040780030C6B30080CF5000E2FF3400CE
:106D20008080200011C0B30001487800E1FF3700E7
:106D30006000B80010A2880021A288003C40070033
:106D4000104798001E4090009E4F500009003A00E6
:106D50009E409000014F7800E34207000080200031
:106D600010407800E14F5000D1FF3A00427C07000C
:106D7000D0FF37009E409000014F78007E3F070013
:106D8000D00D21008040EB0001487800D535070088
:106D9000E14F500034003A00B43902000200000014
:106DA000800D2100104078000004E00007003A0048
:106DB00082350700D36F070015780700900D21007A
:106DC0008040EB000148780022003700CD6F0700BB
:106DD0000F7807000080200010407800E14F50003D
:106DE00004003A00A83E0200020000005A360700E4
:106DF000CA7B0700C00D210010407800F44F5000FE
:106E00000A003C00507C8000617C8000507B880040
:106E1000617B8800C00D2100104078008040E800B0
:106E2000C00D2100014878000A003700B00D210094
:106E30008040EB00014878006000B800507B88007B
:106E4000617B88005D350700C00D210051C1B30092
:106E500001487800B00D210011C0B300014878004E
:106E60000060FE0093FF3700C00D21001040780045
:106E70000004E0000B00320030CBB3002E410700CD
:106E800030C1B3002C410700A0C0B3002A41070065
:106E9000D603020002000000C00D21008040EB007C
:106EA00001487800800E2100104078000004E000C6
:106EB00075003A00D00D2100104078000004E00079
:106EC00001003A003D3507008E6F0700B10307004F
:106ED00080F02000104078000004E000050032003F
:106EE0005A41020002000000624E0200020000004F
:106EF000E50F070010CBB3000F41070000C1B3003E
:106F00000D410700D0C0B3000B4107006625020009
:106F1000020000000080200010407800E14F500087
:106F200002003A000C3607007C7B07005B33070049
:106F3000C0802000104078008040E800C080200021
:106F400001487800C0802000104078008000FB00DD
:106F5000C04F2100104078000000FB00630040009B
:106F6000808F500006003A00A08020008040EB0097
:106F700001487800C08020008040EB000148780084
:106F8000A0802000104078000004E00033003A00A8
:106F9000C0802000104078000004E0002B003A0080
:106FA000C00E210010407800E14F500003003A006D
:106FB0008002020002000000020037003C020200D2
:106FC0000200000060F02000104078000004E000A3
:106FD00003003A005A410200020000001B00370083
:106FE00060F0200010407800E14F500003003A00AC
:106FF000BC490200020000001400370060F02000CD
:1070000010407800E24F500003003A00984602001A
:10701000020000000D00370060F0200010407800F2
:10702000E44F500003003A00A447020002000000B1
:107030000600370060F0200010407800E84F500054
:1070400002003A00B048020002000000C0802000A8
:107050008040EB000148780006003700C080200027
:1070600010407800E14F500002003A000240020058
:1070700002000000D00D210011C0B30001487800CB
:107080000060FE000BFF37000080200010407800F9
:10709000E14F500003003A00CC3E02000200000025
:1070A0001E7B0700E00D210010407800E14F5000EA
:1070B00008003A00F00D21008040EB000148780004
:1070C000D607070087000700E00D21008040EB0095
:1070D00001487800800D210011C0B30001487800FC
:1070E000086F07009C350700D0EA200010407800A8
:1070F000E64F500002003A00CF0807007900070071
:10710000E04C2100104078000004E00009003A0043
:1071100020030700D4030700D0A48000E1A480006E
:10712000B0AE02000000000080407800E04C21007A
:1071300001487800E04C2100104078008040E900D0
:10714000E04C210001487800E04C2100104078001C
:107150000004E00003003D00E04C21008040EB0013
:1071600001487800130E0700CC320700C0802000D1
:10717000104078008040E800C0802000014878007E
:10718000C0802000104078008000FB00C04F21002C
:10719000104078000000FB0063004000808F50002A
:1071A00003003A00A08020008040EB0001487800F6
:1071B000A0802000104078000004E0003F003A006A
:1071C000C0802000104078008000FB00C04F2100EC
:1071D000104078000000FB0063004000808F5000EA
:1071E0002B003A00C00E210010407800E14F500003
:1071F00003003A0080020200020000000200370093
:107200003C0202000200000060F020001040780004
:107210000004E00003003A005A41020002000000AE
:107220001B00370060F0200010407800E14F500054
:1072300003003A00BC4902000200000014003700BD
:1072400060F0200010407800E24F500003003A0048
:1072500098460200020000000D00370060F0200098
:1072600010407800E44F500003003A00A4470200A9
:10727000020000000600370060F020001040780097
:10728000E84F500002003A00B0480200020000003F
:10729000C08020008040EB0001487800C00E210033
:1072A00010407800E14F500002003A0091130700AF
:1072B00080FE37002F0F07007EFE3700C0802000C1
:1072C00010407800E14F500002003A0002400200F6
:1072D00002000000EC0E0700624E020002000000F7
:1072E00074FE37000200FA00800E210011C0B300C6
:1072F00001487800E04C21008040EB000148780014
:107300006000B800A0A68800B1A688006000B800A0
:10731000C0A68800D1A688006000B800E0A688005A
:10732000F1A688006000B80000A7880011A78800B7
:107330006000B80020A7880031A788006000B8006E
:1073400040A7880051A788006000B80060A78800A7
:1073500071A78800C4F320006000B8006011B80075
:10736000009ABE000292BE00C0EA20008040EB00FE
:10737000014878006000B800507B8800617B88007D
:107380000040EB00004F7800070037001E00FB00B4
:10739000C200DD0020F72000008140006000B8003E
:1073A0000089BE001E4FE8001E407800E54F5000E7
:1073B000F6FF34006000B800707B8800817B880095
:1073C0006000B800307C8800417C88006000B80014
:1073D000507C8800617C8800E0F820008040EB0051
:1073E00001487800F0F820008040EB000148780068
:1073F00000F920008040EB00014878000080FA008E
:10740000000006000000FA00D9E2A9002136800041
:10741000F00F2C00808060000060210001007000EF
:107420002036880021E1A900DDE2A900B821EF00A3
:10743000BE21EF00F00F2000E00D880060C02000AA
:10744000C00D8800C0082000D00D88000009800011
:107450000040A0000050A1000009880021E1A80020
:1074600061E2A9004136800000FC2F00008060002E
:10747000A000B3004036880051368000F00F2C0089
:107480008080600000B0200001007000503688004D
:10749000C922A900C902A900D802A900CD22A800CA
:1074A0006022EF00101380000020A1000030A10036
:1074B0000040A10010138800101380000000A000FD
:1074C0000010A0001013880062A2A80062E2A900C8
:1074D0006422EF006822EF006342A9006302A90062
:1074E00062C2A8006322A90061E2A800CD22A9001F
:1074F00000000000BE21EF0000E120008040EB0012
:10750000014878000D00370000E1200010407800AD
:107510000000FB0011E12000614078000000FB004A
:10752000B88802000200000000E12000104078004E
:107530008040E80000E120000148780000E12000E0
:1075400010407800E14F5000EFFF34000080FA0057
:10755000000006000000FA00B00F21001040780083
:107560000000FB00E10F500020003200E10F50004E
:1075700003003C000000E000060032005D00370020
:10758000E20F50002F003200E30F500043003200A2
:107590005800370000E120008040EB0001487800EF
:1075A0000D00370000E12000104078000000FB00D3
:1075B00011E12000614078000000FB00B888020063
:1075C0000200000000E12000104078008040E80048
:1075D00000E120000148780000E120001040780020
:1075E000E14F5000EFFF34004200370000E120007F
:1075F0008040EB00014878000D00370000E12000DA
:10760000104078000000FB00E16F2100614078002D
:107610000000FB00B88802000200000000E120002A
:10762000104078008040E80000E120000148780028
:1076300000E1200010407800E14F5000EFFF3400DF
:107640002C00370000E120008040EB00014878006A
:107650000D00370000E12000104078000000FB0022
:1076600001702100614078000000FB00B888020032
:107670000200000000E12000104078008040E80097
:1076800000E120000148780000E12000104078006F
:10769000E14F5000EFFF34001600370000E12000FA
:1076A0008040EB00014878000D00370000E1200029
:1076B000104078000000FB0021702100614078003C
:1076C0000000FB00B88802000200000000E120007A
:1076D000104078008040E80000E120000148780078
:1076E00000E1200010407800E14F5000EFFF34002F
:1076F00000000000F0072000F00D8800147607005D
:10770000BE21EF0000E120008040EB00014878003E
:107710000D00370000E12000104078000000FB0061
:1077200011E12000614078000000FB00B8880200F1
:107730000200000000E12000104078008040E800D6
:1077400000E120000148780000E1200010407800AE
:10775000E14F5000EFFF34000080FA000000060007
:107760000000FA00B0422100104078000000FB0049
:10777000E10F500020003200E10F500003003C00F8
:107780000000E000060032005D003700E20F50000C
:107790002F003200E30F5000430032005800370042
:1077A00000E120008040EB00014878000D00370028
:1077B00000E12000104078000000FB0011E12000F3
:1077C000614078000000FB00B88802000200000061
:1077D00000E12000104078008040E80000E1200037
:1077E0000148780000E1200010407800E14F50008F
:1077F000EFFF34004200370000E120008040EB0042
:10780000014878000D00370000E1200010407800AA
:107810000000FB00E16F2100614078000000FB00E8
:10782000B88802000200000000E12000104078004B
:107830008040E80000E120000148780000E12000DD
:1078400010407800E14F5000EFFF34002C0037006B
:1078500000E120008040EB00014878000D00370077
:1078600000E12000104078000000FB0001702100C2
:10787000614078000000FB00B888020002000000B0
:1078800000E12000104078008040E80000E1200086
:107890000148780000E1200010407800E14F5000DE
:1078A000EFFF34001600370000E120008040EB00BD
:1078B000014878000D00370000E1200010407800FA
:1078C0000000FB0021702100614078000000FB00F7
:1078D000B88802000200000000E12000104078009B
:1078E0008040E80000E120000148780000E120002D
:1078F00010407800E14F5000EFFF3400000000001E
:10790000F0072000F00D8800A1750700BE21EF00F0
:1079100000E120008040EB00014878000D003700B6
:1079200000E12000104078000000FB0011E1200081
:10793000614078000000FB00B888020002000000EF
:1079400000E12000104078008040E80000E12000C5
:107950000148780000E1200010407800E14F50001D
:10796000EFFF34000080FA00000006000000FA007B
:10797000E0422100104078000000FB00E10F5000C1
:1079800020003200E10F500003003C000000E00046
:10799000060032005D003700E20F50002F00320079
:1079A000E30F5000430032005800370000E1200090
:1079B0008040EB00014878000D00370000E1200016
:1079C000104078000000FB0011E1200061407800C9
:1079D0000000FB00B88802000200000000E1200067
:1079E000104078008040E80000E120000148780065
:1079F00000E1200010407800E14F5000EFFF34001C
:107A00004200370000E120008040EB000148780090
:107A10000D00370000E12000104078000000FB005E
:107A2000E16F2100614078000000FB00B88802008F
:107A30000200000000E12000104078008040E800D3
:107A400000E120000148780000E1200010407800AB
:107A5000E14F5000EFFF34002C00370000E1200020
:107A60008040EB00014878000D00370000E1200065
:107A7000104078000000FB00017021006140780098
:107A80000000FB00B88802000200000000E12000B6
:107A9000104078008040E80000E1200001487800B4
:107AA00000E1200010407800E14F5000EFFF34006B
:107AB0001600370000E120008040EB00014878000C
:107AC0000D00370000E12000104078000000FB00AE
:107AD00021702100614078000000FB00B88802009E
:107AE0000200000000E12000104078008040E80023
:107AF00000E120000148780000E1200010407800FB
:107B0000E14F5000EFFF340000000000F0072000BC
:107B1000F00D88001E750700BE21EF0000E1200077
:107B20008040EB00014878000D00370000E12000A4
:107B3000104078000000FB0011E120006140780057
:107B40000000FB00B88802000200000000E12000F5
:107B5000104078008040E80000E1200001487800F3
:107B600000E1200010407800E14F5000EFFF3400AA
:107B70000080FA00000006000000FA00C8A2A90078
:107B8000CCA2A8000080FA00000006000200FA0063
:107B90006000B80050848800618488006000B800EC
:107BA0007084880081848800200921008040EB00D7
:107BB00001487800300921008040EB00014878003E
:107BC000400921008040EB00014878000040EB00B4
:107BD000004F7800070037001E00FB00C200DD00E8
:107BE000A0F92000008140006000B8000089BE00BC
:107BF0001E4FE800C0C3B3009E40780080CF500005
:107C0000F5FF340011368000F00F2C0080806000FA
:107C10000050210001007000103688001FE1A9000B
:107C2000DD42A900D942A900AE21EF00B021EF004A
:107C300000002000A14F2400B07C8800C17C880097
:107C4000B07C8000C17C80003EAF020000000000DC
:107C500000007800A00D88000080EB00900D8800E7
:107C600060802000700D8800C0082000800D880012
:107C7000F00880000040A0000050A100F00888003B
:107C80001FE1A8000080FA00000006000000FA00D2
:107C90002136800000FC2F00008060002001B3002E
:107CA000203688006136800000FC2F0000806000D4
:107CB0003001B3006036880011E1A900DD22A9007F
:107CC000DD62A900D922A900D962A9009021EF00A4
:107CD0009C21EF006000B800307B8800417B880069
:107CE000307B8000417B80003EAF0200000000003E
:107CF00000007800B00C88000080EB00A00C880029
:107D0000307B8000417B80003EAF0200000000001D
:107D100000007800000D88000080EB00F00C880067
:107D200060002000800C8800C0082000900C8800B3
:107D300060002000D00C8800C0082000E00C880003
:107D4000800880000040A0000050A100800888004A
:107D500011E1A8000080FA00000006000000FA000F
:107D600040E220008040EB0001487800F0A5800050
:107D700001A680005071880061718800D0A5800044
:107D8000E1A5800010728800217288000080FA004E
:107D9000000006001000FA00889FBE008A9FBE0007
:107DA00080F52000104078000004E00004003A0054
:107DB00080F5200011C0B300014878008B00370027
:107DC000F0A5800001A680009EAD0200000000002A
:107DD0000004BE000205BE0000F520003002BE0017
:107DE0002003BE00049FBE000697BE00A0F0200046
:107DF0005001BE004000BE000002BE000203BE00F3
:107E00003E00BE002E01BE0004B2020000000000D1
:107E10000002BE000203BE000800BE000A01BE0050
:107E2000B2B002000000000008B202000000000032
:107E300001F0A100007188001171880004718000B8
:107E40001571800010A6800021A6800018C0B30024
:107E50000001BE000400BE00E0AD02000000000012
:107E60000000E00001003C000044EB000804E000DA
:107E70000500320010A6800021A680000071880055
:107E800011718800120037000471800015718000A4
:107E900030A6800041A6800018C0B3000001BE00DB
:107EA0000400BE00DCAD0200000000000000E000A5
:107EB000010035000044EB000804E000040032003B
:107EC00030A6800041A680000071880011718800F2
:107ED000D4A58000E5A580000071800011718000AC
:107EE0000001BE000400BE0072AC020000000000F1
:107EF0000200200003F82300F0AA020000000000A6
:107F00000001BE000000200001F8230072AC020056
:107F100000000000E0708800F1708800E0708000D0
:107F2000F17080000001BE000000200001F8230075
:107F3000EEAA0200000000009EAD0200000000005A
:107F40000004BE000205BE0000F520005001BE0086
:107F50004000BE000002BE000203BE000800BE00DA
:107F60000A01BE00B2B00200000000000004BE0022
:107F70000205BE00E0708000F17080009EAD02003E
:107F8000000000000002BE000203BE00440798008B
:107F9000550798006607980077079800A0F0200022
:107FA0005001BE004000BE000002BE000203BE0041
:107FB0004E009000DE0090006E019000FE019000E7
:107FC000B2B00200000000000002BE000203BE00CA
:107FD0000800BE000A01BE00F4A902000000000073
:107FE000A4F02000009ABE000292BE00A0F0200083
:107FF0005001BE004000BE0004F52000009ABE0003
:108000000292BE00A0F020005001BE004000BE0061
:1080100008B20200000000007071880081718800C1
:10802000A0F020005001BE004000BE0044F320003C
:10803000009ABE000292BE0040F320005001BE0034
:108040004000BE00BC350200020000004F05BE002B
:108050004F04BE000080FA00000006000000FA0095
:108060000080FA00000006003000FA00889FBE0081
:108070008A9FBE008C1F7800207A8000317A8000B1
:108080009AAF02000000000002002000A347240075
:1080900072AC020000000000000F9800110F980061
:1080A000209E8000319E800018C0B3000E09900011
:1080B0009E099000E0AD0200000000000000E0001A
:1080C00001003C000044EB000804E0002000320006
:1080D000209E8000319E80000E0990009E09900035
:1080E000EEAA0200000000000002BE0050A68000C0
:1080F00061A680000001BE000400BE0072AC020058
:10810000000000000001BE000000200001F8230074
:10811000EEAA0200000000000002BE0090A5800050
:10812000A1A580000001BE000400BE009CB10200B9
:10813000000000009EAD0200000000004007980013
:1081400051079800620798007307980008003700ED
:1081500090A58000A1A580009EAD02000000000057
:10816000400798005107980062079800730798002D
:10817000209E8000319E800018C0B3000E09900040
:108180009E099000DCAD0200000000000000E0004D
:10819000010035000044EB000804E0001D0032003F
:1081A000209E8000319E80000E0990009E09900064
:1081B000EEAA0200000000000002BE0050A68000EF
:1081C00061A680000001BE000400BE0072AC020087
:1081D000000000000200200003F82300F0AA0200C3
:1081E000000000000002BE00B0A58000C1A5800014
:1081F0000001BE000400BE009CB1020000000000AF
:108200009EAD020000000000009FBE000297BE006D
:1082100006003700B0A58000C1A580009EAD020019
:1082200000000000009FBE000297BE00809E8000FC
:10823000919E800018C0B300020020000327240094
:10824000E0AD0200000000000000E00001003C0082
:108250000044EB000804E0001D003200809E800016
:10826000919E80000E0990009E099000EEAA0200E7
:10827000000000000002BE0050A6800061A6800041
:108280000001BE000400BE0072AC0200000000004D
:108290000001BE000000200001F82300EEAA020049
:1082A000000000000002BE00B0A58000C1A5800053
:1082B0000001BE000400BE009CB1020000000000EE
:1082C0009EAD020000000000009FBE000297BE00AD
:1082D0000E0890009E0890009EAD02000000000075
:1082E0000004BE000205BE00A0F020005001BE0048
:1082F0004000BE000002BE000203BE000800BE0037
:108300000A01BE0004B2020000000000A4E6200042
:10831000009ABE000292BE00A0E620005001BE00FE
:108320004000BE0024E72000009ABE000292BE007A
:1083300070A4800081A480009EAD020000000000B7
:108340000004BE000205BE00A0E620005001BE00F1
:108350004000BE000002BE000203BE000800BE00D6
:108360000A01BE00B2B002000000000008B2020024
:108370000000000080A6880091A6880010A580005B
:1083800021A580009EAD0200000000000004BE0098
:108390000205BE00A0E620005001BE004000BE0065
:1083A0001CC0B3000002BE000203BE000800BE00F5
:1083B0000A01BE00AAAB0200000000000000E000BD
:1083C000010035000046EB000C04E00016003A0006
:1083D00030A5800041A5800001F0A2009EAD020002
:1083E000000000000004BE000205BE00A0E6200060
:1083F0005001BE004000BE001CC0B3000002BE0021
:108400000203BE000800BE000A01BE00B4AB0200B9
:10841000000000000000E00001003C000046EB000E
:108420000C04E000040032006000B800C0A6880020
:10843000D1A688008400370090A48000A1A4800009
:108440009EAD0200000000000004BE000205BE0058
:1084500000A7800011A780009EAD02000000000070
:108460000002BE000203BE00041798001517980012
:108470002617980037179800A0E620005001BE008C
:108480004000BE000002BE000203BE000E109000BD
:108490009E1090002E119000BE119000F4A90200D1
:1084A000000000000002BE000203BE000800BE0083
:1084B0000A01BE00B2B00200000000000004BE00CD
:1084C0000205BE00E0A68000F1A680009EAD02007D
:1084D000000000000002BE000203BE000800BE0053
:1084E0000A01BE00F4A902000000000008B2020068
:1084F00000000000C0A68800D1A68800C4A68000A5
:10850000D5A6800080A6800091A680000001BE0054
:108510000400BE00F0AA020000000000200F980036
:10852000310F98002E089000BE0890009EAD02000A
:108530000000000018C0B3004E029000DE02900060
:108540006E039000FE039000B4AB02000000000038
:108550000000E00001003C000044EB000804E000E3
:108560001100320080A6800091A680009EAD02001E
:10857000000000000002BE000203BE004E0090009A
:10858000DE0090006E019000FE01900004B2020037
:108590000000000008B2020000000000E0A6880011
:1085A000F1A68800210037002E089000BE08900038
:1085B0009EAD02000000000018C0B3003E02BE00E5
:1085C0002E03BE00AAAB0200000000000000E00085
:1085D000010035000044EB000804E0000F00320009
:1085E00080A6800091A680009EAD020000000000E1
:1085F0000002BE000203BE003E00BE002E01BE000F
:1086000004B202000000000008B2020000000000F6
:10861000E0A68800F1A6880004003700C0A680000C
:10862000D1A68000E0A68800F1A68800A0E6200080
:108630005001BE004000BE0008B202000000000071
:1086400000A7880011A7880050A5800061A58000C0
:108650009EAD0200000000000004BE000205BE0046
:10866000A0E620005001BE004000BE001CC0B300C8
:108670000002BE000203BE000800BE000A01BE00E8
:10868000AAAB0200000000000000E000010035007D
:108690000046EB000C04E00016003A0070A58000D4
:1086A00081A5800001F0A2009EAD02000000000044
:1086B0000004BE000205BE00A0E620005001BE007E
:1086C0004000BE001CC0B3000002BE000203BE009A
:1086D0000800BE000A01BE00B4AB020000000000AA
:1086E0000000E00001003C000046EB000C04E0004C
:1086F000040032006000B80040A7880051A788003D
:108700002A003700B0A48000C1A480009EAD020002
:10871000000000000004BE000205BE00A0E620002C
:108720003002BE002003BE00441798005517980081
:10873000661798007717980060A7800071A78000DF
:108740009EAD0200000000000002BE000203BE0059
:108750004E109000DE1090006E119000FE119000FF
:1087600004B20200000000000002BE000203BE00CE
:108770000800BE000A01BE00B2B002000000000006
:1087800008B202000000000040A7880051A788003E
:10879000A0E620005001BE004000BE0008B202006A
:1087A0000000000060A7880071A7880084A68000F0
:1087B00095A68000C0A68000D1A680000001BE0062
:1087C0000400BE00F0AA0200000000000002BE008B
:1087D00040A7800051A780000001BE000400BE0039
:1087E000F0AA020000000000507B8800617B880036
:1087F000507B8000617B80009EAD02000000000085
:1088000018C0B3004E029000DE0290006E0390008C
:10881000FE039000B4AB0200000000000000E00086
:1088200001003C000044EB000804E00008003200B6
:108830004E009000DE0090006E019000FE0190005E
:1088400008B2020000000000507B8800617B8800B5
:10885000507B8000617B80009EAD02000000000024
:1088600018C0B3003E02BE002E03BE00AAAB020039
:10887000000000000000E000010035000044EB00B3
:108880000804E000060032003E00BE002E01BE00DB
:1088900008B2020000000000507B8800617B880065
:1088A000507B8000617B800018C0B3006011B8006D
:1088B000E0AD0200000000000000E00001003C000C
:1088C0000044EB000804E0000A003200547B800002
:1088D000657B8000F0A4800001A580000001BE003F
:1088E0000400BE009CB1020000000000507B880024
:1088F000617B8800507B8000617B800018C0B300E2
:1089000002F02F00F3772C00DCAD02000000000025
:108910000000E000010034000044EB000804E00027
:108920000400320000F02F00F1772C00507B88000B
:10893000617B8800507B8000617B800018C0B300A1
:1089400002F02F00F3772400E0AD020000000000E9
:108950000000E00001003D000044EB000804E000DE
:108960000400320000F02F00F1772400507B8800D3
:10897000617B8800D0EA200010407800E54F50006D
:1089800052003A0060A720005001BE004000BE0027
:108990006022B80006802800370C2400B2B0020024
:1089A0000000000008B20200000000000004BE0049
:1089B000E0A720005001BE004000BE006022B800C9
:1089C00006002400F7082400B2B0020000000000F6
:1089D00008B20200000000000001BE000800BE0056
:1089E000F0AA0200000000000004BE0060A8200001
:1089F0005001BE004000BE006022B800060020000A
:108A000097052400B2B002000000000008B2020086
:108A1000000000000001BE000800BE00F0AA020035
:108A2000000000000004BE00E0A820005001BE00CD
:108A30004000BE006022B80006002000470224006B
:108A4000B2B002000000000008B202000000000006
:108A50000001BE000800BE00F0AA020000000000F5
:108A60000004BE0060A920005001BE004000BE000E
:108A700008B20200000000000001BE000800BE00B5
:108A8000F0AA020000000000907C8800A17C880011
:108A9000E0A620005001BE004000BE006022B800E9
:108AA0000600280067042400AAAB020000000000B2
:108AB0000000E00005003A00907C8000A17C80006E
:108AC00001F0A200907C8800A17C8800D0EA200000
:108AD00010407800E54F5000F0003A00907C800094
:108AE000A17C800002F82400337C24009CB10200A9
:108AF0000000000002F02F00F377240072AC0200A7
:108B0000000000009EAD020000000000400F980031
:108B1000510F9800620F9800730F98004E08900054
:108B2000DE0890006E099000FE09900003F0A1009D
:108B3000400F9800510F9800620F9800730F980033
:108B40006022B80006802800370C24004E089000F0
:108B5000DE0890006E099000FE099000BEAB020096
:108B60000000000058AE0200000000000000780085
:108B70001086880011868000007122000088B900EC
:108B800000007800CF80DE0094AF020000000000FB
:108B90000002BE000203BE004E089000DE089000F6
:108BA0006E099000FE09900004B20200000000006F
:108BB00058AE02000000000000007800CF80DE0008
:108BC00094AF0200000000006022B80006002400FC
:108BD000F7082400BEAB02000000000058AE0200FF
:108BE00000000000000078002086880011868000C8
:108BF000007122000088B90000007800CF80DE00FC
:108C000094AF0200000000000002BE000203BE009C
:108C10004E089000DE0890006E099000FE0990005A
:108C200004B20200000000000004BE000205BE0005
:108C300021868000803E20000088B9000000780076
:108C4000CF80DE0094AF0200000000000002BE00F2
:108C50000203BE000800BE000A01BE0004B202000A
:108C60000000000058AE0200000000000000780084
:108C7000CF80DE0094AF0200000000006022B80048
:108C80000600200097052400BEAB02000000000093
:108C900058AE020000000000000078003086880016
:108CA00011868000007122000088B9000000780061
:108CB000CF80DE0094AF0200000000000002BE0082
:108CC0000203BE004E089000DE0890006E0990007E
:108CD000FE09900004B20200000000000004BE0083
:108CE0000205BE0021868000803E20000088B90079
:108CF00000007800CF80DE0094AF0200000000008A
:108D00000002BE000203BE000800BE000A01BE0051
:108D100004B20200000000000004BE000205BE0014
:108D200031868000400620000088B90000007800ED
:108D3000CF80DE0094AF0200000000000002BE0001
:108D40000203BE000800BE000A01BE0004B2020019
:108D50000000000058AE0200000000000000780093
:108D6000CF80DE0094AF0200000000006022B80057
:108D70000600200047022400BEAB020000000000F5
:108D800058AE020000000000000078004086880015
:108D900011868000007122000088B9000000780070
:108DA000CF80DE0094AF0200000000000002BE0091
:108DB0000203BE004E089000DE0890006E0990008D
:108DC000FE09900004B20200000000000004BE0092
:108DD0000205BE0021868000803E20000088B90088
:108DE00000007800CF80DE0094AF02000000000099
:108DF0000002BE000203BE000800BE000A01BE0061
:108E000004B20200000000000004BE000205BE0023
:108E100031868000400620000088B90000007800FC
:108E2000CF80DE0094AF0200000000000002BE0010
:108E30000203BE000800BE000A01BE0004B2020028
:108E4000000000000004BE000205BE004086800055
:108E50006A00B90000007800CF80DE0094AF020005
:108E6000000000000002BE000203BE000800BE00B9
:108E70000A01BE0004B202000000000058AE020069
:108E8000000000000000780050868800907C800080
:108E9000A17C8000507B8800617B8800507B800033
:108EA000617B8000707B8800817B8800E0F8200077
:108EB00010407800E44F50000F003C00E0F8200024
:108EC000104078000001FB00507B8000617B800037
:108ED000C211DD0022F72000028141000089BE009E
:108EE000E0F82000104078008040E800E0F8200022
:108EF0000148780015003700F0F820001040780095
:108F00000001FB00507B8000617B8000C211DD000E
:108F100022F72000028141000089BE00F0F8200005
:108F2000104078008040E800F0F820000148780008
:108F3000F0F8200010407800E54F500003003A00A0
:108F4000F0F820008040EB00014878006000B80095
:108F5000307C8800417C880000F920008040EB00D4
:108F6000014878001400370000F920001040780014
:108F70000000FB00C200DD0020F720000080400060
:108F80001002BE00307C8000417C80000001BE00E9
:108F90000400BE00F0AA020000000000307C88003F
:108FA000417C880000F92000104078008040E800F3
:108FB00000F920000148780000F920009040780076
:108FC000E0F820001040780080CF5000E6FF350028
:108FD000387C8000497C8000E0F820001040780058
:108FE0000000FB00CF80DE009AAF0200000000000E
:108FF0000001BE000800BE0072AC020000000000CC
:10900000507C8800617C88004F0678004F05BE00C8
:109010004F04BE000080FA00000006000200FA00C3
:10902000227A8000337A8000D0D72100010020000E
:10903000800F5100818F590012003C000040EB006E
:10904000004F78000B0037001E81FB001E80FB00E4
:10905000C200DD0040702100008040001000BE0012
:10906000C211DD0062442100028141000089BE007E
:109070001E4FE8001E407800F04F5000F2FF36000F
:10908000A7003700227A8000337A8000D0CB2300FB
:1090900001002000800F5100818F590012003C0018
:1090A0000040EB00004F78000B0037001E81FB00F2
:1090B0001E80FB00C200DD008074210000804000A3
:1090C0001000BE00C211DD00624421000281410097
:1090D0000089BE001E4FE8001E407800F04F50008F
:1090E000F2FF36008E003700227A8000337A80004B
:1090F000D0B9260001002000800F5100818F590057
:1091000012003C000040EB00004F78000B003700DD
:109110001E81FB001E80FB00C200DD00C078210024
:10912000008040001000BE00C211DD00624421003A
:10913000028141000089BE001E4FE8001E407800F9
:10914000F04F5000F2FF360075003700227A8000A1
:10915000337A8000D02A290001002000800F5100BE
:10916000818F590012003C000040EB00004F780056
:109170000B0037001E81FB001E80FB00C200DD00DB
:10918000007D2100008040001000BE00C211DD0003
:1091900062442100028141000089BE001E4FE800A8
:1091A0001E407800F04F5000F2FF36005C003700A0
:1091B000227A8000337A8000D09B2B0001002000AF
:1091C000800F5100818F590012003C000040EB00DD
:1091D000004F78000B0037001E81FB001E80FB0053
:1091E000C200DD0040812100008040001000BE0070
:1091F000C211DD0062442100028141000089BE00ED
:109200001E4FE8001E407800F04F5000F2FF36007D
:1092100043003700227A8000337A800030D82F0054
:1092200001002000800F5100818F590012003C0086
:109230000040EB00004F78000B0037001E81FB0060
:109240001E80FB00C200DD00808521000080400000
:109250001000BE00C211DD00624421000281410005
:109260000089BE001E4FE8001E407800F04F5000FD
:10927000F2FF36002A003700227A8000337A80001D
:10928000F069280011002000800F5100818F5900E3
:1092900012003C000040EB00004F78000B0037004C
:1092A0001E81FB001E80FB00C200DD00C089210082
:1092B000008040001000BE00C211DD0062442100A9
:1092C000028141000089BE001E4FE8001E40780068
:1092D000F04F5000F2FF3600110037000040EB0065
:1092E000004F78000B0037001E81FB001E80FB0042
:1092F000C200DD00008E2100008040001000BE0092
:10930000C211DD0062442100028141000089BE00DB
:109310001E4FE8001E407800F04F5000F2FF36006C
:1093200030A2800041A2800050A4880061A488007F
:1093300050A2800061A2800070A4880081A48800EF
:1093400070A2800081A2800090A48800A1A488005F
:1093500090A28000A1A28000B0A48800C1A48800CF
:10936000B0A28000C1A28000D0A48800E1A488003F
:10937000D0A28000E1A28000F0A4880001A58800AE
:10938000F0A2800001A3800010A5880021A588001C
:1093900010A3800021A3800030A5880041A588008B
:1093A00030A3800041A3800050A5880061A58800FB
:1093B00050A3800061A3800070A5880081A588006B
:1093C00070A3800081A3800090A58800A1A58800DB
:1093D00090A38000A1A38000B0A58800C1A588004B
:1093E000B0A38000C1A38000D0A58800E1A58800BB
:1093F000D0A38000E1A38000F0A5880001A688002A
:10940000F0A3800001A4800010A6880021A6880097
:1094100010A4800021A4800030A6880041A6880006
:1094200030A4800041A4800050A6880061A6880076
:109430000080FA00000006000000FA00889FBE00CD
:109440008A9FBE00E0A920005001BE004000BE007F
:109450006022B8000600200047022400B2B00200DB
:10946000000000000004BE000205BE0060AA20004B
:109470005001BE004000BE000002BE000203BE005C
:109480000800BE000A01BE00F4A9020000000000AE
:109490000004BE000205BE00E0AA20005001BE008C
:1094A0004000BE006022B8000600200047022400F1
:1094B000BEAB02000000000008B202000000000085
:1094C0009EAD0200000000000002BE000203BE00CC
:1094D0000800BE000A01BE00F4A90200000000005E
:1094E00008B202000000000050A4880061A48800B7
:1094F00060AB20005001BE004000BE006022B800FA
:1095000006A02600870F2400B2B002000000000071
:109510000004BE000205BE00E0AB20005001BE000A
:109520004000BE006022B80006802800370C2400EE
:10953000B2B00200000000000002BE000203BE0044
:109540000800BE000A01BE00F4A9020000000000ED
:109550000004BE000205BE0060AC20005001BE0049
:109560004000BE006022B80006002400F708240076
:10957000B2B00200000000000002BE000203BE0004
:109580000800BE000A01BE00F4A9020000000000AD
:109590000004BE000205BE00E0AC20005001BE0089
:1095A0004000BE006022B80006002000970524009D
:1095B000B2B00200000000000002BE000203BE00C4
:1095C0000800BE000A01BE00F4A90200000000006D
:1095D0000004BE000205BE0060AD20005001BE00C8
:1095E0004000BE006022B8000600200047022400B0
:1095F000B2B00200000000000002BE000203BE0084
:109600000800BE000A01BE00F4A90200000000002C
:109610000004BE000205BE00E0AD20005001BE0007
:109620004000BE000002BE000203BE000800BE00F3
:109630000A01BE00F4A90200000000000004BE0000
:109640000205BE0060AE20005001BE004000BE001A
:109650006022B8000600200047022400BEAB0200D2
:109660000000000008B20200000000009EAD0200F1
:10967000000000000002BE000203BE000800BE00A1
:109680000A01BE00F4A90200000000000004BE00B0
:109690000205BE00E0AE20005001BE004000BE004A
:1096A0006022B8000600200097052400BEAB02002F
:1096B0000000000008B20200000000009EAD0200A1
:1096C000000000000002BE000203BE000800BE0051
:1096D0000A01BE00F4A902000000000008B2020066
:1096E0000000000070A4880081A4880060AF200002
:1096F0005001BE004000BE006022B80006002000FD
:1097000097052400B2B00200000000000004BE0073
:109710000205BE00E0AF20005001BE004000BE00C8
:109720006022B8000600200047022400B2B0020008
:10973000000000000002BE000203BE000800BE00E0
:109740000A01BE00F4A90200000000000004BE00EF
:109750000205BE0060B020005001BE004000BE0007
:109760000002BE000203BE000800BE000A01BE00E7
:10977000F4A90200000000000004BE000205BE00C3
:10978000E0B020005001BE004000BE006022B800E2
:109790000600200047022400BEAB020000000000CB
:1097A00008B20200000000009EAD020000000000B0
:1097B0000002BE000203BE000800BE000A01BE0097
:1097C000F4A90200000000000004BE000205BE0073
:1097D00060B120005001BE004000BE006022B80011
:1097E0000600200097052400BEAB02000000000028
:1097F00008B20200000000009EAD02000000000060
:109800000002BE000203BE000800BE000A01BE0046
:10981000F4A902000000000008B2020000000000ED
:1098200090A48800A1A48800E0B120005001BE00EF
:109830004000BE006022B800062D2100371624002B
:10984000B2B00200000000000004BE000205BE002D
:1098500060B220005001BE004000BE006022B8008F
:1098600006482800E7122400B2B002000000000001
:109870000002BE000203BE000800BE000A01BE00D6
:10988000F4A90200000000000004BE000205BE00B2
:10989000E0B220005001BE004000BE006022B800CF
:1098A00006A02600870F2400B2B0020000000000CE
:1098B0000002BE000203BE000800BE000A01BE0096
:1098C000F4A90200000000000004BE000205BE0072
:1098D00060B320005001BE004000BE006022B8000E
:1098E00006802800370C2400B2B0020000000000FF
:1098F0000002BE000203BE000800BE000A01BE0056
:10990000F4A90200000000000004BE000205BE0031
:10991000E0B320005001BE004000BE006022B8004D
:1099200006002400F7082400B2B002000000000086
:109930000002BE000203BE000800BE000A01BE0015
:10994000F4A90200000000000004BE000205BE00F1
:1099500060B420005001BE004000BE006022B8008C
:109960000600200097052400B2B0020000000000AD
:109970000002BE000203BE000800BE000A01BE00D5
:10998000F4A90200000000000004BE000205BE00B1
:10999000E0B420005001BE004000BE006022B800CC
:1099A0000600200047022400B2B0020000000000C0
:1099B0000002BE000203BE000800BE000A01BE0095
:1099C000F4A90200000000000004BE000205BE0071
:1099D00060B520005001BE004000BE000002BE0085
:1099E0000203BE000800BE000A01BE00F4A9020086
:1099F000000000000004BE000205BE00E0B520002B
:109A00005001BE004000BE006022B80006002000E9
:109A100047022400BEAB02000000000008B20200B2
:109A2000000000009EAD0200000000000002BE0029
:109A30000203BE000800BE000A01BE00F4A9020035
:109A4000000000000004BE000205BE0060B6200059
:109A50005001BE004000BE006022B8000600200099
:109A600097052400BEAB02000000000008B202000F
:109A7000000000009EAD0200000000000002BE00D9
:109A80000203BE000800BE000A01BE00F4A90200E5
:109A9000000000000004BE000205BE00E0B6200089
:109AA0005001BE004000BE006022B8000600240045
:109AB000F7082400BEAB02000000000008B202005C
:109AC000000000009EAD0200000000000002BE0089
:109AD0000203BE000800BE000A01BE00F4A9020095
:109AE000000000000004BE000205BE0060B72000B8
:109AF0005001BE004000BE006022B8000680280071
:109B0000370C2400BEAB02000000000008B20200C7
:109B1000000000009EAD0200000000000002BE0038
:109B20000203BE000800BE000A01BE00F4A9020044
:109B3000000000000004BE000205BE00E0B72000E7
:109B40005001BE004000BE006022B80006A0260002
:109B5000870F2400BEAB02000000000008B2020024
:109B6000000000009EAD0200000000000002BE00E8
:109B70000203BE000800BE000A01BE00F4A90200F4
:109B8000000000000004BE000205BE0060B8200016
:109B90005001BE004000BE006022B8000648280008
:109BA000E7122400BEAB02000000000008B2020071
:109BB000000000009EAD0200000000000002BE0098
:109BC0000203BE000800BE000A01BE00F4A90200A4
:109BD0000000000008B2020000000000B0A48800ED
:109BE000C1A48800E0B820005001BE004000BE00C3
:109BF0006022B8000600200047022400B2B0020034
:109C0000000000000004BE000205BE0060B9200094
:109C10005001BE004000BE000002BE000203BE00B4
:109C20000800BE000A01BE00F4A902000000000006
:109C300008B2020000000000D0A48800E1A488005F
:109C4000E0B920003004BE002005BE0060BA20004C
:109C50005001BE004000BE006022B8000600200097
:109C600047022400BEAB02000000000008B2020060
:109C7000000000009EAD0200000000000002BE00D7
:109C80000203BE000800BE000A01BE00F4A90200E3
:109C9000000000000004BE000205BE00E0BA200083
:109CA0005001BE004000BE006022B8000600200047
:109CB00097052400BEAB02000000000008B20200BD
:109CC000000000009EAD0200000000000002BE0087
:109CD0000203BE000800BE000A01BE00F4A9020093
:109CE0000000000008B2020000000000F0A488009C
:109CF00001A5880060BB20003004BE002005BE0026
:109D0000E0BB20005001BE004000BE006022B80051
:109D10000600200047022400BEAB02000000000045
:109D200008B20200000000009EAD0200000000002A
:109D30000002BE000203BE000800BE000A01BE0011
:109D4000F4A90200000000000004BE000205BE00ED
:109D500060BC20005001BE004000BE006022B80080
:109D60000600200097052400BEAB020000000000A2
:109D700008B20200000000009EAD020000000000DA
:109D80000002BE000203BE000800BE000A01BE00C1
:109D9000F4A90200000000000004BE000205BE009D
:109DA000E0BC20005001BE004000BE006022B800B0
:109DB00006002400F7082400BEAB020000000000EB
:109DC00008B20200000000009EAD0200000000008A
:109DD0000002BE000203BE000800BE000A01BE0071
:109DE000F4A902000000000008B202000000000018
:109DF00010A5880021A5880060BD20003004BE00A9
:109E00002005BE00E0BD20005001BE004000BE00A5
:109E10006022B8000600200047022400BEAB02000A
:109E20000000000008B20200000000009EAD020029
:109E3000000000000002BE000203BE000800BE00D9
:109E40000A01BE00F4A90200000000000004BE00E8
:109E50000205BE0060BE20005001BE004000BE00F2
:109E60006022B8000600200097052400BEAB020067
:109E70000000000008B20200000000009EAD0200D9
:109E8000000000000002BE000203BE000800BE0089
:109E90000A01BE00F4A90200000000000004BE0098
:109EA0000205BE00E0BE20005001BE004000BE0022
:109EB0006022B80006002400F7082400BEAB0200B0
:109EC0000000000008B20200000000009EAD020089
:109ED000000000000002BE000203BE000800BE0039
:109EE0000A01BE00F4A902000000000008B202004E
:109EF0000000000030A5880041A5880060BF200058
:109F00003004BE002005BE00E0BF20005001BE00AE
:109F10004000BE006022B800060020004702240076
:109F2000BEAB02000000000008B20200000000000A
:109F30009EAD0200000000000002BE000203BE0051
:109F40000800BE000A01BE00F4A9020000000000E3
:109F50000004BE000205BE0060C020005001BE002B
:109F60004000BE006022B8000600200097052400D3
:109F7000BEAB02000000000008B2020000000000BA
:109F80009EAD0200000000000002BE000203BE0001
:109F90000800BE000A01BE00F4A902000000000093
:109FA0000004BE000205BE00E0C020005001BE005B
:109FB0004000BE006022B80006002400F70824001C
:109FC000BEAB02000000000008B20200000000006A
:109FD0009EAD0200000000000002BE000203BE00B1
:109FE0000800BE000A01BE00F4A902000000000043
:109FF00008B202000000000050A5880061A588009A
:10A0000060C120003004BE002005BE00E0C1200079
:10A010005001BE004000BE006022B80006002000D3
:10A0200047022400BEAB02000000000008B202009C
:10A03000000000009EAD0200000000000002BE0013
:10A040000203BE000800BE000A01BE00F4A902001F
:10A05000000000000004BE000205BE0060C2200037
:10A060005001BE004000BE006022B8000600200083
:10A0700097052400BEAB02000000000008B20200F9
:10A08000000000009EAD0200000000000002BE00C3
:10A090000203BE000800BE000A01BE00F4A90200CF
:10A0A000000000000004BE000205BE00E0C2200067
:10A0B0005001BE004000BE006022B800060024002F
:10A0C000F7082400BEAB02000000000008B2020046
:10A0D000000000009EAD0200000000000002BE0073
:10A0E0000203BE000800BE000A01BE00F4A902007F
:10A0F0000000000008B202000000000070A5880007
:10A1000081A58800E0C320005001BE004000BE00D1
:10A110006022B80006802800370C2400B2B002008C
:10A12000000000000004BE000205BE0060C4200064
:10A130005001BE004000BE006022B80006002400AE
:10A14000F7082400B2B00200000000000002BE00C8
:10A150000203BE000800BE000A01BE00F4A902000E
:10A16000000000000004BE000205BE00E0C42000A4
:10A170005001BE004000BE006022B8000600200072
:10A1800097052400B2B00200000000000002BE00EB
:10A190000203BE000800BE000A01BE00F4A90200CE
:10A1A000000000000004BE000205BE0060C52000E3
:10A1B0005001BE004000BE006022B8000600200032
:10A1C00047022400B2B00200000000000002BE00FE
:10A1D0000203BE000800BE000A01BE00F4A902008E
:10A1E000000000000004BE000205BE00E0C5200023
:10A1F0005001BE004000BE000002BE000203BE00CF
:10A200000800BE000A01BE00F4A902000000000020
:10A210000004BE000205BE0060C620005001BE0062
:10A220004000BE006022B800060020004702240063
:10A23000BEAB02000000000008B2020000000000F7
:10A240009EAD0200000000000002BE000203BE003E
:10A250000800BE000A01BE00F4A9020000000000D0
:10A260000004BE000205BE00E0C620005001BE0092
:10A270004000BE006022B8000600200097052400C0
:10A28000BEAB02000000000008B2020000000000A7
:10A290009EAD0200000000000002BE000203BE00EE
:10A2A0000800BE000A01BE00F4A902000000000080
:10A2B00008B202000000000090A58800A1A5880057
:10A2C00060C320005001BE004000BE006022B80004
:10A2D0000600280067042400AAAB0200000000006A
:10A2E0000000E00005003A0090A58000A1A58000D4
:10A2F00001F0A20090A58800A1A58800E0C7200079
:10A300005001BE004000BE006022B8000680280058
:10A31000370C2400B2B00200000000000004BE00B0
:10A320000205BE0060C820005001BE004000BE0013
:10A330006022B80006002400F7082400B2B0020032
:10A34000000000000002BE000203BE000800BE00C4
:10A350000A01BE00F4A90200000000000004BE00D3
:10A360000205BE00E0C820005001BE004000BE0053
:10A370006022B8000600200097052400B2B0020059
:10A38000000000000002BE000203BE000800BE0084
:10A390000A01BE00F4A90200000000000004BE0093
:10A3A0000205BE0060C920005001BE004000BE0092
:10A3B0006022B8000600200047022400B2B002006C
:10A3C000000000000002BE000203BE000800BE0044
:10A3D0000A01BE00F4A90200000000000004BE0053
:10A3E0000205BE00E0C920005001BE004000BE00D2
:10A3F0000002BE000203BE000800BE000A01BE004B
:10A40000F4A90200000000000004BE000205BE0026
:10A4100060CA20005001BE004000BE006022B800AB
:10A420000600200047022400BEAB0200000000002E
:10A4300008B20200000000009EAD02000000000013
:10A440000002BE000203BE000800BE000A01BE00FA
:10A45000F4A90200000000000004BE000205BE00D6
:10A46000E0CA20005001BE004000BE006022B800DB
:10A470000600200097052400BEAB0200000000008B
:10A4800008B20200000000009EAD020000000000C3
:10A490000002BE000203BE000800BE000A01BE00AA
:10A4A000F4A902000000000008B202000000000051
:10A4B000B0A58800C1A5880060C720005001BE007B
:10A4C0004000BE006022B800060028006704240097
:10A4D000AAAB0200000000000000E00005003A0006
:10A4E000B0A58000C1A5800001F0A200B0A5880041
:10A4F000C1A5880060CB20003004BE002005BE004E
:10A50000E0CB20005001BE004000BE006022B80039
:10A510000600200047022400BEAB0200000000003D
:10A5200008B20200000000009EAD02000000000022
:10A530000002BE000203BE000800BE000A01BE0009
:10A54000F4A90200000000000004BE000205BE00E5
:10A5500060CC20005001BE004000BE006022B80068
:10A560000600200097052400BEAB0200000000009A
:10A5700008B20200000000009EAD020000000000D2
:10A580000002BE000203BE000800BE000A01BE00B9
:10A59000F4A902000000000008B202000000000060
:10A5A000D0A58800E1A58800E0CC20005001BE00C5
:10A5B0004000BE006022B8000600200047022400D0
:10A5C000B2B00200000000000004BE000205BE00A0
:10A5D00060CD20005001BE004000BE000002BE0061
:10A5E0000203BE000800BE000A01BE00F4A902007A
:10A5F000000000000004BE000205BE00E0CD200007
:10A600005001BE004000BE006022B80006002000DD
:10A6100047022400BEAB02000000000008B20200A6
:10A62000000000009EAD0200000000000002BE001D
:10A630000203BE000800BE000A01BE00F4A9020029
:10A64000000000000004BE000205BE0060CE200035
:10A650005001BE004000BE006022B800060020008D
:10A6600097052400BEAB02000000000008B2020003
:10A67000000000009EAD0200000000000002BE00CD
:10A680000203BE000800BE000A01BE00F4A90200D9
:10A690000000000008B2020000000000F0A58800E1
:10A6A00001A68800E0CE20005001BE004000BE00A0
:10A6B0006022B8000600200047022400B2B0020069
:10A6C000000000000004BE000205BE0060CF2000B4
:10A6D0005001BE004000BE000002BE000203BE00EA
:10A6E0000800BE000A01BE00F4A90200000000003C
:10A6F0000004BE000205BE00E0CF20005001BE00F5
:10A700004000BE006022B80006002000470224007E
:10A71000BEAB02000000000008B202000000000012
:10A720009EAD0200000000000002BE000203BE0059
:10A730000800BE000A01BE00F4A9020000000000EB
:10A740000004BE000205BE0060D020005001BE0023
:10A750004000BE006022B8000600200097052400DB
:10A76000BEAB02000000000008B2020000000000C2
:10A770009EAD0200000000000002BE000203BE0009
:10A780000800BE000A01BE00F4A90200000000009B
:10A7900008B202000000000010A6880021A6880070
:10A7A000E0D020005001BE004000BE006022B80092
:10A7B0000600200047022400B2B0020000000000A2
:10A7C0000004BE000205BE0060D120005001BE00A2
:10A7D0004000BE000002BE000203BE000800BE0032
:10A7E0000A01BE00F4A90200000000000004BE003F
:10A7F0000205BE00E0D120005001BE004000BE00B6
:10A800006022B8000600200047022400BEAB020010
:10A810000000000008B20200000000009EAD02002F
:10A82000000000000002BE000203BE000800BE00DF
:10A830000A01BE00F4A90200000000000004BE00EE
:10A840000205BE0060D220005001BE004000BE00E4
:10A850006022B8000600200097052400BEAB02006D
:10A860000000000008B20200000000009EAD0200DF
:10A87000000000000002BE000203BE000800BE008F
:10A880000A01BE00F4A902000000000008B20200A4
:10A890000000000030A6880041A68800E0D2200019
:10A8A0005001BE004000BE006022B800060020003B
:10A8B00047022400B2B00200000000000004BE0005
:10A8C0000205BE0060D320005001BE004000BE0063
:10A8D0000002BE000203BE000800BE000A01BE0066
:10A8E000F4A90200000000000004BE000205BE0042
:10A8F000E0D320005001BE004000BE006022B8003E
:10A900000600200047022400BEAB02000000000049
:10A9100008B20200000000009EAD0200000000002E
:10A920000002BE000203BE000800BE000A01BE0015
:10A93000F4A90200000000000004BE000205BE00F1
:10A9400060D420005001BE004000BE006022B8006C
:10A950000600200097052400BEAB020000000000A6
:10A9600008B20200000000009EAD020000000000DE
:10A970000002BE000203BE000800BE000A01BE00C5
:10A98000F4A902000000000008B20200000000006C
:10A9900050A6880061A68800D0EA20008040EB0025
:10A9A000014878004F05BE004F04BE000080FA0049
:10A9B000000006000400FA00889FBE00507B800063
:10A9C000617B800018C0B3006011B800E0AD0200E8
:10A9D000000000000000E00001003C000044EB002B
:10A9E0000804E0000C0032009621EF00507B80004C
:10A9F000617B8000307B8800417B8800307B800059
:10AA0000417B800001F0A1003EAF02000000000089
:10AA100000007800000D8800507B8000617B800082
:10AA200018C0B3006011B800DCAD020000000000E7
:10AA30000000E000010035000044EB000804E000E5
:10AA40000C003200A021EF00507B8000617B800071
:10AA5000307B8800417B8800307B8000417B800018
:10AA600001F0A1003EAF02000000000000007800ED
:10AA7000B00C8800507B8000617B80006011B800C2
:10AA8000DCAD0200000000000000E00002003A001F
:10AA90009621EF00A021EF00507B8000617B8000B9
:10AAA00002F82400337C24009CB102000000000066
:10AAB00002F02F00F377240072AC020000000000C7
:10AAC000008FBE001E00BE0001F0A100008FBE007E
:10AAD0001E00BE009EAD0200000000006022B80013
:10AAE00006802800370C2400BEAB020000000000E6
:10AAF00058AE02000000000000007800C085880009
:10AB0000C1858000007122000088B9000000780033
:10AB1000CF80DE009AAF0200000000000001BE00FE
:10AB20001E00BE00EEAA020000000000B0AE02004F
:10AB30000000000000007800CF80DE0094AF02002B
:10AB4000000000006022B80006002400F70824007E
:10AB5000BEAB02000000000058AE02000000000082
:10AB600000007800D0858800C18580000071220037
:10AB70000088B90000007800CF80DE009AAF0200A4
:10AB8000000000000001BE001E00BE00EEAA020090
:10AB9000000000000004BE00D1858000803E20003F
:10ABA0000088B90000007800CF80DE009AAF020074
:10ABB000000000000001BE000800BE00EEAA020076
:10ABC00000000000B0AE02000000000000007800AD
:10ABD000CF80DE0094AF0200000000006022B800C9
:10ABE0000600200097052400BEAB02000000000014
:10ABF00058AE02000000000000007800E0858800E8
:10AC0000C1858000007122000088B9000000780032
:10AC1000CF80DE009AAF0200000000000001BE00FD
:10AC20001E00BE00EEAA0200000000000004BE00EC
:10AC3000D1858000803E20000088B90000007800A7
:10AC4000CF80DE009AAF0200000000000001BE00CD
:10AC50000800BE00EEAA0200000000000004BE00D2
:10AC6000E1858000400620000088B90000007800DF
:10AC7000CF80DE009AAF0200000000000001BE009D
:10AC80000800BE00EEAA020000000000B0AE020004
:10AC90000000000000007800CF80DE0094AF0200CA
:10ACA000000000006022B8000600200047022400D7
:10ACB000BEAB02000000000058AE02000000000021
:10ACC00000007800F0858800C185800000712200B6
:10ACD0000088B90000007800CF80DE009AAF020043
:10ACE000000000000001BE001E00BE00EEAA02002F
:10ACF000000000000004BE00D1858000803E2000DE
:10AD00000088B90000007800CF80DE009AAF020012
:10AD1000000000000001BE000800BE00EEAA020014
:10AD2000000000000004BE00E18580004006200015
:10AD30000088B90000007800CF80DE009AAF0200E2
:10AD4000000000000001BE000800BE00EEAA0200E4
:10AD5000000000000004BE00F08580006A00B90019
:10AD600000007800CF80DE009AAF020000000000F3
:10AD70000001BE000800BE00EEAA020000000000B4
:10AD8000B0AE0200000000000000780000868800DD
:10AD90000080200010407800E14F500037003A005A
:10ADA0002A00020002000000507B8000617B8000CE
:10ADB00018C0B3006011B800E0AD02000000000050
:10ADC0000000E00001003C000044EB000804E0004B
:10ADD00003003200B6200200020000000D00370020
:10ADE000507B8000617B800018C0B3006011B80008
:10ADF000DCAD0200000000000000E00001003500B2
:10AE00000044EB000804E00002003200D021020000
:10AE100002000000C085800000407800F82B02008E
:10AE200002000000D085800000407800F82B02006E
:10AE300002000000A624020002000000E08580005D
:10AE400000407800F82B020002000000F08580002E
:10AE500000407800F82B020002000000008680000D
:10AE600000407800F82B0200020000004E1602009D
:10AE70000200000022150200020000004F04BE0084
:10AE80000080FA00000006000000FA00C012210055
:10AE90008040EB000148780015003700C012210007
:10AEA000104078000000FB00C200DD00E01221002D
:10AEB000008140006000B8000089BE00C01221007F
:10AEC000104078000000FB00C200DD00E0212100FE
:10AED000008140006000B8000089BE00C01221005F
:10AEE000104078008040E800C0122100014878003E
:10AEF000C012210090407800B0C3B30080CF500052
:10AF0000E6FF3400C01221008040EB0001487800C9
:10AF1000F03021008040EB00014878000031210032
:10AF20008040EB0001487800100020002078880065
:10AF3000103121008040EB0001487800E031210011
:10AF40008040EB0001487800003321008040EB0096
:10AF50000148780060F020008040EB000148780054
:10AF600080F020008040EB00014878000080FA006B
:10AF7000000006000C00FA00889FBE008A9FBE00F9
:10AF80008C1F780080F0200010407800E14F5000C6
:10AF90000500320080F020009040780000C2B3002D
:10AFA00080CF500038003A00B7FF0700708780005C
:10AFB000CF80DE009AAF02000000000002002000F7
:10AFC000832C240072AC02000000000090988800DE
:10AFD000A1988800000F2100104078000000FB00BD
:10AFE000CF80DE009AAF02000000000002002000C7
:10AFF000832C240072AC020000000000B09888008E
:10B00000C1988800B0988000C19880009EAD020071
:10B010000000000018C0B300A499290095992900E8
:10B020009699290097FA2300AAAB020000000000BD
:10B030000000E000010034000044EB000804E000E0
:10B0400005003200D0CC2C00C1D42300D098880059
:10B05000E198880004003700B0988000C198800013
:10B06000D0988800E198880080F0200081C0B3006B
:10B070000148780060F0200011C0B300014878005A
:10B08000BC4902000200000080F02000104078005F
:10B09000E84F50002D013A00C01221009040780086
:10B0A000B0C3B30080CF500044003C00C012210068
:10B0B000104078000004FB0020F120005001BE0089
:10B0C0004000BE0008B2020000000000C241DD00E6
:10B0D000E2122100028141000089BE00C01221005D
:10B0E000104078008040E800C0122100014878003C
:10B0F000207A8000317A80009AAF020000000000C0
:10B1000002002000A347240072AC020000000000EF
:10B11000008FBE0020F120005001BE004000BE00A4
:10B120000004BE000205BE000BF0A1001E00BE0020
:10B1300001F0A1009EAD0200000000000002BE0070
:10B140000203BE000800BE000A01BE0004B20200F5
:10B15000000000000004BE000205BE000BF0A100CC
:10B16000D0988000E19880009EAD020000000000B1
:10B170001CC0B3000002BE000203BE000800BE00F7
:10B180000A01BE00B4AB0200000000000000E000B5
:10B1900001003D000046EB000C04E000030032001B
:10B1A000C01221008040EB000148780060F02000D0
:10B1B00011C0B30001487800E4003700F0302100EE
:10B1C000104078000004FB0020F120005001BE0078
:10B1D0004000BE0008B2020000000000C241DD00D5
:10B1E000E2122100028141000089BE00F0302100FE
:10B1F000104078000004FB00A0EF20005001BE00CA
:10B200004000BE0008B2020000000000C241DD00A4
:10B21000E2212100028141000089BE00F0302100BE
:10B22000104078008040E800F030210001487800AC
:10B23000F030210090407800C0C3B30080CF5000B0
:10B2400003003A00F03021008040EB000148780014
:10B25000F0302100104078000040E9008040780084
:10B2600000312100014878000031210010407800B1
:10B270000004E00003003D0000312100B1C3B30031
:10B2800001487800F0302100104078000000FB00F9
:10B29000C200DD00E0122100008040001000BE006E
:10B2A0000002BE0005F0A10000312100104078002E
:10B2B0000000FB00C200DD00E01221000080400021
:10B2C0001000BE0001F0A1000001BE000400BE009D
:10B2D000EEAA02000000000001F0A1002007980083
:10B2E00031079800F0302100104078000000FB008A
:10B2F000C200DD00E0212100008040001000BE00FF
:10B300000002BE0005F0A1000031210010407800CD
:10B310000000FB00C200DD00E021210000804000B1
:10B320001000BE0001F0A1000001BE000400BE003C
:10B33000EEAA02000000000001F0A1004007980002
:10B340005107980060F0200010407800E14F500055
:10B3500059003A00207A8000317A80009AAF0200CA
:10B360000000000002002000A347240072AC02008D
:10B3700000000000008FBE00F03021001040780077
:10B380000000FB00C200DD00E01221000080400050
:10B390001000BE000001BE001E00BE00EEAA0200AA
:10B3A000000000000002BE0005F0A100D09880005F
:10B3B000E198800018C0B3000001BE000400BE0088
:10B3C000DCAD0200000000000000E00001003400DD
:10B3D0000044EB000804E0002F003200003121009F
:10B3E000104078000000FB00C200DD00E0122100E8
:10B3F000008040001000BE000001BE001E00BE0024
:10B40000EEAA0200000000000002BE0005F0A1004C
:10B41000D0988000E198800018C0B3000001BE0001
:10B420000400BE00DCAD0200000000000000E000EF
:10B43000010034000044EB000804E0001600320074
:10B44000B0988000C198800018C0B3000001BE0011
:10B450002E009000BE009000DCAD02000000000055
:10B460000000E000010034000044EB000804E000AC
:10B470003600320060F0200041C0B300014878007F
:10B48000A447020002000000207880006A4D0200FC
:10B49000020000002D0037007BFE070080F0200036
:10B4A00081C0B3000148780060F0200011C0B300F3
:10B4B000014878002500370060F020001040780037
:10B4C000E44F500021003A0090988000A19880003D
:10B4D00018C0B3000001BE004E009000DE009000D6
:10B4E000E0AD0200000000000000E00001003D00AF
:10B4F0000044EB000804E0000700320020788000E0
:10B500000000E80020788800207880006A4D020062
:10B51000020000000D003700B0422100104078000A
:10B520000004E000010032008DF0070060F0200010
:10B5300081C0B30001487800B0480200020000005A
:10B54000103121008040EB000148780060F02000BD
:10B5500010407800E84F5000E1023A00003121002D
:10B56000104078000000FB00C200DD00E012210066
:10B57000008040001000BE000200200003122400E2
:10B5800072AC02000000000001F0A100B0AE0200A9
:10B59000000000008040780050EB20000148780057
:10B5A00000312100104078000000FB00C200DD00E7
:10B5B000E0122100008040001000BE0001F0A10058
:10B5C0009EAD0200000000000004BE000205BE00A7
:10B5D00050EB2000104078000000FB006A00B9002A
:10B5E00000007800CF80DE0094AF02000000000071
:10B5F0000002BE000203BE000800BE000A01BE0039
:10B6000004B202000000000058AE0200000000007A
:10B610008040780060EB2000014878000031210074
:10B62000104078000000FB00C200DD00E0122100A5
:10B63000008040001000BE00020020000312240021
:10B640009CB102000000000001F0A1009EAD0200CC
:10B65000000000000004BE000205BE0050EB200008
:10B66000104078008000FB00400620000088B900F0
:10B6700000007800CF80DE0094AF020000000000E0
:10B680000002BE000203BE000800BE000A01BE00A8
:10B6900004B20200000000000004BE000205BE006B
:10B6A00060EB2000104078000000FB006A00B90049
:10B6B00000007800CF80DE0094AF020000000000A0
:10B6C0000002BE000203BE000800BE000A01BE0068
:10B6D00004B202000000000058AE020000000000AA
:10B6E0008040780070EB2000014878000031210094
:10B6F000104078000000FB00C200DD00E0122100D5
:10B70000008040001000BE0002002000832C2400B6
:10B710009CB102000000000001F0A1009EAD0200FB
:10B72000000000000004BE000205BE0050EB200037
:10B73000104078008000FB00803E20000088B900A7
:10B7400000007800CF80DE0094AF0200000000000F
:10B750000002BE000203BE000800BE000A01BE00D7
:10B7600004B20200000000000004BE000205BE009A
:10B7700060EB2000104078008000FB0040062000B5
:10B780000088B90000007800CF80DE0094AF02008E
:10B79000000000000002BE000203BE000800BE0060
:10B7A0000A01BE0004B20200000000000004BE0056
:10B7B0000205BE0070EB2000104078000000FB0086
:10B7C0006A00B90000007800CF80DE0094AF02006C
:10B7D000000000000002BE000203BE000800BE0020
:10B7E0000A01BE0004B202000000000058AE0200D0
:10B7F000000000008040780080EB200001487800C5
:10B8000000312100104078000000FB00C200DD0084
:10B81000E0122100008040001000BE000200200065
:10B82000A34724009CB102000000000001F0A10029
:10B830009EAD0200000000000004BE000205BE0034
:10B8400050EB2000104078008000FB0000712200C7
:10B850000088B90000007800CF80DE0094AF0200BD
:10B86000000000000002BE000203BE000800BE008F
:10B870000A01BE0004B20200000000000004BE0085
:10B880000205BE0060EB2000104078008000FB0045
:10B89000803E20000088B90000007800CF80DE00E4
:10B8A00094AF0200000000000002BE000203BE00D0
:10B8B0000800BE000A01BE0004B202000000000041
:10B8C0000004BE000205BE0070EB200010407800AE
:10B8D0008000FB00400620000088B90000007800CE
:10B8E000CF80DE0094AF0200000000000002BE0026
:10B8F0000203BE000800BE000A01BE0004B202003E
:10B90000000000000004BE000205BE0080EB200025
:10B91000104078000000FB006A00B90000007800C9
:10B92000CF80DE0094AF0200000000000002BE00E5
:10B930000203BE000800BE000A01BE0004B20200FD
:10B940000000000058AE02000000000080407800B7
:10B9500090EB20000148780090EB20001040780028
:10B96000E44F5000F1003400003321001040780013
:10B970000004E000ED003A000031210010407800A2
:10B980000000FB00C200DD00E0122100008040004A
:10B990001000BE0018C0B3006011B800E0AD020096
:10B9A000000000000000E00001003C000044EB004B
:10B9B0000804E00019003200003121001040780036
:10B9C0000004FB0000312100104078000000FB0063
:10B9D000C200DD00E0122100008040001000BE0027
:10B9E0009EAD020000000000B4472100E57A24006B
:10B9F00016AE270047F82300F4A90200000000005B
:10BA000008B2020000000000C241DD00E212210085
:10BA1000028141000089BE0018003700003121007A
:10BA2000104078000004FB00003121001040780035
:10BA30000000FB00C200DD00E01221000080400099
:10BA40001000BE009EAD020000000000B4472100BF
:10BA5000E57A240016AE270047F8230004B202005E
:10BA60000000000008B2020000000000C241DD003A
:10BA7000E2122100028141000089BE000031210054
:10BA8000104078000000FB00C200DD00E012210041
:10BA9000008040001000BE000200200003122400BD
:10BAA00072AC02000000000001F0A100B0AE020084
:10BAB000000000008040780050EB20000148780032
:10BAC00000312100104078000000FB00C200DD00C2
:10BAD000E0122100008040001000BE0001F0A10033
:10BAE0009EAD0200000000000004BE000205BE0082
:10BAF00050EB2000104078000000FB006A00B90005
:10BB000000007800CF80DE0094AF0200000000004B
:10BB10000002BE000203BE000800BE000A01BE0013
:10BB200004B202000000000058AE02000000000055
:10BB30008040780060EB200001487800003121004F
:10BB4000104078000000FB00C200DD00E012210080
:10BB5000008040001000BE000200200003122400FC
:10BB60009CB102000000000001F0A1009EAD0200A7
:10BB7000000000000004BE000205BE0050EB2000E3
:10BB8000104078008000FB00400620000088B900CB
:10BB900000007800CF80DE0094AF020000000000BB
:10BBA0000002BE000203BE000800BE000A01BE0083
:10BBB00004B20200000000000004BE000205BE0046
:10BBC00060EB2000104078000000FB006A00B90024
:10BBD00000007800CF80DE0094AF0200000000007B
:10BBE0000002BE000203BE000800BE000A01BE0043
:10BBF00004B202000000000058AE02000000000085
:10BC00008040780070EB200001487800003121006E
:10BC1000104078000000FB00C200DD00E0122100AF
:10BC2000008040001000BE0002002000832C240091
:10BC30009CB102000000000001F0A1009EAD0200D6
:10BC4000000000000004BE000205BE0050EB200012
:10BC5000104078008000FB00803E20000088B90082
:10BC600000007800CF80DE0094AF020000000000EA
:10BC70000002BE000203BE000800BE000A01BE00B2
:10BC800004B20200000000000004BE000205BE0075
:10BC900060EB2000104078008000FB004006200090
:10BCA0000088B90000007800CF80DE0094AF020069
:10BCB000000000000002BE000203BE000800BE003B
:10BCC0000A01BE0004B20200000000000004BE0031
:10BCD0000205BE0070EB2000104078000000FB0061
:10BCE0006A00B90000007800CF80DE0094AF020047
:10BCF000000000000002BE000203BE000800BE00FB
:10BD00000A01BE0004B202000000000058AE0200AA
:10BD1000000000008040780080EB2000014878009F
:10BD20000033210011C0B300014878000031210028
:10BD3000104078000000FB00C200DD00E02121007F
:10BD4000008040001000BE0002002000832C240070
:10BD500072AC020000000000B0AE02000000000063
:10BD600080407800E0EA200001487800003121009E
:10BD7000104078000000FB00C200DD00E02121003F
:10BD8000008040001004BE00E0EA2000104078006F
:10BD90008000FB00400620000088B9000000780009
:10BDA000CF80DE009AAF0200000000000001BE005C
:10BDB0000800BE00EEAA0200000000000200200001
:10BDC0000312240072AC020000000000B0AE0200BA
:10BDD0000000000080407800F0EA20000148780070
:10BDE00000312100104078000000FB00C200DD009F
:10BDF000E0212100008040001004BE00E0EA2000A5
:10BE0000104078008000FB00400620000088B90048
:10BE100000007800CF80DE009AAF02000000000032
:10BE20000001BE000800BE00EEAA020000000000F3
:10BE30000004BE00F0EA2000104078000000FB0083
:10BE40006A00B90000007800CF80DE009AAF0200DF
:10BE5000000000000001BE000800BE00EEAA0200C3
:10BE600000000000B0AE020000000000804078003A
:10BE700000EB2000014878000031210010407800DC
:10BE80000000FB00C200DD00E02121000080400036
:10BE90001000BE0002002000031224009CB102002A
:10BEA000000000000004BE00E0EA2000104078001E
:10BEB0008000FB00803E20000088B9000000780070
:10BEC000CF80DE009AAF0200000000000001BE003B
:10BED0000800BE00EEAA0200000000000004BE0040
:10BEE000F0EA2000104078008000FB0040062000AF
:10BEF0000088B90000007800CF80DE009AAF020011
:10BF0000000000000001BE000800BE00EEAA020012
:10BF1000000000000004BE0000EB2000104078008C
:10BF20000000FB006A00B90000007800CF80DE004E
:10BF30009AAF0200000000000001BE000800BE0031
:10BF4000EEAA020000000000B0AE020000000000F7
:10BF50008040780010EB200001487800003121007B
:10BF6000104078000000FB00C200DD00E02121004D
:10BF7000008040001000BE0002002000832C24003E
:10BF80009CB10200000000000004BE00E0EA2000B6
:10BF9000104078008000FB00007122000088B9008A
:10BFA00000007800CF80DE009AAF020000000000A1
:10BFB0000001BE000800BE00EEAA02000000000062
:10BFC0000004BE00F0EA2000104078008000FB0072
:10BFD000803E20000088B90000007800CF80DE009D
:10BFE0009AAF0200000000000001BE000800BE0081
:10BFF000EEAA0200000000000004BE0000EB2000DA
:10C00000104078008000FB00400620000088B90046
:10C0100000007800CF80DE009AAF02000000000030
:10C020000001BE000800BE00EEAA020000000000F1
:10C030000004BE0010EB2000104078000000FB0060
:10C040006A00B90000007800CF80DE009AAF0200DD
:10C05000000000000001BE000800BE00EEAA0200C1
:10C0600000000000B0AE0200000000008040780038
:10C0700020EB200001487800A02C02000200000004
:10C080001A2D020002000000207880006A4D020094
:10C0900002000000B04802000200000060F0200032
:10C0A00081C0B3000148780080F020001040780083
:10C0B000F04F500007003A0060F020008040EB0095
:10C0C000014878005A41020002000000624E02005E
:10C0D0000200000080F020008040EB000148780062
:10C0E0004F0678004F05BE004F04BE000080FA00E6
:10C0F000000006002800FA00889FBE008A9FBE004C
:10C100008C1F780080F0200010407800E14F500034
:10C110000500320080F020009040780000C2B3009B
:10C1200080CF500086003A0057FB0700303B2100CB
:10C130008040EB0001487800243321006000B80003
:10C140006011B800009ABE000292BE00A434210023
:10C150006000B8006011B800009ABE000292BE00F4
:10C16000243521006000B8006011B800009ABE00BC
:10C170000292BE00A43521006000B8006011B80032
:10C18000009ABE000292BE00243621006000B80072
:10C190006011B800009ABE000292BE00A4362100D1
:10C1A0006000B8006011B800009ABE000292BE00A4
:10C1B000243721006000B8006011B800009ABE006A
:10C1C0000292BE00A43921006000B8006011B800DE
:10C1D000009ABE000292BE00243A21006000B8001E
:10C1E0006011B800009ABE000292BE00A43A21007D
:10C1F0006000B8006011B800009ABE000292BE0054
:10C20000A43721006000B8006011B800009ABE0099
:10C210000292BE00243821006000B8006011B8000E
:10C22000009ABE000292BE00A43821006000B8004F
:10C230006011B800009ABE000292BE0024392100AD
:10C240006000B8006011B800009ABE000292BE0003
:10C25000203B21008040EB0001487800300F210096
:10C26000104078008000FB00C00320000088B90067
:10C2700000007800CF80DE0094AF020000000000D4
:10C2800084322100009ABE000292BE00400F2100BD
:10C29000104078000000FB00CF80DE009AAF020063
:10C2A0000000000002002000832C240072AC020079
:10C2B0000000000000998800119988000099800012
:10C2C000119980009EAD02000000000018C0B3006C
:10C2D000A4992900959929009699290097FA230095
:10C2E000AAAB0200000000000000E00001003400E2
:10C2F0000044EB000804E00005003200D0CC2C0024
:10C30000C1D42300209988003199880004003700A7
:10C310000099800011998000209988003199880047
:10C3200080F0200081C0B3000148780060F0200058
:10C3300011C0B30001487800BC49020002000000AF
:10C3400080F0200010407800E84F50009A023A0038
:10C35000C012210090407800B0C3B30080CF5000DD
:10C3600041003C00C0122100104078000004FB0096
:10C3700020F120005001BE004000BE0008B20200C3
:10C3800000000000C241DD00E212210002814100F4
:10C390000089BE00C0122100104078008040E800F3
:10C3A000C012210001487800207A8000317A800094
:10C3B0009AAF02000000000002002000A347240002
:10C3C00072AC020000000000008FBE0020F12000CF
:10C3D0005001BE004000BE000004BE000205BE00C9
:10C3E0000BF0A1001E00BE0001F0A1009EAD0200F6
:10C3F000000000000002BE000203BE000800BE00F4
:10C400000A01BE0004B20200000000000004BE00E9
:10C410000205BE000BF0A100209980003199800038
:10C420009EAD0200000000001CC0B3000002BE0070
:10C430000203BE000800BE000A01BE00B4AB020049
:10C44000000000000000E00001003D000046EB009D
:10C450000C04E00058023200C01221008040EB00C2
:10C460000148780054023700F03021001040780075
:10C470000004FB0020F120005001BE004000BE007F
:10C4800008B2020000000000C241DD00E2122100FB
:10C49000028141000089BE00F03021001040780088
:10C4A0008040E800F030210001487800F0302100A1
:10C4B00090407800C0C3B30080CF500003003A0022
:10C4C000F03021008040EB0001487800F03021007E
:10C4D000104078000040E9008040780000312100E1
:10C4E0000148780000312100104078000004E0008D
:10C4F00003003D0000312100B1C3B30001487800C2
:10C50000F0302100104078000000FB00C200DD0088
:10C51000E0122100008040001000BE000002BE00BA
:10C5200005F0A10000312100104078000000FB0060
:10C53000C200DD00E0122100008040001000BE00BB
:10C5400001F0A1000001BE000400BE00EEAA02003E
:10C550000000000001F0A1002007980031079800BA
:10C5600060F0200010407800E14F500056003A0083
:10C57000207A8000317A80009AAF0200000000002B
:10C5800002002000A347240072AC0200000000005B
:10C59000008FBE00F0302100104078000000FB004A
:10C5A000C200DD00E0122100008040001000BE004B
:10C5B0000001BE001E00BE00EEAA02000000000046
:10C5C0000002BE0005F0A100209980003199800092
:10C5D00018C0B3000001BE000400BE00DCAD0200C4
:10C5E000000000000000E000010034000044EB0007
:10C5F0000804E0002C0032000031210010407800D7
:10C600000000FB00C200DD00E012210000804000BD
:10C610001000BE000001BE001E00BE00EEAA020017
:10C62000000000000002BE0005F0A100209980007B
:10C630003199800018C0B3000001BE000400BE00A4
:10C64000DCAD0200000000000000E000010034004A
:10C650000044EB000804E000130032000099800061
:10C660001199800018C0B3000001BE002E00900098
:10C67000BE009000DCAD0200000000000000E00001
:10C68000010034000044EB000804E000CA0132005D
:10C6900060F0200021C0B3000148780098460200F5
:10C6A00002000000C4013700F7F9070080F0200005
:10C6B00081C0B3000148780060F0200011C0B300D1
:10C6C00001487800BC01370060F02000104078007D
:10C6D000E24F500032003A00803221003004BE00A8
:10C6E0002005BE0020788000CF80DE0094AF0200DD
:10C6F000000000000002BE000203BE000800BE00F1
:10C700000A01BE0004B202000000000058AE0200A0
:10C7100000000000000078006A4D020002000000E6
:10C72000207880000000E8002078880020788000D1
:10C73000CF80DE0094AF0200000000000004BE00C5
:10C740000205BE00803221005001BE004000BE0044
:10C750001CC0B3000002BE000203BE000800BE0001
:10C760000A01BE00B4AB0200000000000000E000BF
:10C7700001003C000046EB000C04E0008E0132009A
:10C7800060F0200041C0B30001487800A4470200D7
:10C79000020000000000EB002078880086013700CE
:10C7A00060F0200010407800E44F500082013A0011
:10C7B000207880000000E800207888002078800041
:10C7C000CF80DE0094AF0200000000000004BE0035
:10C7D0000205BE00803221005001BE004000BE00B4
:10C7E0000002BE000203BE000800BE000A01BE0037
:10C7F000F4A902000000000024332100009ABE00CA
:10C800000292BE0020788000CF80DE0094AF02004C
:10C8100000000000A4332100009ABE000292BE0076
:10C82000A03321003004BE002005BE0020332100CB
:10C830003002BE002003BE00040F9800150F9800C0
:10C84000260F9800370F9800203321005001BE00BA
:10C850004000BE000002BE000203BE000E089000B1
:10C860009E0890002E099000BE099000B2B0020010
:10C87000000000000002BE000203BE000800BE006F
:10C880000A01BE00BEAB0200000000000004BE00B2
:10C890000205BE00203621005001BE004000BE004F
:10C8A0000002BE000203BE000800BE000A01BE0076
:10C8B000F4A9020000000000A4342100009ABE0088
:10C8C0000292BE00A03321003004BE002005BE004D
:10C8D000203321005001BE004000BE000002BE0017
:10C8E0000203BE000800BE000A01BE00BEAB02008B
:10C8F000000000000004BE000205BE00A0362100BA
:10C900005001BE004000BE000002BE000203BE0097
:10C910000800BE000A01BE00F4A9020000000000E9
:10C9200024352100009ABE000292BE00203721006B
:10C930003004BE002005BE00A03321005001BE001F
:10C940004000BE000002BE000203BE000800BE00A0
:10C950000A01BE00F4A9020000000000A435210075
:10C96000009ABE000292BE00A03321003004BE0037
:10C970002005BE00A0EF20005001BE004000BE0018
:10C980000002BE000203BE000800BE000A01BE0095
:10C99000B2B00200000000000004BE000205BE00AC
:10C9A000203321005001BE004000BE000002BE0046
:10C9B0000203BE000800BE000A01BE00BEAB0200BA
:10C9C000000000000004BE000205BE00A0382100E7
:10C9D0005001BE004000BE000002BE000203BE00C7
:10C9E0000800BE000A01BE00F4A902000000000019
:10C9F000A4372100009ABE000292BE00A03321009D
:10CA00003004BE002005BE00A0EF20005001BE0093
:10CA10004000BE000002BE000203BE000800BE00CF
:10CA20000A01BE00B2B00200000000000004BE0017
:10CA30000205BE00203921005001BE004000BE00AA
:10CA40000002BE000203BE000800BE000A01BE00D4
:10CA5000F4A902000000000024382100009ABE0062
:10CA60000292BE00A03421005001BE004000BE0072
:10CA700024362100009ABE000292BE00203521001B
:10CA80005001BE004000BE00A4362100009ABE0046
:10CA90000292BE00A03521005001BE004000BE0041
:10CAA00024372100009ABE000292BE00A037210068
:10CAB0005001BE004000BE00A4382100009ABE0014
:10CAC0000292BE00203821005001BE004000BE008E
:10CAD00024392100009ABE000292BE0020352100B8
:10CAE0003004BE002005BE00203521005001BE00EC
:10CAF0004000BE000002BE000203BE000800BE00EF
:10CB00000A01BE00B2B00200000000000004BE0036
:10CB10000205BE00A03521003002BE002003BE0089
:10CB2000440F9800550F9800660F9800770F9800F3
:10CB3000A03421005001BE004000BE000002BE0033
:10CB40000203BE004E089000DE0890006E099000BF
:10CB5000FE099000B2B00200000000000002BE001A
:10CB60000203BE000800BE000A01BE0004B20200BB
:10CB700000000000400798005107980062079800E5
:10CB8000730798006022B8006033B8004E00900030
:10CB9000DE0090006E019000FE019000AAAB020042
:10CBA000000000000000E0000D003A00A0EF2000AF
:10CBB0005001BE004000BE00A4392100009ABE0012
:10CBC0000292BE00A03921005001BE004000BE000C
:10CBD000243A2100009ABE000292BE006E00370087
:10CBE000203521003004BE002005BE00A037210002
:10CBF0005001BE004000BE000002BE000203BE00A5
:10CC00000800BE000A01BE00B2B002000000000031
:10CC10000004BE000205BE00A03421003002BE00A8
:10CC20002003BE00041798001517980026179800D7
:10CC300037179800203821005001BE004000BE0088
:10CC40000002BE000203BE000E1090009E10900075
:10CC50002E119000BE119000B2B002000000000042
:10CC60000002BE000203BE000800BE000A01BE00B2
:10CC700004B20200000000004E029000DE029000AC
:10CC80006E039000FE039000BEAB020000000000A7
:10CC9000A4392100009ABE000292BE00A0392100F2
:10CCA0003004BE002005BE00203A21005001BE0025
:10CCB0004000BE000002BE000203BE000800BE002D
:10CCC0000A01BE0004B2020000000000A43A2100E4
:10CCD000009ABE000292BE0020788000E20F500051
:10CCE00027003400A03A21005001BE004000BE00E1
:10CCF00003F0A10018C0B300B4472100E57A240076
:10CD000016AE270047FA2300AAAB0200000000007D
:10CD10000000E000010034000044EB000804E000E3
:10CD200006003200203B2100104078008040E800DF
:10CD3000203B21000148780003003700203B210000
:10CD40008040EB0001487800203B21001040780033
:10CD5000E34F50000A003A00E04221001040780002
:10CD60000004E0000100320000EB0700B0480200C0
:10CD70000200000060F0200081C0B300014878008C
:10CD8000A03921005001BE004000BE00243A21001D
:10CD9000009ABE000292BE00303B21001040780095
:10CDA0008040E900303B2100014878002078800075
:10CDB0006A4D02000200000060F020001040780080
:10CDC000E84F5000EA023A0000312100104078009C
:10CDD0000000FB00C200DD00E012210000804000E6
:10CDE0001000BE00020020000312240072AC0200FA
:10CDF0000000000001F0A100B0AE02000000000041
:10CE00008040780050EB200001487800003121007C
:10CE1000104078000000FB00C200DD00E01221009D
:10CE2000008040001000BE0001F0A1009EAD020095
:10CE3000000000000004BE000205BE0050EB200010
:10CE4000104078000000FB006A00B9000000780084
:10CE5000CF80DE0094AF0200000000000002BE00A0
:10CE60000203BE000800BE000A01BE0004B20200B8
:10CE70000000000058AE0200000000008040780072
:10CE800060EB20000148780000312100104078005C
:10CE90000000FB00C200DD00E01221000080400025
:10CEA0001000BE0002002000031224009CB102000A
:10CEB0000000000001F0A1009EAD02000000000093
:10CEC0000004BE000205BE0050EB200010407800B8
:10CED0008000FB00400620000088B90000007800B8
:10CEE000CF80DE0094AF0200000000000002BE0010
:10CEF0000203BE000800BE000A01BE0004B2020028
:10CF0000000000000004BE000205BE0060EB20002F
:10CF1000104078000000FB006A00B90000007800B3
:10CF2000CF80DE0094AF0200000000000002BE00CF
:10CF30000203BE000800BE000A01BE0004B20200E7
:10CF40000000000058AE02000000000080407800A1
:10CF500070EB20000148780000312100104078007B
:10CF60000000FB00C200DD00E01221000080400054
:10CF70001000BE0002002000832C24009CB102009F
:10CF80000000000001F0A1009EAD020000000000C2
:10CF90000004BE000205BE0050EB200010407800E7
:10CFA0008000FB00803E20000088B900000078006F
:10CFB000CF80DE0094AF0200000000000002BE003F
:10CFC0000203BE000800BE000A01BE0004B2020057
:10CFD000000000000004BE000205BE0060EB20005F
:10CFE000104078008000FB00400620000088B90057
:10CFF00000007800CF80DE0094AF02000000000047
:10D000000002BE000203BE000800BE000A01BE000E
:10D0100004B20200000000000004BE000205BE00D1
:10D0200070EB2000104078000000FB006A00B9009F
:10D0300000007800CF80DE0094AF02000000000006
:10D040000002BE000203BE000800BE000A01BE00CE
:10D0500004B202000000000058AE02000000000010
:10D060008040780080EB20000148780000312100EA
:10D07000104078000000FB00C200DD00E01221003B
:10D08000008040001000BE0002002000A3472400E2
:10D090009CB102000000000001F0A1009EAD020062
:10D0A000000000000004BE000205BE0050EB20009E
:10D0B000104078008000FB00007122000088B90059
:10D0C00000007800CF80DE0094AF02000000000076
:10D0D0000002BE000203BE000800BE000A01BE003E
:10D0E00004B20200000000000004BE000205BE0001
:10D0F00060EB2000104078008000FB00803E2000A4
:10D100000088B90000007800CF80DE0094AF0200F4
:10D11000000000000002BE000203BE000800BE00C6
:10D120000A01BE0004B20200000000000004BE00BC
:10D130000205BE0070EB2000104078008000FB006C
:10D14000400620000088B90000007800CF80DE0093
:10D1500094AF0200000000000002BE000203BE0007
:10D160000800BE000A01BE0004B202000000000078
:10D170000004BE000205BE0080EB200010407800D5
:10D180000000FB006A00B90000007800CF80DE00DC
:10D1900094AF0200000000000002BE000203BE00C7
:10D1A0000800BE000A01BE0004B202000000000038
:10D1B00058AE0200000000008040780090EB200094
:10D1C0000148780090EB200010407800E44F5000B8
:10D1D000F100340000332100104078000004E0002A
:10D1E000ED003A0000312100104078000000FB0003
:10D1F000C200DD00E0122100008040001000BE00EF
:10D2000018C0B3006011B800E0AD020000000000DB
:10D210000000E00001003C000044EB000804E000D6
:10D220001900320000312100104078000004FB009A
:10D2300000312100104078000000FB00C200DD003A
:10D24000E0122100008040001000BE009EAD0200F0
:10D2500000000000B4472100E57A240016AE270044
:10D2600047F82300F4A902000000000008B2020001
:10D2700000000000C241DD00E212210002814100F5
:10D280000089BE00180037000031210010407800EE
:10D290000004FB0000312100104078000000FB007A
:10D2A000C200DD00E0122100008040001000BE003E
:10D2B0009EAD020000000000B4472100E57A240082
:10D2C00016AE270047F8230004B202000000000059
:10D2D00008B2020000000000C241DD00E21221009D
:10D2E000028141000089BE00003121001040780019
:10D2F0000000FB00C200DD00E012210000804000C1
:10D300001000BE00020020000312240072AC0200D4
:10D310000000000001F0A100B0AE0200000000001B
:10D320008040780050EB2000014878000031210057
:10D33000104078000000FB00C200DD00E012210078
:10D34000008040001000BE0001F0A1009EAD020070
:10D35000000000000004BE000205BE0050EB2000EB
:10D36000104078000000FB006A00B900000078005F
:10D37000CF80DE0094AF0200000000000002BE007B
:10D380000203BE000800BE000A01BE0004B2020093
:10D390000000000058AE020000000000804078004D
:10D3A00060EB200001487800003121001040780037
:10D3B0000000FB00C200DD00E01221000080400000
:10D3C0001000BE0002002000031224009CB10200E5
:10D3D0000000000001F0A1009EAD0200000000006E
:10D3E0000004BE000205BE0050EB20001040780093
:10D3F0008000FB00400620000088B9000000780093
:10D40000CF80DE0094AF0200000000000002BE00EA
:10D410000203BE000800BE000A01BE0004B2020002
:10D42000000000000004BE000205BE0060EB20000A
:10D43000104078000000FB006A00B900000078008E
:10D44000CF80DE0094AF0200000000000002BE00AA
:10D450000203BE000800BE000A01BE0004B20200C2
:10D460000000000058AE020000000000804078007C
:10D4700070EB200001487800003121001040780056
:10D480000000FB00C200DD00E0122100008040002F
:10D490001000BE0002002000832C24009CB102007A
:10D4A0000000000001F0A1009EAD0200000000009D
:10D4B0000004BE000205BE0050EB200010407800C2
:10D4C0008000FB00803E20000088B900000078004A
:10D4D000CF80DE0094AF0200000000000002BE001A
:10D4E0000203BE000800BE000A01BE0004B2020032
:10D4F000000000000004BE000205BE0060EB20003A
:10D50000104078008000FB00400620000088B90031
:10D5100000007800CF80DE0094AF02000000000021
:10D520000002BE000203BE000800BE000A01BE00E9
:10D5300004B20200000000000004BE000205BE00AC
:10D5400070EB2000104078000000FB006A00B9007A
:10D5500000007800CF80DE0094AF020000000000E1
:10D560000002BE000203BE000800BE000A01BE00A9
:10D5700004B202000000000058AE020000000000EB
:10D580008040780080EB20000148780000332100C3
:10D5900011C0B30001487800A03921005001BE003D
:10D5A0004000BE006022B80006002000970524005D
:10D5B000BEAB02000000000058AE020000000000F8
:10D5C00080407800E0EA200001487800A03921007E
:10D5D0003004BE002005BE00E0EA200010407800C4
:10D5E0008000FB00400620000088B90000007800A1
:10D5F000CF80DE0094AF0200000000000002BE00F9
:10D600000203BE000800BE000A01BE0004B2020010
:10D61000000000006022B80006002000470224003D
:10D62000BEAB02000000000058AE02000000000087
:10D6300080407800F0EA200001487800A0392100FD
:10D640003004BE002005BE00E0EA20001040780053
:10D650008000FB00400620000088B9000000780030
:10D66000CF80DE0094AF0200000000000002BE0088
:10D670000203BE000800BE000A01BE0004B20200A0
:10D68000000000000004BE000205BE00F0EA200019
:10D69000104078000000FB006A00B900000078002C
:10D6A000CF80DE0094AF0200000000000002BE0048
:10D6B0000203BE000800BE000A01BE0004B2020060
:10D6C0000000000058AE020000000000804078001A
:10D6D00000EB200001487800A03921005001BE0075
:10D6E0004000BE006022B80006002000470224006F
:10D6F000B2B00200000000000004BE000205BE003F
:10D70000E0EA2000104078008000FB00803E20000E
:10D710000088B90000007800CF80DE0094AF0200DE
:10D72000000000000002BE000203BE000800BE00B0
:10D730000A01BE0004B20200000000000004BE00A6
:10D740000205BE00F0EA2000104078008000FB00D7
:10D75000400620000088B90000007800CF80DE007D
:10D7600094AF0200000000000002BE000203BE00F1
:10D770000800BE000A01BE0004B202000000000062
:10D780000004BE000205BE0000EB2000104078003F
:10D790000000FB006A00B90000007800CF80DE00C6
:10D7A00094AF0200000000000002BE000203BE00B1
:10D7B0000800BE000A01BE0004B202000000000022
:10D7C00058AE0200000000008040780010EB2000FE
:10D7D00001487800A03921005001BE004000BE0081
:10D7E0006022B8000600200097052400B2B00200B5
:10D7F000000000000004BE000205BE00E0EA2000B8
:10D80000104078008000FB00007122000088B90001
:10D8100000007800CF80DE0094AF0200000000001E
:10D820000002BE000203BE000800BE000A01BE00E6
:10D8300004B20200000000000004BE000205BE00A9
:10D84000F0EA2000104078008000FB00803E2000BD
:10D850000088B90000007800CF80DE0094AF02009D
:10D86000000000000002BE000203BE000800BE006F
:10D870000A01BE0004B20200000000000004BE0065
:10D880000205BE0000EB2000104078008000FB0085
:10D89000400620000088B90000007800CF80DE003C
:10D8A00094AF0200000000000002BE000203BE00B0
:10D8B0000800BE000A01BE0004B202000000000021
:10D8C0000004BE000205BE0010EB200010407800EE
:10D8D0000000FB006A00B90000007800CF80DE0085
:10D8E00094AF0200000000000002BE000203BE0070
:10D8F0000800BE000A01BE0004B2020000000000E1
:10D9000058AE0200000000008040780020EB2000AC
:10D91000014878001A2D020002000000F04C0200BD
:10D9200002000000207880006A4D02000200000022
:10D93000B04802000200000080F020001040780093
:10D94000F04F500007003A0060F020008040EB00EC
:10D95000014878005A41020002000000624E0200B5
:10D960000200000080F020008040EB0001487800B9
:10D97000D0EA200010407800E74F500001003A0044
:10D98000050007004F0678004F05BE004F04BE009B
:10D990000080FA00000006000000FA00889FBE0028
:10D9A0008A9FBE0021788000400620000001780098
:10D9B000110009008200D800F0A78800F1A78000BC
:10D9C000C0F92F000088B90080007800207880001E
:10D9D00080804000A00020000001780011000900B4
:10D9E0008200D80000A88800F1A78000C0F92F00AD
:10D9F0000088B9000001780001A8800060FF2F00B6
:10DA00000088B90000007800800041002078800084
:10DA10000080400010A88800A03421005001BE0002
:10DA20004000BE006022B80006002000470224002B
:10DA3000BEAB020000000000E4AD020000000000E8
:10DA400044502100009ABE000292BE00A034210082
:10DA50003004BE002005BE00405021005001BE0031
:10DA60004000BE00A4002000050020006033B80084
:10DA70007EB202000000000074AF0200000000004F
:10DA80000002BE000203BE000800BE000A01BE0084
:10DA900004B2020000000000E4AD0200000000003B
:10DAA000C4502100009ABE000292BE00A0342100A2
:10DAB0005001BE004000BE006022B80006002000F9
:10DAC00047022400B2B00200000000000004BE00C3
:10DAD0000205BE00405021005001BE004000BE00C3
:10DAE00044062000050020006033B8007EB202002A
:10DAF0000000000074AF0200000000000002BE0041
:10DB00000203BE000800BE000A01BE0004B202000B
:10DB1000000000000004BE000205BE00C05021004D
:10DB20005001BE004000BE00A400200005002000FF
:10DB30006033B8007EB202000000000074AF020043
:10DB4000000000000002BE000203BE000800BE008C
:10DB50000A01BE0004B2020000000000E4AD0200B1
:10DB60000000000044512100009ABE000292BE0055
:10DB7000A03421005001BE004000BE006022B80069
:10DB80000600200097052400B2B00200000000004B
:10DB90000004BE000205BE00405021005001BE003E
:10DBA0004000BE00843E2000050020006033B80025
:10DBB0007EB202000000000074AF0200000000000E
:10DBC0000002BE000203BE000800BE000A01BE0043
:10DBD00004B20200000000000004BE000205BE0006
:10DBE000C05021005001BE004000BE00440620008D
:10DBF000050020006033B8007EB202000000000083
:10DC000074AF0200000000000002BE000203BE006C
:10DC10000800BE000A01BE0004B2020000000000BD
:10DC20000004BE000205BE00405121005001BE00AC
:10DC30004000BE00A4002000050020006033B800B2
:10DC40007EB202000000000074AF0200000000007D
:10DC50000002BE000203BE000800BE000A01BE00B2
:10DC600004B2020000000000E4AD02000000000069
:10DC7000C4512100009ABE000292BE00A0342100CF
:10DC80005001BE004000BE006022B8000600240023
:10DC9000F7082400B2B00200000000000004BE003B
:10DCA0000205BE00405021005001BE004000BE00F1
:10DCB00004712200050020006033B8007EB202002B
:10DCC0000000000074AF0200000000000002BE006F
:10DCD0000203BE000800BE000A01BE0004B202003A
:10DCE000000000000004BE000205BE00C05021007C
:10DCF0005001BE004000BE00843E20000500200010
:10DD00006033B8007EB202000000000074AF020071
:10DD1000000000000002BE000203BE000800BE00BA
:10DD20000A01BE0004B20200000000000004BE00B0
:10DD30000205BE00405121005001BE004000BE005F
:10DD400044062000050020006033B8007EB20200C7
:10DD50000000000074AF0200000000000002BE00DE
:10DD60000203BE000800BE000A01BE0004B20200A9
:10DD7000000000000004BE000205BE00C0512100EA
:10DD80005001BE004000BE00A4002000050020009D
:10DD90006033B8007EB202000000000074AF0200E1
:10DDA000000000000002BE000203BE000800BE002A
:10DDB0000A01BE0004B2020000000000E4AD02004F
:10DDC0000000000044522100009ABE000292BE00F2
:10DDD000A03421005001BE004000BE006022B80007
:10DDE00006802800370C2400B2B0020000000000BA
:10DDF0000004BE000205BE00405021005001BE00DC
:10DE00004000BE00046A2800150020006033B800FE
:10DE10007EB202000000000074AF020000000000AB
:10DE20000002BE000203BE000800BE000A01BE00E0
:10DE300004B20200000000000004BE000205BE00A3
:10DE4000C05021005001BE004000BE0004712200FD
:10DE5000050020006033B8007EB202000000000020
:10DE600074AF0200000000000002BE000203BE000A
:10DE70000800BE000A01BE0004B20200000000005B
:10DE80000004BE000205BE00405121005001BE004A
:10DE90004000BE00843E2000050020006033B80032
:10DEA0007EB202000000000074AF0200000000001B
:10DEB0000002BE000203BE000800BE000A01BE0050
:10DEC00004B20200000000000004BE000205BE0013
:10DED000C05121005001BE004000BE004406200099
:10DEE000050020006033B8007EB202000000000090
:10DEF00074AF0200000000000002BE000203BE007A
:10DF00000800BE000A01BE0004B2020000000000CA
:10DF10000004BE000205BE00405221005001BE00B8
:10DF20004000BE00A4002000050020006033B800BF
:10DF30007EB202000000000074AF0200000000008A
:10DF40000002BE000203BE000800BE000A01BE00BF
:10DF500004B2020000000000E4AD02000000000076
:10DF6000C4522100009ABE000292BE00A0342100DB
:10DF70005001BE004000BE006022B80006A026008E
:10DF8000870F2400B2B00200000000000004BE00B1
:10DF90000205BE00405021005001BE004000BE00FE
:10DFA00004242400F50020006033B8007EB2020093
:10DFB0000000000074AF0200000000000002BE007C
:10DFC0000203BE000800BE000A01BE0004B2020047
:10DFD000000000000004BE000205BE00C050210089
:10DFE0005001BE004000BE00046A28001500200059
:10DFF0006033B8007EB202000000000074AF02007F
:10E00000000000000002BE000203BE000800BE00C7
:10E010000A01BE0004B20200000000000004BE00BD
:10E020000205BE00405121005001BE004000BE006C
:10E0300004712200050020006033B8007EB20200A7
:10E040000000000074AF0200000000000002BE00EB
:10E050000203BE000800BE000A01BE0004B20200B6
:10E06000000000000004BE000205BE00C0512100F7
:10E070005001BE004000BE00843E2000050020008C
:10E080006033B8007EB202000000000074AF0200EE
:10E09000000000000002BE000203BE000800BE0037
:10E0A0000A01BE0004B20200000000000004BE002D
:10E0B0000205BE00405221005001BE004000BE00DB
:10E0C00044062000050020006033B8007EB2020044
:10E0D0000000000074AF0200000000000002BE005B
:10E0E0000203BE000800BE000A01BE0004B2020026
:10E0F000000000000004BE000205BE00C052210066
:10E100005001BE004000BE00A40020000500200019
:10E110006033B8007EB202000000000074AF02005D
:10E12000000000000002BE000203BE000800BE00A6
:10E130000A01BE0004B2020000000000E4AD0200CB
:10E140000000000044532100009ABE000292BE006D
:10E15000A03421005001BE004000BE006022B80083
:10E1600006482800E7122400B2B0020000000000B8
:10E170000004BE000205BE00405021005001BE0058
:10E180004000BE0004682900850920006033B80003
:10E190007EB202000000000074AF02000000000028
:10E1A0000002BE000203BE000800BE000A01BE005D
:10E1B00004B20200000000000004BE000205BE0020
:10E1C000C05021005001BE004000BE0004242400C5
:10E1D000F50020006033B8007EB2020000000000AD
:10E1E00074AF0200000000000002BE000203BE0087
:10E1F0000800BE000A01BE0004B2020000000000D8
:10E200000004BE000205BE00405121005001BE00C6
:10E210004000BE00046A2800150020006033B800EA
:10E220007EB202000000000074AF02000000000097
:10E230000002BE000203BE000800BE000A01BE00CC
:10E2400004B20200000000000004BE000205BE008F
:10E25000C05121005001BE004000BE0004712200E8
:10E26000050020006033B8007EB20200000000000C
:10E2700074AF0200000000000002BE000203BE00F6
:10E280000800BE000A01BE0004B202000000000047
:10E290000004BE000205BE00405221005001BE0035
:10E2A0004000BE00843E2000050020006033B8001E
:10E2B0007EB202000000000074AF02000000000007
:10E2C0000002BE000203BE000800BE000A01BE003C
:10E2D00004B20200000000000004BE000205BE00FF
:10E2E000C05221005001BE004000BE004406200084
:10E2F000050020006033B8007EB20200000000007C
:10E3000074AF0200000000000002BE000203BE0065
:10E310000800BE000A01BE0004B2020000000000B6
:10E320000004BE000205BE00405321005001BE00A3
:10E330004000BE00A4002000050020006033B800AB
:10E340007EB202000000000074AF02000000000076
:10E350000002BE000203BE000800BE000A01BE00AB
:10E3600004B2020000000000E4AD02000000000062
:10E37000C4532100009ABE000292BE00A0342100C6
:10E380005001BE004000BE006022B800062D2100F2
:10E3900037162400B2B00200000000000004BE00E6
:10E3A0000205BE00405021005001BE004000BE00EA
:10E3B00004102E00555F20006033B8007EB20200CA
:10E3C0000000000074AF0200000000000002BE0068
:10E3D0000203BE000800BE000A01BE0004B2020033
:10E3E000000000000004BE000205BE00C050210075
:10E3F0005001BE004000BE000468290085092000CD
:10E400006033B8007EB202000000000074AF02006A
:10E41000000000000002BE000203BE000800BE00B3
:10E420000A01BE0004B20200000000000004BE00A9
:10E430000205BE00405121005001BE004000BE0058
:10E4400004242400F50020006033B8007EB20200EE
:10E450000000000074AF0200000000000002BE00D7
:10E460000203BE000800BE000A01BE0004B20200A2
:10E47000000000000004BE000205BE00C0512100E3
:10E480005001BE004000BE00046A280015002000B4
:10E490006033B8007EB202000000000074AF0200DA
:10E4A000000000000002BE000203BE000800BE0023
:10E4B0000A01BE0004B20200000000000004BE0019
:10E4C0000205BE00405221005001BE004000BE00C7
:10E4D00004712200050020006033B8007EB2020003
:10E4E0000000000074AF0200000000000002BE0047
:10E4F0000203BE000800BE000A01BE0004B2020012
:10E50000000000000004BE000205BE00C052210051
:10E510005001BE004000BE00843E200005002000E7
:10E520006033B8007EB202000000000074AF020049
:10E53000000000000002BE000203BE000800BE0092
:10E540000A01BE0004B20200000000000004BE0088
:10E550000205BE00405321005001BE004000BE0035
:10E5600044062000050020006033B8007EB202009F
:10E570000000000074AF0200000000000002BE00B6
:10E580000203BE000800BE000A01BE0004B2020081
:10E59000000000000004BE000205BE00C0532100C0
:10E5A0005001BE004000BE00A40020000500200075
:10E5B0006033B8007EB202000000000074AF0200B9
:10E5C000000000000002BE000203BE000800BE0002
:10E5D0000A01BE0004B2020000000000E4AD020027
:10E5E0000000000044542100009ABE000292BE00C8
:10E5F000203521005001BE004000BE006022B8005E
:10E6000006002400F7082400BEAB02000000000052
:10E61000E4AD020000000000C4542100009ABE00D6
:10E620000292BE00203521003004BE002005BE004D
:10E63000C05421005001BE004000BE00843E2000B6
:10E64000050020006033B8007EB202000000000028
:10E6500074AF0200000000000002BE000203BE0012
:10E660000800BE000A01BE0004B202000000000063
:10E670006022B8000600200097052400BEAB02000F
:10E6800000000000E4AD020000000000445521003D
:10E69000009ABE000292BE00203521003004BE0068
:10E6A0002005BE00C05421005001BE004000BE0045
:10E6B000843E2000050020006033B8007EB20200D6
:10E6C0000000000074AF0200000000000002BE0065
:10E6D0000203BE000800BE000A01BE0004B2020030
:10E6E000000000000004BE000205BE0040552100ED
:10E6F0005001BE004000BE0044062000050020007E
:10E700006033B8007EB202000000000074AF020067
:10E71000000000000002BE000203BE000800BE00B0
:10E720000A01BE0004B20200000000006022B8002E
:10E730000600200047022400BEAB020000000000DB
:10E74000E4AD020000000000C4552100009ABE00A4
:10E750000292BE00203521003004BE002005BE001C
:10E76000C05421005001BE004000BE00843E200085
:10E77000050020006033B8007EB2020000000000F7
:10E7800074AF0200000000000002BE000203BE00E1
:10E790000800BE000A01BE0004B202000000000032
:10E7A0000004BE000205BE00405521005001BE001D
:10E7B0004000BE0044062000050020006033B80081
:10E7C0007EB202000000000074AF020000000000F2
:10E7D0000002BE000203BE000800BE000A01BE0027
:10E7E00004B20200000000000004BE000205BE00EA
:10E7F000C05521005001BE004000BE00A400200012
:10E80000050020006033B8007EB202000000000066
:10E8100074AF0200000000000002BE000203BE0050
:10E820000800BE000A01BE0004B2020000000000A1
:10E83000E4AD02000000000044562100009ABE0032
:10E840000292BE00203521005001BE004000BE00F3
:10E850006022B8000600200047022400B2B0020087
:10E86000000000000004BE000205BE00C0542100EC
:10E870005001BE004000BE000471220005002000CF
:10E880006033B8007EB202000000000074AF0200E6
:10E89000000000000002BE000203BE000800BE002F
:10E8A0000A01BE0004B20200000000000004BE0025
:10E8B0000205BE00405521005001BE004000BE00D0
:10E8C000843E2000050020006033B8007EB20200C4
:10E8D0000000000074AF0200000000000002BE0053
:10E8E0000203BE000800BE000A01BE0004B202001E
:10E8F000000000000004BE000205BE00C05521005B
:10E900005001BE004000BE0044062000050020006B
:10E910006033B8007EB202000000000074AF020055
:10E92000000000000002BE000203BE000800BE009E
:10E930000A01BE0004B20200000000000004BE0094
:10E940000205BE00405621005001BE004000BE003E
:10E95000A4002000050020006033B8007EB2020051
:10E960000000000074AF0200000000000002BE00C2
:10E970000203BE000800BE000A01BE0004B202008D
:10E9800000000000E4AD020000000000C4562100B9
:10E99000009ABE000292BE00203521005001BE0048
:10E9A0004000BE006022B800060020009705240049
:10E9B000B2B00200000000000004BE000205BE006C
:10E9C000C05421005001BE004000BE00046A28006F
:10E9D000150020006033B8007EB202000000000085
:10E9E00074AF0200000000000002BE000203BE007F
:10E9F0000800BE000A01BE0004B2020000000000D0
:10EA00000004BE000205BE00405521005001BE00BA
:10EA10004000BE0004712200050020006033B800F1
:10EA20007EB202000000000074AF0200000000008F
:10EA30000002BE000203BE000800BE000A01BE00C4
:10EA400004B20200000000000004BE000205BE0087
:10EA5000C05521005001BE004000BE00843E200091
:10EA6000050020006033B8007EB202000000000004
:10EA700074AF0200000000000002BE000203BE00EE
:10EA80000800BE000A01BE0004B20200000000003F
:10EA90000004BE000205BE00405621005001BE0029
:10EAA0004000BE0044062000050020006033B8008E
:10EAB0007EB202000000000074AF020000000000FF
:10EAC0000002BE000203BE000800BE000A01BE0034
:10EAD00004B20200000000000004BE000205BE00F7
:10EAE000C05621005001BE004000BE00A40020001E
:10EAF000050020006033B8007EB202000000000074
:10EB000074AF0200000000000002BE000203BE005D
:10EB10000800BE000A01BE0004B2020000000000AE
:10EB2000E4AD02000000000044572100009ABE003E
:10EB30000292BE00203521005001BE004000BE0000
:10EB40006022B80006002400F7082400B2B00200DA
:10EB5000000000000004BE000205BE00C0542100F9
:10EB60005001BE004000BE0004242400F500200037
:10EB70006033B8007EB202000000000074AF0200F3
:10EB8000000000000002BE000203BE000800BE003C
:10EB90000A01BE0004B20200000000000004BE0032
:10EBA0000205BE00405521005001BE004000BE00DD
:10EBB000046A2800150020006033B8007EB202000D
:10EBC0000000000074AF0200000000000002BE0060
:10EBD0000203BE000800BE000A01BE0004B202002B
:10EBE000000000000004BE000205BE00C055210068
:10EBF0005001BE004000BE0004712200050020004C
:10EC00006033B8007EB202000000000074AF020062
:10EC1000000000000002BE000203BE000800BE00AB
:10EC20000A01BE0004B20200000000000004BE00A1
:10EC30000205BE00405621005001BE004000BE004B
:10EC4000843E2000050020006033B8007EB2020040
:10EC50000000000074AF0200000000000002BE00CF
:10EC60000203BE000800BE000A01BE0004B202009A
:10EC7000000000000004BE000205BE00C0562100D6
:10EC80005001BE004000BE004406200005002000E8
:10EC90006033B8007EB202000000000074AF0200D2
:10ECA000000000000002BE000203BE000800BE001B
:10ECB0000A01BE0004B20200000000000004BE0011
:10ECC0000205BE00405721005001BE004000BE00BA
:10ECD000A4002000050020006033B8007EB20200CE
:10ECE0000000000074AF0200000000000002BE003F
:10ECF0000203BE000800BE000A01BE0004B202000A
:10ED000000000000E4AD020000000000C457210034
:10ED1000009ABE000292BE00203521005001BE00C4
:10ED20004000BE006022B80006802800370C240096
:10ED3000B2B00200000000000004BE000205BE00E8
:10ED4000C05421005001BE004000BE0004682900EC
:10ED5000850920006033B8007EB202000000000088
:10ED600074AF0200000000000002BE000203BE00FB
:10ED70000800BE000A01BE0004B20200000000004C
:10ED80000004BE000205BE00405521005001BE0037
:10ED90004000BE0004242400F50020006033B800C9
:10EDA0007EB202000000000074AF0200000000000C
:10EDB0000002BE000203BE000800BE000A01BE0041
:10EDC00004B20200000000000004BE000205BE0004
:10EDD000C05521005001BE004000BE00046A28005A
:10EDE000150020006033B8007EB202000000000071
:10EDF00074AF0200000000000002BE000203BE006B
:10EE00000800BE000A01BE0004B2020000000000BB
:10EE10000004BE000205BE00405621005001BE00A5
:10EE20004000BE0004712200050020006033B800DD
:10EE30007EB202000000000074AF0200000000007B
:10EE40000002BE000203BE000800BE000A01BE00B0
:10EE500004B20200000000000004BE000205BE0073
:10EE6000C05621005001BE004000BE00843E20007C
:10EE7000050020006033B8007EB2020000000000F0
:10EE800074AF0200000000000002BE000203BE00DA
:10EE90000800BE000A01BE0004B20200000000002B
:10EEA0000004BE000205BE00405721005001BE0014
:10EEB0004000BE0044062000050020006033B8007A
:10EEC0007EB202000000000074AF020000000000EB
:10EED0000002BE000203BE000800BE000A01BE0020
:10EEE00004B20200000000000004BE000205BE00E3
:10EEF000C05721005001BE004000BE00A400200009
:10EF0000050020006033B8007EB20200000000005F
:10EF100074AF0200000000000002BE000203BE0049
:10EF20000800BE000A01BE0004B20200000000009A
:10EF3000E4AD02000000000044582100009ABE0029
:10EF40000292BE00203521005001BE004000BE00EC
:10EF50006022B80006A02600870F2400B2B002008D
:10EF6000000000000004BE000205BE00C0542100E5
:10EF70005001BE004000BE0004102E00555F20006E
:10EF80006033B8007EB202000000000074AF0200DF
:10EF9000000000000002BE000203BE000800BE0028
:10EFA0000A01BE0004B20200000000000004BE001E
:10EFB0000205BE00405521005001BE004000BE00C9
:10EFC00004682900850920006033B8007EB2020081
:10EFD0000000000074AF0200000000000002BE004C
:10EFE0000203BE000800BE000A01BE0004B2020017
:10EFF000000000000004BE000205BE00C055210054
:10F000005001BE004000BE0004242400F500200092
:10F010006033B8007EB202000000000074AF02004E
:10F02000000000000002BE000203BE000800BE0097
:10F030000A01BE0004B20200000000000004BE008D
:10F040000205BE00405621005001BE004000BE0037
:10F05000046A2800150020006033B8007EB2020068
:10F060000000000074AF0200000000000002BE00BB
:10F070000203BE000800BE000A01BE0004B2020086
:10F08000000000000004BE000205BE00C0562100C2
:10F090005001BE004000BE000471220005002000A7
:10F0A0006033B8007EB202000000000074AF0200BE
:10F0B000000000000002BE000203BE000800BE0007
:10F0C0000A01BE0004B20200000000000004BE00FD
:10F0D0000205BE00405721005001BE004000BE00A6
:10F0E000843E2000050020006033B8007EB202009C
:10F0F0000000000074AF0200000000000002BE002B
:10F100000203BE000800BE000A01BE0004B20200F5
:10F11000000000000004BE000205BE00C057210030
:10F120005001BE004000BE00440620000500200043
:10F130006033B8007EB202000000000074AF02002D
:10F14000000000000002BE000203BE000800BE0076
:10F150000A01BE0004B20200000000000004BE006C
:10F160000205BE00405821005001BE004000BE0014
:10F17000A4002000050020006033B8007EB2020029
:10F180000000000074AF0200000000000002BE009A
:10F190000203BE000800BE000A01BE0004B2020065
:10F1A00000000000E4AD020000000000C45821008F
:10F1B000009ABE000292BE00203521005001BE0020
:10F1C0004000BE006022B80006482800E712240074
:10F1D000B2B00200000000000004BE000205BE0044
:10F1E000C05421005001BE004000BE0004A02C000D
:10F1F000A5B923006033B8007EB202000000000011
:10F2000074AF0200000000000002BE000203BE0056
:10F210000800BE000A01BE0004B2020000000000A7
:10F220000004BE000205BE00405521005001BE0092
:10F230004000BE0004102E00555F20006033B8006F
:10F240007EB202000000000074AF02000000000067
:10F250000002BE000203BE000800BE000A01BE009C
:10F2600004B20200000000000004BE000205BE005F
:10F27000C05521005001BE004000BE0004682900B6
:10F28000850920006033B8007EB202000000000053
:10F2900074AF0200000000000002BE000203BE00C6
:10F2A0000800BE000A01BE0004B202000000000017
:10F2B0000004BE000205BE00405621005001BE0001
:10F2C0004000BE0004242400F50020006033B80094
:10F2D0007EB202000000000074AF020000000000D7
:10F2E0000002BE000203BE000800BE000A01BE000C
:10F2F00004B20200000000000004BE000205BE00CF
:10F30000C05621005001BE004000BE00046A280023
:10F31000150020006033B8007EB20200000000003B
:10F3200074AF0200000000000002BE000203BE0035
:10F330000800BE000A01BE0004B202000000000086
:10F340000004BE000205BE00405721005001BE006F
:10F350004000BE0004712200050020006033B800A8
:10F360007EB202000000000074AF02000000000046
:10F370000002BE000203BE000800BE000A01BE007B
:10F3800004B20200000000000004BE000205BE003E
:10F39000C05721005001BE004000BE00843E200046
:10F3A000050020006033B8007EB2020000000000BB
:10F3B00074AF0200000000000002BE000203BE00A5
:10F3C0000800BE000A01BE0004B2020000000000F6
:10F3D0000004BE000205BE00405821005001BE00DE
:10F3E0004000BE0044062000050020006033B80045
:10F3F0007EB202000000000074AF020000000000B6
:10F400000002BE000203BE000800BE000A01BE00EA
:10F4100004B20200000000000004BE000205BE00AD
:10F42000C05821005001BE004000BE00A4002000D2
:10F43000050020006033B8007EB20200000000002A
:10F4400074AF0200000000000002BE000203BE0014
:10F450000800BE000A01BE0004B202000000000065
:10F46000E4AD02000000000044592100009ABE00F3
:10F470000292BE00203521005001BE004000BE00B7
:10F480006022B800062D210037162400B2B0020019
:10F49000000000000004BE000205BE00C0542100B0
:10F4A0005001BE004000BE0004402E00B5402500C3
:10F4B00026002000070020007EB2020000000000AD
:10F4C00074AF0200000000000002BE000203BE0094
:10F4D0000800BE000A01BE0004B2020000000000E5
:10F4E0000004BE000205BE00405521005001BE00D0
:10F4F0004000BE0004A02C00A5B923006033B80072
:10F500007EB202000000000074AF020000000000A4
:10F510000002BE000203BE000800BE000A01BE00D9
:10F5200004B20200000000000004BE000205BE009C
:10F53000C05521005001BE004000BE0004102E0046
:10F54000555F20006033B8007EB20200000000006A
:10F5500074AF0200000000000002BE000203BE0003
:10F560000800BE000A01BE0004B202000000000054
:10F570000004BE000205BE00405621005001BE003E
:10F580004000BE0004682900850920006033B800EF
:10F590007EB202000000000074AF02000000000014
:10F5A0000002BE000203BE000800BE000A01BE0049
:10F5B00004B20200000000000004BE000205BE000C
:10F5C000C05621005001BE004000BE0004242400AB
:10F5D000F50020006033B8007EB202000000000099
:10F5E00074AF0200000000000002BE000203BE0073
:10F5F0000800BE000A01BE0004B2020000000000C4
:10F600000004BE000205BE00405721005001BE00AC
:10F610004000BE00046A2800150020006033B800D6
:10F620007EB202000000000074AF02000000000083
:10F630000002BE000203BE000800BE000A01BE00B8
:10F6400004B20200000000000004BE000205BE007B
:10F65000C05721005001BE004000BE0004712200CE
:10F66000050020006033B8007EB2020000000000F8
:10F6700074AF0200000000000002BE000203BE00E2
:10F680000800BE000A01BE0004B202000000000033
:10F690000004BE000205BE00405821005001BE001B
:10F6A0004000BE00843E2000050020006033B8000A
:10F6B0007EB202000000000074AF020000000000F3
:10F6C0000002BE000203BE000800BE000A01BE0028
:10F6D00004B20200000000000004BE000205BE00EB
:10F6E000C05821005001BE004000BE00440620006A
:10F6F000050020006033B8007EB202000000000068
:10F7000074AF0200000000000002BE000203BE0051
:10F710000800BE000A01BE0004B2020000000000A2
:10F720000004BE000205BE00405921005001BE0089
:10F730004000BE00A4002000050020006033B80097
:10F740007EB202000000000074AF02000000000062
:10F750000002BE000203BE000800BE000A01BE0097
:10F7600004B2020000000000E4AD0200000000004E
:10F77000C4592100009ABE000292BE00A0352100AB
:10F780005001BE004000BE000400200005802E0095
:10F790006687240077232400BEAB0200000000002F
:10F7A000E4AD020000000000445A2100009ABE00AF
:10F7B0000292BE00A03521003004BE002005BE002C
:10F7C000405A21005001BE004000BE0004802E00BF
:10F7D0006587240076012000070020007EB2020029
:10F7E0000000000074AF0200000000000002BE0034
:10F7F0000203BE000800BE000A01BE0004B20200FF
:10F80000000000000400200005002200F6052A0088
:10F8100027202400BEAB020000000000E4AD02007F
:10F8200000000000C45A2100009ABE000292BE00EF
:10F83000A03521003004BE002005BE00405A210042
:10F840005001BE004000BE0004802E0065872400E9
:10F8500076012000070020007EB2020000000000B8
:10F8600074AF0200000000000002BE000203BE00F0
:10F870000800BE000A01BE0004B202000000000041
:10F880000004BE000205BE00C05A21005001BE00A7
:10F890004000BE0004402E00B54025002600200098
:10F8A000070020007EB202000000000074AF0200DA
:10F8B000000000000002BE000203BE000800BE00FF
:10F8C0000A01BE0004B20200000000006022B8007D
:10F8D00056D62C00D71C2400BEAB0200000000004E
:10F8E000E4AD020000000000445B2100009ABE006D
:10F8F0000292BE00A03521003004BE002005BE00EB
:10F90000405A21005001BE004000BE0004802E007D
:10F910006587240076012000070020007EB20200E7
:10F920000000000074AF0200000000000002BE00F2
:10F930000203BE000800BE000A01BE0004B20200BD
:10F94000000000000004BE000205BE00C05A2100F5
:10F950005001BE004000BE0004402E00B54025000E
:10F9600026002000070020007EB2020000000000F8
:10F9700074AF0200000000000002BE000203BE00DF
:10F980000800BE000A01BE0004B202000000000030
:10F990000004BE000205BE00405B21005001BE0015
:10F9A0004000BE0004A02C00A5B923006033B800BD
:10F9B0007EB202000000000074AF020000000000F0
:10F9C0000002BE000203BE000800BE000A01BE0025
:10F9D00004B20200000000006022B80046782D004A
:10F9E00077192400BEAB020000000000E4AD020065
:10F9F00000000000C45B2100009ABE000292BE001D
:10FA0000A03521003004BE002005BE00405A210070
:10FA10005001BE004000BE0004802E006587240017
:10FA200076012000070020007EB2020000000000E6
:10FA300074AF0200000000000002BE000203BE001E
:10FA40000800BE000A01BE0004B20200000000006F
:10FA50000004BE000205BE00C05A21005001BE00D5
:10FA60004000BE0004402E00B540250026002000C6
:10FA7000070020007EB202000000000074AF020008
:10FA8000000000000002BE000203BE000800BE002D
:10FA90000A01BE0004B20200000000000004BE0023
:10FAA0000205BE00405B21005001BE004000BE00C8
:10FAB00004A02C00A5B923006033B8007EB2020078
:10FAC0000000000074AF0200000000000002BE0051
:10FAD0000203BE000800BE000A01BE0004B202001C
:10FAE000000000000004BE000205BE00C05B210053
:10FAF0005001BE004000BE0004102E00555F2000E3
:10FB00006033B8007EB202000000000074AF020053
:10FB1000000000000002BE000203BE000800BE009C
:10FB20000A01BE0004B20200000000006022B8001A
:10FB3000062D210037162400BEAB02000000000095
:10FB4000E4AD020000000000445C2100009ABE0009
:10FB50000292BE00A03521003004BE002005BE0088
:10FB6000405A21005001BE004000BE0004802E001B
:10FB70006587240076012000070020007EB2020085
:10FB80000000000074AF0200000000000002BE0090
:10FB90000203BE000800BE000A01BE0004B202005B
:10FBA000000000000004BE000205BE00C05A210093
:10FBB0005001BE004000BE0004402E00B5402500AC
:10FBC00026002000070020007EB202000000000096
:10FBD00074AF0200000000000002BE000203BE007D
:10FBE0000800BE000A01BE0004B2020000000000CE
:10FBF0000004BE000205BE00405B21005001BE00B3
:10FC00004000BE0004A02C00A5B923006033B8005A
:10FC10007EB202000000000074AF0200000000008D
:10FC20000002BE000203BE000800BE000A01BE00C2
:10FC300004B20200000000000004BE000205BE0085
:10FC4000C05B21005001BE004000BE0004102E0029
:10FC5000555F20006033B8007EB202000000000053
:10FC600074AF0200000000000002BE000203BE00EC
:10FC70000800BE000A01BE0004B20200000000003D
:10FC80000004BE000205BE00405C21005001BE0021
:10FC90004000BE0004682900850920006033B800D8
:10FCA0007EB202000000000074AF020000000000FD
:10FCB0000002BE000203BE000800BE000A01BE0032
:10FCC00004B20200000000006022B80006482800CC
:10FCD000E7122400BEAB020000000000E4AD020009
:10FCE00000000000C45C2100009ABE000292BE0029
:10FCF000A03521003004BE002005BE00405A21007E
:10FD00005001BE004000BE0004802E006587240024
:10FD100076012000070020007EB2020000000000F3
:10FD200074AF0200000000000002BE000203BE002B
:10FD30000800BE000A01BE0004B20200000000007C
:10FD40000004BE000205BE00C05A21005001BE00E2
:10FD50004000BE0004402E00B540250026002000D3
:10FD6000070020007EB202000000000074AF020015
:10FD7000000000000002BE000203BE000800BE003A
:10FD80000A01BE0004B20200000000000004BE0030
:10FD90000205BE00405B21005001BE004000BE00D5
:10FDA00004A02C00A5B923006033B8007EB2020085
:10FDB0000000000074AF0200000000000002BE005E
:10FDC0000203BE000800BE000A01BE0004B2020029
:10FDD000000000000004BE000205BE00C05B210060
:10FDE0005001BE004000BE0004102E00555F2000F0
:10FDF0006033B8007EB202000000000074AF020061
:10FE0000000000000002BE000203BE000800BE00A9
:10FE10000A01BE0004B20200000000000004BE009F
:10FE20000205BE00405C21005001BE004000BE0043
:10FE300004682900850920006033B8007EB2020002
:10FE40000000000074AF0200000000000002BE00CD
:10FE50000203BE000800BE000A01BE0004B2020098
:10FE6000000000000004BE000205BE00C05C2100CE
:10FE70005001BE004000BE0004242400F500200014
:10FE80006033B8007EB202000000000074AF0200D0
:10FE9000000000000002BE000203BE000800BE0019
:10FEA0000A01BE0004B20200000000006022B80097
:10FEB00006A02600870F2400BEAB02000000000051
:10FEC000E4AD020000000000445D2100009ABE0085
:10FED0000292BE00A03521003004BE002005BE0005
:10FEE000405A21005001BE004000BE0004802E0098
:10FEF0006587240076012000070020007EB2020002
:10FF00000000000074AF0200000000000002BE000C
:10FF10000203BE000800BE000A01BE0004B20200D7
:10FF2000000000000004BE000205BE00C05A21000F
:10FF30005001BE004000BE0004402E00B540250028
:10FF400026002000070020007EB202000000000012
:10FF500074AF0200000000000002BE000203BE00F9
:10FF60000800BE000A01BE0004B20200000000004A
:10FF70000004BE000205BE00405B21005001BE002F
:10FF80004000BE0004A02C00A5B923006033B800D7
:10FF90007EB202000000000074AF0200000000000A
:10FFA0000002BE000203BE000800BE000A01BE003F
:10FFB00004B20200000000000004BE000205BE0002
:10FFC000C05B21005001BE004000BE0004102E00A6
:10FFD000555F20006033B8007EB2020000000000D0
:10FFE00074AF0200000000000002BE000203BE0069
:10FFF0000800BE000A01BE0004B2020000000000BA
:020000040002F8
:100000000004BE000205BE00405C21005001BE009D
:100010004000BE0004682900850920006033B80054
:100020007EB202000000000074AF02000000000079
:100030000002BE000203BE000800BE000A01BE00AE
:1000400004B20200000000000004BE000205BE0071
:10005000C05C21005001BE004000BE00042424000A
:10006000F50020006033B8007EB2020000000000FE
:1000700074AF0200000000000002BE000203BE00D8
:100080000800BE000A01BE0004B202000000000029
:100090000004BE000205BE00405D21005001BE000C
:1000A0004000BE00046A2800150020006033B8003C
:1000B0007EB202000000000074AF020000000000E9
:1000C0000002BE000203BE000800BE000A01BE001E
:1000D00004B20200000000006022B8000680280080
:1000E000370C2400BEAB020000000000E4AD0200AB
:1000F00000000000C45D2100009ABE000292BE0014
:10010000A03521003004BE002005BE00405A210069
:100110005001BE004000BE0004802E006587240010
:1001200076012000070020007EB2020000000000DF
:1001300074AF0200000000000002BE000203BE0017
:100140000800BE000A01BE0004B202000000000068
:100150000004BE000205BE00C05A21005001BE00CE
:100160004000BE0004402E00B540250026002000BF
:10017000070020007EB202000000000074AF020001
:10018000000000000002BE000203BE000800BE0026
:100190000A01BE0004B20200000000000004BE001C
:1001A0000205BE00405B21005001BE004000BE00C1
:1001B00004A02C00A5B923006033B8007EB2020071
:1001C0000000000074AF0200000000000002BE004A
:1001D0000203BE000800BE000A01BE0004B2020015
:1001E000000000000004BE000205BE00C05B21004C
:1001F0005001BE004000BE0004102E00555F2000DC
:100200006033B8007EB202000000000074AF02004C
:10021000000000000002BE000203BE000800BE0095
:100220000A01BE0004B20200000000000004BE008B
:100230000205BE00405C21005001BE004000BE002F
:1002400004682900850920006033B8007EB20200EE
:100250000000000074AF0200000000000002BE00B9
:100260000203BE000800BE000A01BE0004B2020084
:10027000000000000004BE000205BE00C05C2100BA
:100280005001BE004000BE0004242400F500200000
:100290006033B8007EB202000000000074AF0200BC
:1002A000000000000002BE000203BE000800BE0005
:1002B0000A01BE0004B20200000000000004BE00FB
:1002C0000205BE00405D21005001BE004000BE009E
:1002D000046A2800150020006033B8007EB20200D6
:1002E0000000000074AF0200000000000002BE0029
:1002F0000203BE000800BE000A01BE0004B20200F4
:10030000000000000004BE000205BE00C05D210028
:100310005001BE004000BE00047122000500200014
:100320006033B8007EB202000000000074AF02002B
:10033000000000000002BE000203BE000800BE0074
:100340000A01BE0004B20200000000006022B800F2
:1003500006002400F7082400BEAB020000000000E5
:10036000E4AD020000000000445E2100009ABE00DF
:100370000292BE00A03521003004BE002005BE0060
:10038000405A21005001BE004000BE0004802E00F3
:100390006587240076012000070020007EB202005D
:1003A0000000000074AF0200000000000002BE0068
:1003B0000203BE000800BE000A01BE0004B2020033
:1003C000000000000004BE000205BE00C05A21006B
:1003D0005001BE004000BE0004402E00B540250084
:1003E00026002000070020007EB20200000000006E
:1003F00074AF0200000000000002BE000203BE0055
:100400000800BE000A01BE0004B2020000000000A5
:100410000004BE000205BE00405B21005001BE008A
:100420004000BE0004A02C00A5B923006033B80032
:100430007EB202000000000074AF02000000000065
:100440000002BE000203BE000800BE000A01BE009A
:1004500004B20200000000000004BE000205BE005D
:10046000C05B21005001BE004000BE0004102E0001
:10047000555F20006033B8007EB20200000000002B
:1004800074AF0200000000000002BE000203BE00C4
:100490000800BE000A01BE0004B202000000000015
:1004A0000004BE000205BE00405C21005001BE00F9
:1004B0004000BE0004682900850920006033B800B0
:1004C0007EB202000000000074AF020000000000D5
:1004D0000002BE000203BE000800BE000A01BE000A
:1004E00004B20200000000000004BE000205BE00CD
:1004F000C05C21005001BE004000BE000424240066
:10050000F50020006033B8007EB202000000000059
:1005100074AF0200000000000002BE000203BE0033
:100520000800BE000A01BE0004B202000000000084
:100530000004BE000205BE00405D21005001BE0067
:100540004000BE00046A2800150020006033B80097
:100550007EB202000000000074AF02000000000044
:100560000002BE000203BE000800BE000A01BE0079
:1005700004B20200000000000004BE000205BE003C
:10058000C05D21005001BE004000BE000471220089
:10059000050020006033B8007EB2020000000000B9
:1005A00074AF0200000000000002BE000203BE00A3
:1005B0000800BE000A01BE0004B2020000000000F4
:1005C0000004BE000205BE00405E21005001BE00D6
:1005D0004000BE00843E2000050020006033B800CB
:1005E0007EB202000000000074AF020000000000B4
:1005F0000002BE000203BE000800BE000A01BE00E9
:1006000004B20200000000006022B80006002000D2
:1006100097052400BEAB020000000000E4AD02001C
:1006200000000000C45E2100009ABE000292BE00DD
:10063000A03521003004BE002005BE00405A210034
:100640005001BE004000BE0004802E0065872400DB
:1006500076012000070020007EB2020000000000AA
:1006600074AF0200000000000002BE000203BE00E2
:100670000800BE000A01BE0004B202000000000033
:100680000004BE000205BE00C05A21005001BE0099
:100690004000BE0004402E00B5402500260020008A
:1006A000070020007EB202000000000074AF0200CC
:1006B000000000000002BE000203BE000800BE00F1
:1006C0000A01BE0004B20200000000000004BE00E7
:1006D0000205BE00405B21005001BE004000BE008C
:1006E00004A02C00A5B923006033B8007EB202003C
:1006F0000000000074AF0200000000000002BE0015
:100700000203BE000800BE000A01BE0004B20200DF
:10071000000000000004BE000205BE00C05B210016
:100720005001BE004000BE0004102E00555F2000A6
:100730006033B8007EB202000000000074AF020017
:10074000000000000002BE000203BE000800BE0060
:100750000A01BE0004B20200000000000004BE0056
:100760000205BE00405C21005001BE004000BE00FA
:1007700004682900850920006033B8007EB20200B9
:100780000000000074AF0200000000000002BE0084
:100790000203BE000800BE000A01BE0004B202004F
:1007A000000000000004BE000205BE00C05C210085
:1007B0005001BE004000BE0004242400F5002000CB
:1007C0006033B8007EB202000000000074AF020087
:1007D000000000000002BE000203BE000800BE00D0
:1007E0000A01BE0004B20200000000000004BE00C6
:1007F0000205BE00405D21005001BE004000BE0069
:10080000046A2800150020006033B8007EB20200A0
:100810000000000074AF0200000000000002BE00F3
:100820000203BE000800BE000A01BE0004B20200BE
:10083000000000000004BE000205BE00C05D2100F3
:100840005001BE004000BE000471220005002000DF
:100850006033B8007EB202000000000074AF0200F6
:10086000000000000002BE000203BE000800BE003F
:100870000A01BE0004B20200000000000004BE0035
:100880000205BE00405E21005001BE004000BE00D7
:10089000843E2000050020006033B8007EB20200D4
:1008A0000000000074AF0200000000000002BE0063
:1008B0000203BE000800BE000A01BE0004B202002E
:1008C000000000000004BE000205BE00C05E210062
:1008D0005001BE004000BE0044062000050020007C
:1008E0006033B8007EB202000000000074AF020066
:1008F000000000000002BE000203BE000800BE00AF
:100900000A01BE0004B20200000000006022B8002C
:100910000600200047022400BEAB020000000000D9
:10092000E4AD020000000000445F2100009ABE0018
:100930000292BE00A03521003004BE002005BE009A
:10094000405A21005001BE004000BE0004802E002D
:100950006587240076012000070020007EB2020097
:100960000000000074AF0200000000000002BE00A2
:100970000203BE000800BE000A01BE0004B202006D
:10098000000000000004BE000205BE00C05A2100A5
:100990005001BE004000BE0004402E00B5402500BE
:1009A00026002000070020007EB2020000000000A8
:1009B00074AF0200000000000002BE000203BE008F
:1009C0000800BE000A01BE0004B2020000000000E0
:1009D0000004BE000205BE00405B21005001BE00C5
:1009E0004000BE0004A02C00A5B923006033B8006D
:1009F0007EB202000000000074AF020000000000A0
:100A00000002BE000203BE000800BE000A01BE00D4
:100A100004B20200000000000004BE000205BE0097
:100A2000C05B21005001BE004000BE0004102E003B
:100A3000555F20006033B8007EB202000000000065
:100A400074AF0200000000000002BE000203BE00FE
:100A50000800BE000A01BE0004B20200000000004F
:100A60000004BE000205BE00405C21005001BE0033
:100A70004000BE0004682900850920006033B800EA
:100A80007EB202000000000074AF0200000000000F
:100A90000002BE000203BE000800BE000A01BE0044
:100AA00004B20200000000000004BE000205BE0007
:100AB000C05C21005001BE004000BE0004242400A0
:100AC000F50020006033B8007EB202000000000094
:100AD00074AF0200000000000002BE000203BE006E
:100AE0000800BE000A01BE0004B2020000000000BF
:100AF0000004BE000205BE00405D21005001BE00A2
:100B00004000BE00046A2800150020006033B800D1
:100B10007EB202000000000074AF0200000000007E
:100B20000002BE000203BE000800BE000A01BE00B3
:100B300004B20200000000000004BE000205BE0076
:100B4000C05D21005001BE004000BE0004712200C3
:100B5000050020006033B8007EB2020000000000F3
:100B600074AF0200000000000002BE000203BE00DD
:100B70000800BE000A01BE0004B20200000000002E
:100B80000004BE000205BE00405E21005001BE0010
:100B90004000BE00843E2000050020006033B80005
:100BA0007EB202000000000074AF020000000000EE
:100BB0000002BE000203BE000800BE000A01BE0023
:100BC00004B20200000000000004BE000205BE00E6
:100BD000C05E21005001BE004000BE00440620005F
:100BE000050020006033B8007EB202000000000063
:100BF00074AF0200000000000002BE000203BE004D
:100C00000800BE000A01BE0004B20200000000009D
:100C10000004BE000205BE00405F21005001BE007E
:100C20004000BE00A4002000050020006033B80092
:100C30007EB202000000000074AF0200000000005D
:100C40000002BE000203BE000800BE000A01BE0092
:100C500004B2020000000000E4AD02000000000049
:100C6000C45F2100009ABE000292BE00A03721009E
:100C70005001BE004000BE000400200005802E0090
:100C80006687240077232400BEAB0200000000002A
:100C9000E4AD02000000000044602100009ABE00A4
:100CA0000292BE00A03721003004BE002005BE0025
:100CB000406021005001BE004000BE0004802E00B4
:100CC0006587240076012000070020007EB2020024
:100CD0000000000074AF0200000000000002BE002F
:100CE0000203BE000800BE000A01BE0004B20200FA
:100CF000000000000400200005002200F6052A0084
:100D000027202400BEAB020000000000E4AD02007A
:100D100000000000C4602100009ABE000292BE00E4
:100D2000A03721003004BE002005BE004060210035
:100D30005001BE004000BE0004802E0065872400E4
:100D400076012000070020007EB2020000000000B3
:100D500074AF0200000000000002BE000203BE00EB
:100D60000800BE000A01BE0004B20200000000003C
:100D70000004BE000205BE00C06021005001BE009C
:100D80004000BE0004402E00B54025002600200093
:100D9000070020007EB202000000000074AF0200D5
:100DA000000000000002BE000203BE000800BE00FA
:100DB0000A01BE0004B20200000000006022B80078
:100DC00056D62C00D71C2400BEAB02000000000049
:100DD000E4AD02000000000044612100009ABE0062
:100DE0000292BE00A03721003004BE002005BE00E4
:100DF000406021005001BE004000BE0004802E0073
:100E00006587240076012000070020007EB20200E2
:100E10000000000074AF0200000000000002BE00ED
:100E20000203BE000800BE000A01BE0004B20200B8
:100E3000000000000004BE000205BE00C0602100EA
:100E40005001BE004000BE0004402E00B540250009
:100E500026002000070020007EB2020000000000F3
:100E600074AF0200000000000002BE000203BE00DA
:100E70000800BE000A01BE0004B20200000000002B
:100E80000004BE000205BE00406121005001BE000A
:100E90004000BE0004A02C00A5B923006033B800B8
:100EA0007EB202000000000074AF020000000000EB
:100EB0000002BE000203BE000800BE000A01BE0020
:100EC00004B20200000000006022B80046782D0045
:100ED00077192400BEAB020000000000E4AD020060
:100EE00000000000C4612100009ABE000292BE0012
:100EF000A03721003004BE002005BE004060210064
:100F00005001BE004000BE0004802E006587240012
:100F100076012000070020007EB2020000000000E1
:100F200074AF0200000000000002BE000203BE0019
:100F30000800BE000A01BE0004B20200000000006A
:100F40000004BE000205BE00C06021005001BE00CA
:100F50004000BE0004402E00B540250026002000C1
:100F6000070020007EB202000000000074AF020003
:100F7000000000000002BE000203BE000800BE0028
:100F80000A01BE0004B20200000000000004BE001E
:100F90000205BE00406121005001BE004000BE00BD
:100FA00004A02C00A5B923006033B8007EB2020073
:100FB0000000000074AF0200000000000002BE004C
:100FC0000203BE000800BE000A01BE0004B2020017
:100FD000000000000004BE000205BE00C061210048
:100FE0005001BE004000BE0004102E00555F2000DE
:100FF0006033B8007EB202000000000074AF02004F
:10100000000000000002BE000203BE000800BE0097
:101010000A01BE0004B20200000000006022B80015
:10102000062D210037162400BEAB02000000000090
:10103000E4AD02000000000044622100009ABE00FE
:101040000292BE00A03721003004BE002005BE0081
:10105000406021005001BE004000BE0004802E0010
:101060006587240076012000070020007EB2020080
:101070000000000074AF0200000000000002BE008B
:101080000203BE000800BE000A01BE0004B2020056
:10109000000000000004BE000205BE00C060210088
:1010A0005001BE004000BE0004402E00B5402500A7
:1010B00026002000070020007EB202000000000091
:1010C00074AF0200000000000002BE000203BE0078
:1010D0000800BE000A01BE0004B2020000000000C9
:1010E0000004BE000205BE00406121005001BE00A8
:1010F0004000BE0004A02C00A5B923006033B80056
:101100007EB202000000000074AF02000000000088
:101110000002BE000203BE000800BE000A01BE00BD
:1011200004B20200000000000004BE000205BE0080
:10113000C06121005001BE004000BE0004102E001E
:10114000555F20006033B8007EB20200000000004E
:1011500074AF0200000000000002BE000203BE00E7
:101160000800BE000A01BE0004B202000000000038
:101170000004BE000205BE00406221005001BE0016
:101180004000BE0004682900850920006033B800D3
:101190007EB202000000000074AF020000000000F8
:1011A0000002BE000203BE000800BE000A01BE002D
:1011B00004B20200000000006022B80006482800C7
:1011C000E7122400BEAB020000000000E4AD020004
:1011D00000000000C4622100009ABE000292BE001E
:1011E000A03721003004BE002005BE004060210071
:1011F0005001BE004000BE0004802E006587240020
:1012000076012000070020007EB2020000000000EE
:1012100074AF0200000000000002BE000203BE0026
:101220000800BE000A01BE0004B202000000000077
:101230000004BE000205BE00C06021005001BE00D7
:101240004000BE0004402E00B540250026002000CE
:10125000070020007EB202000000000074AF020010
:10126000000000000002BE000203BE000800BE0035
:101270000A01BE0004B20200000000000004BE002B
:101280000205BE00406121005001BE004000BE00CA
:1012900004A02C00A5B923006033B8007EB2020080
:1012A0000000000074AF0200000000000002BE0059
:1012B0000203BE000800BE000A01BE0004B2020024
:1012C000000000000004BE000205BE00C061210055
:1012D0005001BE004000BE0004102E00555F2000EB
:1012E0006033B8007EB202000000000074AF02005C
:1012F000000000000002BE000203BE000800BE00A5
:101300000A01BE0004B20200000000000004BE009A
:101310000205BE00406221005001BE004000BE0038
:1013200004682900850920006033B8007EB20200FD
:101330000000000074AF0200000000000002BE00C8
:101340000203BE000800BE000A01BE0004B2020093
:10135000000000000004BE000205BE00C0622100C3
:101360005001BE004000BE0004242400F50020000F
:101370006033B8007EB202000000000074AF0200CB
:10138000000000000002BE000203BE000800BE0014
:101390000A01BE0004B20200000000006022B80092
:1013A00006A02600870F2400BEAB0200000000004C
:1013B000E4AD02000000000044632100009ABE007A
:1013C0000292BE00A03721003004BE002005BE00FE
:1013D000406021005001BE004000BE0004802E008D
:1013E0006587240076012000070020007EB20200FD
:1013F0000000000074AF0200000000000002BE0008
:101400000203BE000800BE000A01BE0004B20200D2
:10141000000000000004BE000205BE00C060210004
:101420005001BE004000BE0004402E00B540250023
:1014300026002000070020007EB20200000000000D
:1014400074AF0200000000000002BE000203BE00F4
:101450000800BE000A01BE0004B202000000000045
:101460000004BE000205BE00406121005001BE0024
:101470004000BE0004A02C00A5B923006033B800D2
:101480007EB202000000000074AF02000000000005
:101490000002BE000203BE000800BE000A01BE003A
:1014A00004B20200000000000004BE000205BE00FD
:1014B000C06121005001BE004000BE0004102E009B
:1014C000555F20006033B8007EB2020000000000CB
:1014D00074AF0200000000000002BE000203BE0064
:1014E0000800BE000A01BE0004B2020000000000B5
:1014F0000004BE000205BE00406221005001BE0093
:101500004000BE0004682900850920006033B8004F
:101510007EB202000000000074AF02000000000074
:101520000002BE000203BE000800BE000A01BE00A9
:1015300004B20200000000000004BE000205BE006C
:10154000C06221005001BE004000BE0004242400FF
:10155000F50020006033B8007EB2020000000000F9
:1015600074AF0200000000000002BE000203BE00D3
:101570000800BE000A01BE0004B202000000000024
:101580000004BE000205BE00406321005001BE0001
:101590004000BE00046A2800150020006033B80037
:1015A0007EB202000000000074AF020000000000E4
:1015B0000002BE000203BE000800BE000A01BE0019
:1015C00004B20200000000006022B800068028007B
:1015D000370C2400BEAB020000000000E4AD0200A6
:1015E00000000000C4632100009ABE000292BE0009
:1015F000A03721003004BE002005BE00406021005D
:101600005001BE004000BE0004802E00658724000B
:1016100076012000070020007EB2020000000000DA
:1016200074AF0200000000000002BE000203BE0012
:101630000800BE000A01BE0004B202000000000063
:101640000004BE000205BE00C06021005001BE00C3
:101650004000BE0004402E00B540250026002000BA
:10166000070020007EB202000000000074AF0200FC
:10167000000000000002BE000203BE000800BE0021
:101680000A01BE0004B20200000000000004BE0017
:101690000205BE00406121005001BE004000BE00B6
:1016A00004A02C00A5B923006033B8007EB202006C
:1016B0000000000074AF0200000000000002BE0045
:1016C0000203BE000800BE000A01BE0004B2020010
:1016D000000000000004BE000205BE00C061210041
:1016E0005001BE004000BE0004102E00555F2000D7
:1016F0006033B8007EB202000000000074AF020048
:10170000000000000002BE000203BE000800BE0090
:101710000A01BE0004B20200000000000004BE0086
:101720000205BE00406221005001BE004000BE0024
:1017300004682900850920006033B8007EB20200E9
:101740000000000074AF0200000000000002BE00B4
:101750000203BE000800BE000A01BE0004B202007F
:10176000000000000004BE000205BE00C0622100AF
:101770005001BE004000BE0004242400F5002000FB
:101780006033B8007EB202000000000074AF0200B7
:10179000000000000002BE000203BE000800BE0000
:1017A0000A01BE0004B20200000000000004BE00F6
:1017B0000205BE00406321005001BE004000BE0093
:1017C000046A2800150020006033B8007EB20200D1
:1017D0000000000074AF0200000000000002BE0024
:1017E0000203BE000800BE000A01BE0004B20200EF
:1017F000000000000004BE000205BE00C06321001E
:101800005001BE004000BE0004712200050020000F
:101810006033B8007EB202000000000074AF020026
:10182000000000000002BE000203BE000800BE006F
:101830000A01BE0004B20200000000006022B800ED
:1018400006002400F7082400BEAB020000000000E0
:10185000E4AD02000000000044642100009ABE00D4
:101860000292BE00A03721003004BE002005BE0059
:10187000406021005001BE004000BE0004802E00E8
:101880006587240076012000070020007EB2020058
:101890000000000074AF0200000000000002BE0063
:1018A0000203BE000800BE000A01BE0004B202002E
:1018B000000000000004BE000205BE00C060210060
:1018C0005001BE004000BE0004402E00B54025007F
:1018D00026002000070020007EB202000000000069
:1018E00074AF0200000000000002BE000203BE0050
:1018F0000800BE000A01BE0004B2020000000000A1
:101900000004BE000205BE00406121005001BE007F
:101910004000BE0004A02C00A5B923006033B8002D
:101920007EB202000000000074AF02000000000060
:101930000002BE000203BE000800BE000A01BE0095
:1019400004B20200000000000004BE000205BE0058
:10195000C06121005001BE004000BE0004102E00F6
:10196000555F20006033B8007EB202000000000026
:1019700074AF0200000000000002BE000203BE00BF
:101980000800BE000A01BE0004B202000000000010
:101990000004BE000205BE00406221005001BE00EE
:1019A0004000BE0004682900850920006033B800AB
:1019B0007EB202000000000074AF020000000000D0
:1019C0000002BE000203BE000800BE000A01BE0005
:1019D00004B20200000000000004BE000205BE00C8
:1019E000C06221005001BE004000BE00042424005B
:1019F000F50020006033B8007EB202000000000055
:101A000074AF0200000000000002BE000203BE002E
:101A10000800BE000A01BE0004B20200000000007F
:101A20000004BE000205BE00406321005001BE005C
:101A30004000BE00046A2800150020006033B80092
:101A40007EB202000000000074AF0200000000003F
:101A50000002BE000203BE000800BE000A01BE0074
:101A600004B20200000000000004BE000205BE0037
:101A7000C06321005001BE004000BE00047122007E
:101A8000050020006033B8007EB2020000000000B4
:101A900074AF0200000000000002BE000203BE009E
:101AA0000800BE000A01BE0004B2020000000000EF
:101AB0000004BE000205BE00406421005001BE00CB
:101AC0004000BE00843E2000050020006033B800C6
:101AD0007EB202000000000074AF020000000000AF
:101AE0000002BE000203BE000800BE000A01BE00E4
:101AF00004B20200000000006022B80006002000CE
:101B000097052400BEAB020000000000E4AD020017
:101B100000000000C4642100009ABE000292BE00D2
:101B2000A03721003004BE002005BE004060210027
:101B30005001BE004000BE0004802E0065872400D6
:101B400076012000070020007EB2020000000000A5
:101B500074AF0200000000000002BE000203BE00DD
:101B60000800BE000A01BE0004B20200000000002E
:101B70000004BE000205BE00C06021005001BE008E
:101B80004000BE0004402E00B54025002600200085
:101B9000070020007EB202000000000074AF0200C7
:101BA000000000000002BE000203BE000800BE00EC
:101BB0000A01BE0004B20200000000000004BE00E2
:101BC0000205BE00406121005001BE004000BE0081
:101BD00004A02C00A5B923006033B8007EB2020037
:101BE0000000000074AF0200000000000002BE0010
:101BF0000203BE000800BE000A01BE0004B20200DB
:101C0000000000000004BE000205BE00C06121000B
:101C10005001BE004000BE0004102E00555F2000A1
:101C20006033B8007EB202000000000074AF020012
:101C3000000000000002BE000203BE000800BE005B
:101C40000A01BE0004B20200000000000004BE0051
:101C50000205BE00406221005001BE004000BE00EF
:101C600004682900850920006033B8007EB20200B4
:101C70000000000074AF0200000000000002BE007F
:101C80000203BE000800BE000A01BE0004B202004A
:101C9000000000000004BE000205BE00C06221007A
:101CA0005001BE004000BE0004242400F5002000C6
:101CB0006033B8007EB202000000000074AF020082
:101CC000000000000002BE000203BE000800BE00CB
:101CD0000A01BE0004B20200000000000004BE00C1
:101CE0000205BE00406321005001BE004000BE005E
:101CF000046A2800150020006033B8007EB202009C
:101D00000000000074AF0200000000000002BE00EE
:101D10000203BE000800BE000A01BE0004B20200B9
:101D2000000000000004BE000205BE00C0632100E8
:101D30005001BE004000BE000471220005002000DA
:101D40006033B8007EB202000000000074AF0200F1
:101D5000000000000002BE000203BE000800BE003A
:101D60000A01BE0004B20200000000000004BE0030
:101D70000205BE00406421005001BE004000BE00CC
:101D8000843E2000050020006033B8007EB20200CF
:101D90000000000074AF0200000000000002BE005E
:101DA0000203BE000800BE000A01BE0004B2020029
:101DB000000000000004BE000205BE00C064210057
:101DC0005001BE004000BE00440620000500200077
:101DD0006033B8007EB202000000000074AF020061
:101DE000000000000002BE000203BE000800BE00AA
:101DF0000A01BE0004B20200000000006022B80028
:101E00000600200047022400BEAB020000000000D4
:101E1000E4AD02000000000044652100009ABE000D
:101E20000292BE00A03721003004BE002005BE0093
:101E3000406021005001BE004000BE0004802E0022
:101E40006587240076012000070020007EB2020092
:101E50000000000074AF0200000000000002BE009D
:101E60000203BE000800BE000A01BE0004B2020068
:101E7000000000000004BE000205BE00C06021009A
:101E80005001BE004000BE0004402E00B5402500B9
:101E900026002000070020007EB2020000000000A3
:101EA00074AF0200000000000002BE000203BE008A
:101EB0000800BE000A01BE0004B2020000000000DB
:101EC0000004BE000205BE00406121005001BE00BA
:101ED0004000BE0004A02C00A5B923006033B80068
:101EE0007EB202000000000074AF0200000000009B
:101EF0000002BE000203BE000800BE000A01BE00D0
:101F000004B20200000000000004BE000205BE0092
:101F1000C06121005001BE004000BE0004102E0030
:101F2000555F20006033B8007EB202000000000060
:101F300074AF0200000000000002BE000203BE00F9
:101F40000800BE000A01BE0004B20200000000004A
:101F50000004BE000205BE00406221005001BE0028
:101F60004000BE0004682900850920006033B800E5
:101F70007EB202000000000074AF0200000000000A
:101F80000002BE000203BE000800BE000A01BE003F
:101F900004B20200000000000004BE000205BE0002
:101FA000C06221005001BE004000BE000424240095
:101FB000F50020006033B8007EB20200000000008F
:101FC00074AF0200000000000002BE000203BE0069
:101FD0000800BE000A01BE0004B2020000000000BA
:101FE0000004BE000205BE00406321005001BE0097
:101FF0004000BE00046A2800150020006033B800CD
:102000007EB202000000000074AF02000000000079
:102010000002BE000203BE000800BE000A01BE00AE
:1020200004B20200000000000004BE000205BE0071
:10203000C06321005001BE004000BE0004712200B8
:10204000050020006033B8007EB2020000000000EE
:1020500074AF0200000000000002BE000203BE00D8
:102060000800BE000A01BE0004B202000000000029
:102070000004BE000205BE00406421005001BE0005
:102080004000BE00843E2000050020006033B80000
:102090007EB202000000000074AF020000000000E9
:1020A0000002BE000203BE000800BE000A01BE001E
:1020B00004B20200000000000004BE000205BE00E1
:1020C000C06421005001BE004000BE004406200054
:1020D000050020006033B8007EB20200000000005E
:1020E00074AF0200000000000002BE000203BE0048
:1020F0000800BE000A01BE0004B202000000000099
:102100000004BE000205BE00406521005001BE0073
:102110004000BE00A4002000050020006033B8008D
:102120007EB202000000000074AF02000000000058
:102130000002BE000203BE000800BE000A01BE008D
:1021400004B2020000000000E4AD02000000000044
:10215000C4652100009ABE000292BE002038210012
:102160005001BE004000BE000400200005802E008B
:102170006687240077232400BEAB02000000000025
:10218000E4AD02000000000044672100009ABE0098
:102190000292BE00203821003004BE002005BE009F
:1021A000406721005001BE004000BE0004802E00A8
:1021B0006587240076012000070020007EB202001F
:1021C0000000000074AF0200000000000002BE002A
:1021D0000203BE000800BE000A01BE0004B20200F5
:1021E000000000000400200005002200F6052A007F
:1021F00027202400BEAB020000000000E4AD020076
:1022000000000000C4672100009ABE000292BE00D8
:10221000203821003004BE002005BE0040672100A8
:102220005001BE004000BE0004802E0065872400DF
:1022300076012000070020007EB2020000000000AE
:1022400074AF0200000000000002BE000203BE00E6
:102250000800BE000A01BE0004B202000000000037
:102260000004BE000205BE00C06721005001BE0090
:102270004000BE0004402E00B5402500260020008E
:10228000070020007EB202000000000074AF0200D0
:10229000000000000002BE000203BE000800BE00F5
:1022A0000A01BE0004B20200000000006022B80073
:1022B00056D62C00D71C2400BEAB02000000000044
:1022C000E4AD02000000000044682100009ABE0056
:1022D0000292BE00203821003004BE002005BE005E
:1022E000406721005001BE004000BE0004802E0067
:1022F0006587240076012000070020007EB20200DE
:102300000000000074AF0200000000000002BE00E8
:102310000203BE000800BE000A01BE0004B20200B3
:10232000000000000004BE000205BE00C0672100DE
:102330005001BE004000BE0004402E00B540250004
:1023400026002000070020007EB2020000000000EE
:1023500074AF0200000000000002BE000203BE00D5
:102360000800BE000A01BE0004B202000000000026
:102370000004BE000205BE00406821005001BE00FE
:102380004000BE0004A02C00A5B923006033B800B3
:102390007EB202000000000074AF020000000000E6
:1023A0000002BE000203BE000800BE000A01BE001B
:1023B00004B20200000000006022B80046782D0040
:1023C00077192400BEAB020000000000E4AD02005B
:1023D00000000000C4682100009ABE000292BE0006
:1023E000203821003004BE002005BE0040672100D7
:1023F0005001BE004000BE0004802E00658724000E
:1024000076012000070020007EB2020000000000DC
:1024100074AF0200000000000002BE000203BE0014
:102420000800BE000A01BE0004B202000000000065
:102430000004BE000205BE00C06721005001BE00BE
:102440004000BE0004402E00B540250026002000BC
:10245000070020007EB202000000000074AF0200FE
:10246000000000000002BE000203BE000800BE0023
:102470000A01BE0004B20200000000000004BE0019
:102480000205BE00406821005001BE004000BE00B1
:1024900004A02C00A5B923006033B8007EB202006E
:1024A0000000000074AF0200000000000002BE0047
:1024B0000203BE000800BE000A01BE0004B2020012
:1024C000000000000004BE000205BE00C06821003C
:1024D0005001BE004000BE0004102E00555F2000D9
:1024E0006033B8007EB202000000000074AF02004A
:1024F000000000000002BE000203BE000800BE0093
:102500000A01BE0004B20200000000006022B80010
:10251000062D210037162400BEAB0200000000008B
:10252000E4AD02000000000044692100009ABE00F2
:102530000292BE00203821003004BE002005BE00FB
:10254000406721005001BE004000BE0004802E0004
:102550006587240076012000070020007EB202007B
:102560000000000074AF0200000000000002BE0086
:102570000203BE000800BE000A01BE0004B2020051
:10258000000000000004BE000205BE00C06721007C
:102590005001BE004000BE0004402E00B5402500A2
:1025A00026002000070020007EB20200000000008C
:1025B00074AF0200000000000002BE000203BE0073
:1025C0000800BE000A01BE0004B2020000000000C4
:1025D0000004BE000205BE00406821005001BE009C
:1025E0004000BE0004A02C00A5B923006033B80051
:1025F0007EB202000000000074AF02000000000084
:102600000002BE000203BE000800BE000A01BE00B8
:1026100004B20200000000000004BE000205BE007B
:10262000C06821005001BE004000BE0004102E0012
:10263000555F20006033B8007EB202000000000049
:1026400074AF0200000000000002BE000203BE00E2
:102650000800BE000A01BE0004B202000000000033
:102660000004BE000205BE00406921005001BE000A
:102670004000BE0004682900850920006033B800CE
:102680007EB202000000000074AF020000000000F3
:102690000002BE000203BE000800BE000A01BE0028
:1026A00004B20200000000006022B80006482800C2
:1026B000E7122400BEAB020000000000E4AD0200FF
:1026C00000000000C4692100009ABE000292BE0012
:1026D000203821003004BE002005BE0040672100E4
:1026E0005001BE004000BE0004802E00658724001B
:1026F00076012000070020007EB2020000000000EA
:1027000074AF0200000000000002BE000203BE0021
:102710000800BE000A01BE0004B202000000000072
:102720000004BE000205BE00C06721005001BE00CB
:102730004000BE0004402E00B540250026002000C9
:10274000070020007EB202000000000074AF02000B
:10275000000000000002BE000203BE000800BE0030
:102760000A01BE0004B20200000000000004BE0026
:102770000205BE00406821005001BE004000BE00BE
:1027800004A02C00A5B923006033B8007EB202007B
:102790000000000074AF0200000000000002BE0054
:1027A0000203BE000800BE000A01BE0004B202001F
:1027B000000000000004BE000205BE00C068210049
:1027C0005001BE004000BE0004102E00555F2000E6
:1027D0006033B8007EB202000000000074AF020057
:1027E000000000000002BE000203BE000800BE00A0
:1027F0000A01BE0004B20200000000000004BE0096
:102800000205BE00406921005001BE004000BE002C
:1028100004682900850920006033B8007EB20200F8
:102820000000000074AF0200000000000002BE00C3
:102830000203BE000800BE000A01BE0004B202008E
:10284000000000000004BE000205BE00C0692100B7
:102850005001BE004000BE0004242400F50020000A
:102860006033B8007EB202000000000074AF0200C6
:10287000000000000002BE000203BE000800BE000F
:102880000A01BE0004B20200000000006022B8008D
:1028900006A02600870F2400BEAB02000000000047
:1028A000E4AD020000000000446A2100009ABE006E
:1028B0000292BE00203821003004BE002005BE0078
:1028C000406721005001BE004000BE0004802E0081
:1028D0006587240076012000070020007EB20200F8
:1028E0000000000074AF0200000000000002BE0003
:1028F0000203BE000800BE000A01BE0004B20200CE
:10290000000000000004BE000205BE00C0672100F8
:102910005001BE004000BE0004402E00B54025001E
:1029200026002000070020007EB202000000000008
:1029300074AF0200000000000002BE000203BE00EF
:102940000800BE000A01BE0004B202000000000040
:102950000004BE000205BE00406821005001BE0018
:102960004000BE0004A02C00A5B923006033B800CD
:102970007EB202000000000074AF02000000000000
:102980000002BE000203BE000800BE000A01BE0035
:1029900004B20200000000000004BE000205BE00F8
:1029A000C06821005001BE004000BE0004102E008F
:1029B000555F20006033B8007EB2020000000000C6
:1029C00074AF0200000000000002BE000203BE005F
:1029D0000800BE000A01BE0004B2020000000000B0
:1029E0000004BE000205BE00406921005001BE0087
:1029F0004000BE0004682900850920006033B8004B
:102A00007EB202000000000074AF0200000000006F
:102A10000002BE000203BE000800BE000A01BE00A4
:102A200004B20200000000000004BE000205BE0067
:102A3000C06921005001BE004000BE0004242400F3
:102A4000F50020006033B8007EB2020000000000F4
:102A500074AF0200000000000002BE000203BE00CE
:102A60000800BE000A01BE0004B20200000000001F
:102A70000004BE000205BE00406A21005001BE00F5
:102A80004000BE00046A2800150020006033B80032
:102A90007EB202000000000074AF020000000000DF
:102AA0000002BE000203BE000800BE000A01BE0014
:102AB00004B20200000000006022B8000680280076
:102AC000370C2400BEAB020000000000E4AD0200A1
:102AD00000000000C46A2100009ABE000292BE00FD
:102AE000203821003004BE002005BE0040672100D0
:102AF0005001BE004000BE0004802E006587240007
:102B000076012000070020007EB2020000000000D5
:102B100074AF0200000000000002BE000203BE000D
:102B20000800BE000A01BE0004B20200000000005E
:102B30000004BE000205BE00C06721005001BE00B7
:102B40004000BE0004402E00B540250026002000B5
:102B5000070020007EB202000000000074AF0200F7
:102B6000000000000002BE000203BE000800BE001C
:102B70000A01BE0004B20200000000000004BE0012
:102B80000205BE00406821005001BE004000BE00AA
:102B900004A02C00A5B923006033B8007EB2020067
:102BA0000000000074AF0200000000000002BE0040
:102BB0000203BE000800BE000A01BE0004B202000B
:102BC000000000000004BE000205BE00C068210035
:102BD0005001BE004000BE0004102E00555F2000D2
:102BE0006033B8007EB202000000000074AF020043
:102BF000000000000002BE000203BE000800BE008C
:102C00000A01BE0004B20200000000000004BE0081
:102C10000205BE00406921005001BE004000BE0018
:102C200004682900850920006033B8007EB20200E4
:102C30000000000074AF0200000000000002BE00AF
:102C40000203BE000800BE000A01BE0004B202007A
:102C5000000000000004BE000205BE00C0692100A3
:102C60005001BE004000BE0004242400F5002000F6
:102C70006033B8007EB202000000000074AF0200B2
:102C8000000000000002BE000203BE000800BE00FB
:102C90000A01BE0004B20200000000000004BE00F1
:102CA0000205BE00406A21005001BE004000BE0087
:102CB000046A2800150020006033B8007EB20200CC
:102CC0000000000074AF0200000000000002BE001F
:102CD0000203BE000800BE000A01BE0004B20200EA
:102CE000000000000004BE000205BE00C06A210012
:102CF0005001BE004000BE0004712200050020000B
:102D00006033B8007EB202000000000074AF020021
:102D1000000000000002BE000203BE000800BE006A
:102D20000A01BE0004B20200000000006022B800E8
:102D300006002400F7082400BEAB020000000000DB
:102D4000E4AD020000000000446B2100009ABE00C8
:102D50000292BE00203821003004BE002005BE00D3
:102D6000406721005001BE004000BE0004802E00DC
:102D70006587240076012000070020007EB2020053
:102D80000000000074AF0200000000000002BE005E
:102D90000203BE000800BE000A01BE0004B2020029
:102DA000000000000004BE000205BE00C067210054
:102DB0005001BE004000BE0004402E00B54025007A
:102DC00026002000070020007EB202000000000064
:102DD00074AF0200000000000002BE000203BE004B
:102DE0000800BE000A01BE0004B20200000000009C
:102DF0000004BE000205BE00406821005001BE0074
:102E00004000BE0004A02C00A5B923006033B80028
:102E10007EB202000000000074AF0200000000005B
:102E20000002BE000203BE000800BE000A01BE0090
:102E300004B20200000000000004BE000205BE0053
:102E4000C06821005001BE004000BE0004102E00EA
:102E5000555F20006033B8007EB202000000000021
:102E600074AF0200000000000002BE000203BE00BA
:102E70000800BE000A01BE0004B20200000000000B
:102E80000004BE000205BE00406921005001BE00E2
:102E90004000BE0004682900850920006033B800A6
:102EA0007EB202000000000074AF020000000000CB
:102EB0000002BE000203BE000800BE000A01BE0000
:102EC00004B20200000000000004BE000205BE00C3
:102ED000C06921005001BE004000BE00042424004F
:102EE000F50020006033B8007EB202000000000050
:102EF00074AF0200000000000002BE000203BE002A
:102F00000800BE000A01BE0004B20200000000007A
:102F10000004BE000205BE00406A21005001BE0050
:102F20004000BE00046A2800150020006033B8008D
:102F30007EB202000000000074AF0200000000003A
:102F40000002BE000203BE000800BE000A01BE006F
:102F500004B20200000000000004BE000205BE0032
:102F6000C06A21005001BE004000BE000471220072
:102F7000050020006033B8007EB2020000000000AF
:102F800074AF0200000000000002BE000203BE0099
:102F90000800BE000A01BE0004B2020000000000EA
:102FA0000004BE000205BE00406B21005001BE00BF
:102FB0004000BE00843E2000050020006033B800C1
:102FC0007EB202000000000074AF020000000000AA
:102FD0000002BE000203BE000800BE000A01BE00DF
:102FE00004B20200000000006022B80006002000C9
:102FF00097052400BEAB020000000000E4AD020013
:1030000000000000C46B2100009ABE000292BE00C6
:10301000203821003004BE002005BE00406721009A
:103020005001BE004000BE0004802E0065872400D1
:1030300076012000070020007EB2020000000000A0
:1030400074AF0200000000000002BE000203BE00D8
:103050000800BE000A01BE0004B202000000000029
:103060000004BE000205BE00C06721005001BE0082
:103070004000BE0004402E00B54025002600200080
:10308000070020007EB202000000000074AF0200C2
:10309000000000000002BE000203BE000800BE00E7
:1030A0000A01BE0004B20200000000000004BE00DD
:1030B0000205BE00406821005001BE004000BE0075
:1030C00004A02C00A5B923006033B8007EB2020032
:1030D0000000000074AF0200000000000002BE000B
:1030E0000203BE000800BE000A01BE0004B20200D6
:1030F000000000000004BE000205BE00C068210000
:103100005001BE004000BE0004102E00555F20009C
:103110006033B8007EB202000000000074AF02000D
:10312000000000000002BE000203BE000800BE0056
:103130000A01BE0004B20200000000000004BE004C
:103140000205BE00406921005001BE004000BE00E3
:1031500004682900850920006033B8007EB20200AF
:103160000000000074AF0200000000000002BE007A
:103170000203BE000800BE000A01BE0004B2020045
:10318000000000000004BE000205BE00C06921006E
:103190005001BE004000BE0004242400F5002000C1
:1031A0006033B8007EB202000000000074AF02007D
:1031B000000000000002BE000203BE000800BE00C6
:1031C0000A01BE0004B20200000000000004BE00BC
:1031D0000205BE00406A21005001BE004000BE0052
:1031E000046A2800150020006033B8007EB2020097
:1031F0000000000074AF0200000000000002BE00EA
:103200000203BE000800BE000A01BE0004B20200B4
:10321000000000000004BE000205BE00C06A2100DC
:103220005001BE004000BE000471220005002000D5
:103230006033B8007EB202000000000074AF0200EC
:10324000000000000002BE000203BE000800BE0035
:103250000A01BE0004B20200000000000004BE002B
:103260000205BE00406B21005001BE004000BE00C0
:10327000843E2000050020006033B8007EB20200CA
:103280000000000074AF0200000000000002BE0059
:103290000203BE000800BE000A01BE0004B2020024
:1032A000000000000004BE000205BE00C06B21004B
:1032B0005001BE004000BE00440620000500200072
:1032C0006033B8007EB202000000000074AF02005C
:1032D000000000000002BE000203BE000800BE00A5
:1032E0000A01BE0004B20200000000006022B80023
:1032F0000600200047022400BEAB020000000000D0
:10330000E4AD020000000000446C2100009ABE0001
:103310000292BE00203821003004BE002005BE000D
:10332000406721005001BE004000BE0004802E0016
:103330006587240076012000070020007EB202008D
:103340000000000074AF0200000000000002BE0098
:103350000203BE000800BE000A01BE0004B2020063
:10336000000000000004BE000205BE00C06721008E
:103370005001BE004000BE0004402E00B5402500B4
:1033800026002000070020007EB20200000000009E
:1033900074AF0200000000000002BE000203BE0085
:1033A0000800BE000A01BE0004B2020000000000D6
:1033B0000004BE000205BE00406821005001BE00AE
:1033C0004000BE0004A02C00A5B923006033B80063
:1033D0007EB202000000000074AF02000000000096
:1033E0000002BE000203BE000800BE000A01BE00CB
:1033F00004B20200000000000004BE000205BE008E
:10340000C06821005001BE004000BE0004102E0024
:10341000555F20006033B8007EB20200000000005B
:1034200074AF0200000000000002BE000203BE00F4
:103430000800BE000A01BE0004B202000000000045
:103440000004BE000205BE00406921005001BE001C
:103450004000BE0004682900850920006033B800E0
:103460007EB202000000000074AF02000000000005
:103470000002BE000203BE000800BE000A01BE003A
:1034800004B20200000000000004BE000205BE00FD
:10349000C06921005001BE004000BE000424240089
:1034A000F50020006033B8007EB20200000000008A
:1034B00074AF0200000000000002BE000203BE0064
:1034C0000800BE000A01BE0004B2020000000000B5
:1034D0000004BE000205BE00406A21005001BE008B
:1034E0004000BE00046A2800150020006033B800C8
:1034F0007EB202000000000074AF02000000000075
:103500000002BE000203BE000800BE000A01BE00A9
:1035100004B20200000000000004BE000205BE006C
:10352000C06A21005001BE004000BE0004712200AC
:10353000050020006033B8007EB2020000000000E9
:1035400074AF0200000000000002BE000203BE00D3
:103550000800BE000A01BE0004B202000000000024
:103560000004BE000205BE00406B21005001BE00F9
:103570004000BE00843E2000050020006033B800FB
:103580007EB202000000000074AF020000000000E4
:103590000002BE000203BE000800BE000A01BE0019
:1035A00004B20200000000000004BE000205BE00DC
:1035B000C06B21005001BE004000BE004406200048
:1035C000050020006033B8007EB202000000000059
:1035D00074AF0200000000000002BE000203BE0043
:1035E0000800BE000A01BE0004B202000000000094
:1035F0000004BE000205BE00406C21005001BE0068
:103600004000BE00A4002000050020006033B80088
:103610007EB202000000000074AF02000000000053
:103620000002BE000203BE000800BE000A01BE0088
:1036300004B2020000000000E4AD0200000000003F
:10364000C46C2100009ABE000292BE00A039210085
:103650005001BE004000BE0003F0A1006022B8008F
:1036600006002400F7082400BEAB020000000000A2
:1036700058AE02000000000020B7880031B7880073
:10368000A03921005001BE004000BE000004BE0071
:103690000205BE000BF0A10020B7800031B780000A
:1036A000823E20000289B900020178006002B90060
:1036B0008401780003014100833E20000300B8002C
:1036C000010141008200780094AF02000000000078
:1036D0000002BE000203BE000800BE000A01BE00D8
:1036E00004B20200000000006022B80006002000C2
:1036F00097052400BEAB02000000000058AE020097
:103700000000000040B7880051B78800A0392100B0
:103710005001BE004000BE000004BE000205BE0015
:103720000BF0A10020B7800031B78000823E20005E
:103730000289B900020178006002B90084017800B2
:1037400003014100833E20000300B8000101410055
:103750008200780094AF0200000000000002BE006A
:103760000203BE000800BE000A01BE0004B202004F
:10377000000000000004BE000205BE0040B780004B
:1037800051B78000420620000289B900020178008A
:103790006002B90084017800030141004306200063
:1037A0000300B800010141008200780094AF0200DC
:1037B000000000000002BE000203BE000800BE00C0
:1037C0000A01BE0004B20200000000006022B8003E
:1037D0000600200047022400BEAB020000000000EB
:1037E00058AE02000000000060B7880071B7880082
:1037F000A03921005001BE004000BE000004BE0000
:103800000205BE000BF0A10020B7800031B7800098
:10381000823E20000289B900020178006002B900EE
:103820008401780003014100833E20000300B800BA
:10383000010141008200780094AF02000000000006
:103840000002BE000203BE000800BE000A01BE0066
:1038500004B20200000000000004BE000205BE0029
:1038600040B7800051B78000420620000289B900AD
:10387000020178006002B900840178000301410070
:10388000430620000300B8000101410082007800D7
:1038900094AF0200000000000002BE000203BE0060
:1038A0000800BE000A01BE0004B2020000000000D1
:1038B0000004BE000205BE0060B7800071B7800042
:1038C0006A09B900020178006002B9008401780039
:1038D00003014100A30020000300B80001014100E2
:1038E0008200780094AF0200000000000002BE00D9
:1038F0000203BE000800BE000A01BE0004B20200BE
:103900000000000058AE02000000000080B78800F0
:1039100091B78800A03921005001BE004000BE00D0
:1039200003F0A1006022B800060020004702240036
:10393000B2B00200000000000004BE000205BE009C
:1039400020B7800031B78000027122000289B900DF
:10395000020178006002B90084017800030141008F
:10396000037122000300B8000101410082007800C9
:1039700094AF0200000000000002BE000203BE007F
:103980000800BE000A01BE0004B2020000000000F0
:103990000004BE000205BE0040B7800051B78000A1
:1039A000823E20000289B900020178006002B9005D
:1039B0008401780003014100833E20000300B80029
:1039C000010141008200780094AF02000000000075
:1039D0000002BE000203BE000800BE000A01BE00D5
:1039E00004B20200000000000004BE000205BE0098
:1039F00060B7800071B78000420620000289B900DC
:103A0000020178006002B9008401780003014100DE
:103A1000430620000300B800010141008200780045
:103A200094AF0200000000000002BE000203BE00CE
:103A30000800BE000A01BE0004B20200000000003F
:103A40000004BE000205BE0080B7800091B7800070
:103A50006A09B900020178006002B90084017800A7
:103A600003014100A30020000300B8000101410050
:103A70008200780094AF0200000000000002BE0047
:103A80000203BE000800BE000A01BE0004B202002C
:103A90000000000058AE020000000000A0B788003F
:103AA000B1B78800A03921005001BE004000BE001F
:103AB00003F0A1006022B800060020009705240052
:103AC000B2B00200000000000004BE000205BE000B
:103AD00020B7800031B78000026A28000289B9004F
:103AE000020178006102B9008401780003014100FD
:103AF000036A28000300B800010141008200780039
:103B000094AF0200000000000002BE000203BE00ED
:103B10000800BE000A01BE0004B20200000000005E
:103B20000004BE000205BE0040B7800051B780000F
:103B3000027122000289B900020178006002B90016
:103B40008401780003014100037122000300B800E2
:103B5000010141008200780094AF020000000000E3
:103B60000002BE000203BE000800BE000A01BE0043
:103B700004B20200000000000004BE000205BE0006
:103B800060B7800071B78000823E20000289B900D2
:103B9000020178006002B90084017800030141004D
:103BA000833E20000300B80001014100820078003C
:103BB00094AF0200000000000002BE000203BE003D
:103BC0000800BE000A01BE0004B2020000000000AE
:103BD0000004BE000205BE0080B7800091B78000DF
:103BE000420620000289B900020178006002B90093
:103BF0008401780003014100430620000300B8005F
:103C0000010141008200780094AF02000000000032
:103C10000002BE000203BE000800BE000A01BE0092
:103C200004B20200000000000004BE000205BE0055
:103C3000A0B78000B1B780006A09B900020178001E
:103C40006002B9008401780003014100A300200054
:103C50000300B800010141008200780094AF020027
:103C6000000000000002BE000203BE000800BE000B
:103C70000A01BE0004B202000000000058AE0200BB
:103C800000000000C0B78800D1B788004F05BE0013
:103C90004F04BE000080FA00000006000000FA0099
:103CA000889FBE002009210090407800B0C3B30077
:103CB00080CF500017003C00200921001040780000
:103CC0000004FB00507B8000617B800002F8240030
:103CD000337C24009CB102000000000002F02F00A1
:103CE000F377240072AC020000000000C241DD0046
:103CF000A2F92000028141000089BE0020092100B4
:103D0000104078008040E800200921000148780038
:103D10001E00370030092100104078000004FB002D
:103D2000507B8000617B800002F82400337C2400FB
:103D30009CB102000000000002F02F00F377240085
:103D400072AC020000000000C241DD00A2F92000B8
:103D5000028141000089BE00300921001040780036
:103D60008040E80030092100014878003009210036
:103D700090407800C0C3B30080CF500003003A00E9
:103D8000300921008040EB00014878006000B80055
:103D90005084880061848800400921008040EB0045
:103DA00001487800140037004009210010407800D5
:103DB0000000FB00C200DD00A0F9200000804000F0
:103DC0001002BE0050848000618480000001BE00AB
:103DD0000400BE00F0AA0200000000005084880029
:103DE0006184880040092100104078008040E8008C
:103DF00040092100014878004009210090407800E6
:103E0000200921001040780080CF5000E6FF3500E7
:103E100058848000698480002009210010407800C7
:103E20000000FB00CF80DE009AAF0200000000001F
:103E30000001BE000800BE0072AC020000000000DD
:103E400070848800818488000000000070848000F5
:103E50008184800018C0B3006011B800E0AD02009A
:103E6000000000000000E00001003C000044EB0006
:103E70000804E0000300320030332300A00D880066
:103E800049003700708480008184800001F0A10027
:103E900018C0B30002F82400337C2400E0AD020017
:103EA000000000000000E00001003C000044EB00C6
:103EB0000804E0000500320000F82400317C2400F2
:103EC000708488008184880024003700708480001A
:103ED0008184800001F0A1009EAD0200000000007E
:103EE0006022B8000600200087002400B2B0020063
:103EF000000000006022B80006802800370D240072
:103F0000F4A902000000000008B202000000000056
:103F1000708488008184880070848000818480009F
:103F200001F0A10018C0B30002F82400337C240083
:103F3000E0AD0200000000000000E00001003C00D5
:103F40000044EB000804E0000400320000F8240004
:103F5000317C240070848800818488007084800013
:103F60008184800001F0A1009EAD020000000000ED
:103F70006022B80006FE2F00F70E2400B2B0020047
:103F8000000000006022B800069F2600870F240072
:103F9000BEAB020000000000F2AE02000000000014
:103FA00000007800A00D88000080200010407800FC
:103FB000E14F5000FE003A00708480008184800050
:103FC0009EAD0200000000006022B80006802800BC
:103FD000370C2400BEAB02000000000058AE020007
:103FE0000000000000007800B08488007884800021
:103FF00089848000B1848000007122000088B900AB
:1040000000007800CF80DE009AAF020000000000C0
:104010000001BE000800BE00EEAA02000000000081
:10402000B0AE02000000000000007800CF80DE008B
:1040300094AF0200000000006022B80006002400D7
:10404000F7082400BEAB02000000000058AE0200DA
:104050000000000000007800C084880078848000A0
:1040600089848000B1848000007122000088B9003A
:1040700000007800CF80DE009AAF02000000000050
:104080000001BE000800BE00EEAA02000000000011
:104090000004BE00C1848000803E20000088B9007A
:1040A00000007800CF80DE009AAF02000000000020
:1040B0000001BE000800BE00EEAA020000000000E1
:1040C000B0AE02000000000000007800CF80DE00EB
:1040D00094AF0200000000006022B800060020003B
:1040E00097052400BEAB02000000000058AE02009D
:1040F0000000000000007800D084880078848000F0
:1041000089848000B1848000007122000088B90099
:1041100000007800CF80DE009AAF020000000000AF
:104120000001BE000800BE00EEAA02000000000070
:104130000004BE00C1848000803E20000088B900D9
:1041400000007800CF80DE009AAF0200000000007F
:104150000001BE000800BE00EEAA02000000000040
:104160000004BE00D1848000400620000088B90011
:1041700000007800CF80DE009AAF0200000000004F
:104180000001BE000800BE00EEAA02000000000010
:10419000B0AE02000000000000007800CF80DE001A
:1041A00094AF0200000000006022B800060020006A
:1041B00047022400BEAB02000000000058AE02001F
:1041C0000000000000007800E0848800788480000F
:1041D00089848000B1848000007122000088B900C9
:1041E00000007800CF80DE009AAF020000000000DF
:1041F0000001BE000800BE00EEAA020000000000A0
:104200000004BE00C1848000803E20000088B90008
:1042100000007800CF80DE009AAF020000000000AE
:104220000001BE000800BE00EEAA0200000000006F
:104230000004BE00D1848000400620000088B90040
:1042400000007800CF80DE009AAF0200000000007E
:104250000001BE000800BE00EEAA0200000000003F
:104260000004BE00E08480006A00B900000078000D
:10427000CF80DE009AAF0200000000000001BE0007
:104280000800BE00EEAA020000000000B0AE02006E
:104290000000000000007800F08488004200020066
:1042A00002000000B084800000407800F82B02007B
:1042B00002000000C084800000407800F82B02005B
:1042C00002000000A624020002000000D08480004A
:1042D00000407800F82B020002000000E08480001B
:1042E00000407800F82B020002000000F0848000FB
:1042F00000407800F82B020002000000C613020004
:1043000002000000BE15020002000000503402004E
:1043100002000000000A2100104078000004E000C4
:1043200003003A00361902000200000004003700C2
:10433000000A210010407800F82B02000200000063
:10434000100A2100104078000004E00003003A0049
:10435000361902000200000004003700100A210094
:1043600010407800F82B020002000000200A210013
:1043700010407800F82B020002000000A624020082
:1043800002000000300A210010407800F82B0200E3
:10439000020000000040EB00F82B020002000000C9
:1043A00026170200020000004E1602000200000064
:1043B0004F04BE000080FA00000006000000FA0072
:1043C0009621EF00A021EF006000B800507B88002C
:1043D000617B88000000EB00C08588000000EB00D6
:1043E000D08588000000EB00E08588000000EB002D
:1043F000F08588000000EB00008688000080200027
:1044000010407800E14F50001E003A002A000200E0
:1044100002000000B620020002000000C0858000FB
:1044200000407800F82B020002000000D0858000D8
:1044300000407800F82B020002000000A6240200D1
:1044400002000000E085800000407800F82B0200A8
:1044500002000000F085800000407800F82B020088
:10446000020000000086800000407800F82B020067
:10447000020000004E160200020000002215020099
:10448000020000000080FA00000006000000FA00B0
:104490009621EF00A021EF0000012400A00D88006C
:1044A0000080FA00000006000000FA00F4C2A80034
:1044B000F0C2A9000080FA00000006000000FA0027
:1044C000F4C2A900C2420700F0C2A9000080FA00AD
:1044D000000006000000FA00D8A2A8000080FA0040
:1044E000000006000000FA00D11680000002200043
:1044F000008060000000E00006003200F522A80005
:10450000A00D21008040EB00014878000040EB0046
:1045100005003700F522A900A00D210011C0B3004D
:104520000148780010C0B3000080FA0000000600C7
:104530000000FA00E2C4A800E2E4A800E364A800D6
:10454000E3C4A800E3E4A800C8C2A800C8E2A80029
:10455000C962A800C9C2A800C9E2A800DE04A90077
:104560001019800000D0A10000E0A10000F0A1001F
:104570001019880010C0B30024E3B70000198000B0
:104580000050A0000060A0000070A000001988008A
:1045900021198000F00F2E00808060000050200064
:1045A0000100700020198800001980000080A1001F
:1045B0000090A100001988002043A9001119800073
:1045C00030F82F00008060001019880021E3A80057
:1045D0003023EF00C0E82200A1DB2300A09D88006B
:1045E000B19D8800803E21008040EB0001487800AA
:1045F000903E21008040EB0001487800A03E210061
:104600008040EB0001487800B03E21008040EB0084
:1046100001487800C03E21008040EB00014878004E
:104620000000EB00F09D8800803B21008040EB0003
:104630000148780048000700803B210011C0B3000A
:10464000014878000080FA00000006000000FA002F
:10465000E2C4A900E2E4A900E364A900E3C4A9005C
:10466000E3E4A900E2C4A800E2E4A800E364A8002F
:10467000E3C4A800E3E4A800C8C2A800C8E2A800F8
:10468000C962A800C9C2A800C9E2A800DE04A90046
:104690001019800000D0A10000E0A10000F0A100EE
:1046A0001019880010C0B30024E3B700001980007F
:1046B0000050A0000060A0000070A0000019880059
:1046C00021198000F00F2E00808060000050200033
:1046D0000100700020198800001980000080A100EE
:1046E0000090A100001988002043A9001119800042
:1046F00030F82F00008060001019880021E3A80026
:104700003023EF00C0E82200A1DB2300A09D880039
:10471000B19D8800803E21008040EB000148780078
:10472000903E21008040EB0001487800A03E21002F
:104730008040EB0001487800B03E21008040EB0053
:1047400001487800C03E21008040EB00014878001D
:104750000080FA00000006003400FA00889FBE00C6
:104760000000EB00600F98006000B8002007980080
:10477000310798004119800000FE2F000080600082
:104780006000B300401988000040EB00004F780043
:10479000120037002023A80000000000001980004C
:1047A000610060000000E000FCFF32002023A9004F
:1047B00000188000600F98006E089000CF80DE0027
:1047C0002E019000BE01900002004000838048004E
:1047D00020079800310798001E4FE8001E4078001F
:1047E000E94F5000EBFF34002E009000BE00900017
:1047F000A200200003002000F6AC02000000000030
:10480000600F98000000EB00700F98006000B80087
:1048100040079800510798004119800000FE2F00C2
:10482000008060007000B300401988000040EB0079
:10483000004F7800120037002023A800000000007D
:1048400000198000610060000000E000FCFF320001
:104850002023A90000188000700F98007E089000A7
:10486000CF80DE004E019000DE019000020040008B
:104870008380480040079800510798001E4FE800C9
:104880001E407800E94F5000EBFF34004E009000CE
:10489000DE009000A200200003002000F6AC020021
:1048A00000000000700F9800108020001040780079
:1048B000E34F500029003A000000EB001007980079
:1048C0006000B800600798007107980041198000E7
:1048D00000FE2F0000806000B000B3004019880087
:1048E0000040EB00004F7800120037002023A800A2
:1048F0000000000000198000610060000000E0007E
:10490000FCFF32002023A900001880001007980047
:104910001E009000CF80DE006E019000FE0190002E
:1049200002004000838048006007980071079800EB
:104930001E4FE8001E407800E94F5000EBFF3400A6
:104940006E009000FE009000A200200003002000F6
:10495000F6AC020000000000100798000000EB0019
:10496000001798006000B800000F9800110F980021
:104970004119800000FE2F0000806000E000B300BD
:10498000401988000040EB00004F7800120037000B
:104990002023A800000000000019800061006000D2
:1049A0000000E000FCFF32002023A9000018800076
:1049B000001798000E109000CF80DE000E099000C6
:1049C0009E0990000200400083804800000F98007C
:1049D000110F98001E4FE8001E407800E94F50006C
:1049E000EBFF34000E0890009E089000A20020000B
:1049F00003002000F6AC0200000000000017980041
:104A00000000EB00101798006000B800200F98001D
:104A1000310F98004119800000FE2F0000806000D7
:104A2000F000B300401988000040EB00004F780010
:104A3000120037002023A8000000000000198000A9
:104A4000610060000000E000FCFF32002023A900AC
:104A500000188000101798001E109000CF80DE0014
:104A60002E099000BE09900002004000838048009B
:104A7000200F9800310F98001E4FE8001E4078006C
:104A8000E94F5000EBFF34002E089000BE08900064
:104A9000A200200003002000F6AC0200000000008D
:104AA000101798006E089000CF80DE009AAF0200C9
:104AB0000000000002002400E30424009CB1020076
:104AC0000000000020179800311798007E08900021
:104AD000CF80DE009AAF0200000000000200240038
:104AE000E30424009CB1020000000000401798007D
:104AF000511798001080200010407800E34F5000BC
:104B00000A003A001E009000CF80DE009AAF02003B
:104B10000000000002002400E30424009CB1020015
:104B200000000000400F9800510F98000E109000F8
:104B3000CF80DE009AAF02000000000002002400D7
:104B4000E30424009CB102000000000060179800FC
:104B5000711798001E109000CF80DE009AAF0200FF
:104B60000000000002002400E30424009CB10200C5
:104B700000000000001F9800111F980002002D0087
:104B8000435224002E109000BE109000EEAA0200A6
:104B90000000000001F0A2009EAD02000000000035
:104BA000E483230045142800367E2D0027FB2300D4
:104BB000B2B002000000000008B2020000000000D5
:104BC000009E8800119E880002002D0043522400A0
:104BD0004E109000DE109000EEAA020000000000CF
:104BE00001F0A2009EAD020000000000E48323005B
:104BF00045142800367E2D0027FB2300B2B00200AA
:104C00000000000008B2020000000000209E8800A2
:104C1000319E88001080200010407800E34F500043
:104C200013003A0002002D00435224004E08900069
:104C3000DE089000EEAA02000000000001F0A200D1
:104C40009EAD020000000000E4832300451428000C
:104C5000367E2D0027FB2300B2B0020000000000CA
:104C600008B2020000000000409E8800519E8800AB
:104C700002002D00435224006E109000FE109000A0
:104C8000EEAA02000000000001F0A2009EAD0200AA
:104C900000000000E483230045142800367E2D0028
:104CA00027FB2300B2B002000000000008B202009F
:104CB00000000000609E8800719E880002002D00A8
:104CC000435224000E1890009E189000EEAA020095
:104CD0000000000001F0A2009EAD020000000000F4
:104CE000E483230045142800367E2D0027FB230093
:104CF000B2B002000000000008B202000000000094
:104D0000809E8800919E8800803B210010407800A2
:104D1000E14F500031013A00A09E8000B19E80001A
:104D20000200200003122400F0AA0200000000008C
:104D30000002BE00009E8000119E800018C0B300DB
:104D40000001BE000400BE00DCAD02000000000057
:104D50000000E000010035000044EB000804E00022
:104D600085003A00A09E8000B19E800002002000D5
:104D700003122400EEAA0200000000000002BE00A0
:104D8000009E8000119E800018C0B3000001BE008C
:104D90000400BE00E0AD0200000000000000E000E2
:104DA00001003C000044EB000804E00072003A00FF
:104DB000C09E8000D19E80000200200003122400CB
:104DC000F0AA0200000000000002BE00209E800049
:104DD000319E800018C0B3000001BE000400BE0078
:104DE000DCAD0200000000000000E0000100350022
:104DF0000044EB000804E0005F003A00C09E800021
:104E0000D19E80000200200003122400EEAA0200BE
:104E1000000000000002BE00209E8000319E800045
:104E200018C0B3000001BE000400BE00E0AD0200E7
:104E3000000000000000E00001003C000044EB0026
:104E40000804E0004C003A00009F8000119F8000A1
:104E50000200200003122400F0AA0200000000005B
:104E60000002BE00609E8000719E800018C0B300EA
:104E70000001BE000400BE00DCAD02000000000026
:104E80000000E000010035000044EB000804E000F1
:104E900039003A00009F8000119F8000020020002E
:104EA00003122400EEAA0200000000000002BE006F
:104EB000609E8000719E800018C0B3000001BE009B
:104EC0000400BE00E0AD0200000000000000E000B1
:104ED00001003C000044EB000804E00026003A001A
:104EE000209F8000319F80000200200003122400D8
:104EF000F0AA0200000000000002BE00809E8000B8
:104F0000919E800018C0B3000001BE000400BE00E6
:104F1000DCAD0200000000000000E00001003500F0
:104F20000044EB000804E00013003A00209F8000DA
:104F3000319F80000200200003122400EEAA02002C
:104F4000000000000002BE00809E8000919E800054
:104F500018C0B3000001BE000400BE00E0AD0200B6
:104F6000000000000000E00001003C000044EB00F5
:104F70000804E00004003200B4FD0700F09D80004A
:104F80000000E800F09D8800A09D8000B19D800099
:104F90000001BE000000200001F82300EEAA02007C
:104FA000000000000002BE00A09E8000B19E8000B4
:104FB0000001BE000400BE009CB102000000000021
:104FC0000004BE00A49D8000B59D8000009E80006E
:104FD000119E80000001BE000400BE009CB10200D2
:104FE000000000000001BE000800BE00F0AA0200A0
:104FF00000000000009E8800119E8800A09D800097
:10500000B19D80000001BE000000200001F82300D7
:10501000EEAA0200000000000002BE00C09E800058
:10502000D19E80000001BE000400BE009CB10200C1
:10503000000000000004BE00A49D8000B59D80001B
:10504000209E8000319E80000001BE000400BE0052
:105050009CB10200000000000001BE000800BE007C
:10506000F0AA020000000000209E8800319E880007
:105070001080200010407800E34F50001D003A00DF
:10508000A09D8000B19D80000001BE0000002000B6
:1050900001F82300EEAA0200000000000002BE009A
:1050A000E09E8000F19E80000001BE000400BE0072
:1050B0009CB10200000000000004BE00A49D80001E
:1050C000B59D8000409E8000519E80000001BE0082
:1050D0000400BE009CB10200000000000001BE0000
:1050E0000800BE00F0AA020000000000409E8800F8
:1050F000519E8800A09D8000B19D80000001BE00EF
:105100000000200001F82300EEAA020000000000C9
:105110000002BE00009F8000119F80000001BE00C1
:105120000400BE009CB10200000000000004BE00AC
:10513000A49D8000B59D8000609E8000719E8000CF
:105140000001BE000400BE009CB10200000000008F
:105150000001BE000800BE00F0AA0200000000002E
:10516000609E8800719E8800A09D8000B19D800097
:105170000001BE000000200001F82300EEAA02009A
:10518000000000000002BE00209F8000319F8000D0
:105190000001BE000400BE009CB10200000000003F
:1051A0000004BE00A49D8000B59D8000809E80000C
:1051B000919E80000001BE000400BE009CB1020070
:1051C000000000000001BE000800BE00F0AA0200BE
:1051D00000000000809E8800919E8800009E800054
:1051E000119E8000A09E8800B19E8800209E8000B5
:1051F000319E8000C09E8800D19E880010802000D3
:1052000010407800E34F500004003A00409E8000B8
:10521000519E8000E09E8800F19E8800609E800084
:10522000719E8000009F8800119F8800809E8000F2
:10523000919E8000209F8800319F8800009E800002
:10524000119E800018C0B30002002000832C2400AF
:10525000E0AD0200000000000000E00001003D00A1
:105260000044EB000804E000090032009000200038
:10527000709F880090002000809F88009000200090
:10528000909F880090002000A09F88004600370073
:10529000009E8000119E8000020020000312240066
:1052A00072AC02000000000001F0A100B0AE0200EC
:1052B0000000000000007800709F8800009E8000C1
:1052C000119E800001F0A100B0AE020000000000BD
:1052D00000017800719F800060FF2F000088B900F6
:1052E0000000780000004100809F8800009E800040
:1052F000119E800002002000031224009CB10200D5
:105300000000000001F0A100B0AE020000000000AB
:1053100000017800819F800060FF2F000088B900A5
:1053200080017800719F8000C0F92F000088B900CB
:10533000000078000080410000004100909F88003C
:10534000009E8000119E800002002000832C24001B
:105350009CB102000000000001F0A100B0AE02000C
:105360000000000000017800819F8000C0F92F003C
:105370000088B90080017800719F800080C12F00F3
:105380000088B90000007800008041000001410061
:10539000919F800060FF2F000088B9000000780016
:1053A00000004100A09F8800209E8000319E800068
:1053B00018C0B30002002000832C2400E0AD0200DE
:1053C000000000000000E00001003D000044EB0090
:1053D0000804E0000900320090002000B09F88001F
:1053E00090002000C09F880090002000D09F88007F
:1053F00090002000E09F880046003700209E80003B
:10540000319E8000020020000312240072AC0200D2
:105410000000000001F0A100B0AE0200000000009A
:1054200000007800B09F8800209E8000319E8000A0
:1054300001F0A100B0AE0200000000000001780001
:10544000B19F800060FF2F000088B9000000780045
:1054500000004100C09F8800209E8000319E800097
:1054600002002000031224009CB102000000000092
:1054700001F0A100B0AE02000000000000017800C1
:10548000C19F800060FF2F000088B9008001780074
:10549000B19F8000C0F92F000088B900000078009B
:1054A0000080410000004100D09F8800209E8000C5
:1054B000319E800002002000832C24009CB1020059
:1054C0000000000001F0A100B0AE020000000000EA
:1054D00000017800C19F8000C0F92F000088B9004A
:1054E00080017800B19F800080C12F000088B90042
:1054F000000078000080410000014100D19F800041
:1055000060FF2F000088B900000078000000410013
:10551000E09F88001080200010407800E34F50008A
:105520005B003A00409E8000519E800018C0B3008E
:1055300002002000832C2400E0AD020000000000E7
:105540000000E00001003D000044EB000804E00022
:105550000900320090002000F09F88009000200099
:1055600000A088009000200010A08800900020007B
:1055700020A0880046003700409E8000519E800099
:10558000020020000312240072AC020000000000A0
:1055900001F0A100B0AE02000000000000007800A1
:1055A000F09F8800409E8000519E800001F0A10085
:1055B000B0AE02000000000000017800F19F800002
:1055C00060FF2F000088B900000078000000410053
:1055D00000A08800409E8000519E800002002000B4
:1055E000031224009CB102000000000001F0A100A1
:1055F000B0AE0200000000000001780001A08000B1
:1056000060FF2F000088B90080017800F19F8000C2
:10561000C0F92F000088B900000078000080410028
:105620000000410010A08800409E8000519E800034
:1056300002002000832C24009CB102000000000026
:1056400001F0A100B0AE02000000000000017800EF
:1056500001A08000C0F92F000088B9008001780007
:10566000F19F800080C12F000088B9000000780001
:10567000008041000001410011A0800060FF2F0068
:105680000088B900000078000000410020A08800D8
:10569000609E8000719E800018C0B3000200200050
:1056A000832C2400E0AD0200000000000000E000B8
:1056B00001003D000044EB000804E0000900320056
:1056C0009000200030A088009000200040A08800BA
:1056D0009000200050A088009000200060A088006A
:1056E00046003700609E8000719E8000020020000E
:1056F0000312240072AC02000000000001F0A100BF
:10570000B0AE0200000000000000780030A0880069
:10571000609E8000719E800001F0A100B0AE02008A
:10572000000000000001780031A0800060FF2F0021
:105730000088B900000078000000410040A0880007
:10574000609E8000719E80000200200003122400F1
:105750009CB102000000000001F0A100B0AE020008
:10576000000000000001780041A0800060FF2F00D1
:105770000088B9008001780031A08000C0F92F00B6
:105780000088B9000000780000804100000041005E
:1057900050A08800609E8000719E80000200200062
:1057A000832C24009CB102000000000001F0A10045
:1057B000B0AE0200000000000001780041A08000AF
:1057C000C0F92F000088B9008001780031A0800066
:1057D00080C12F000088B9000000780000804100DF
:1057E0000001410051A0800060FF2F000088B90037
:1057F000000078000000410060A08800809E8000CA
:10580000919E800018C0B30002002000832C240069
:10581000E0AD0200000000000000E00001003D00DB
:105820000044EB000804E000090032009000200072
:1058300070A088009000200080A0880090002000C8
:1058400090A0880090002000A0A0880046003700AB
:10585000809E8000919E80000200200003122400A0
:1058600072AC02000000000001F0A100B0AE020026
:10587000000000000000780070A08800809E80007A
:10588000919E800001F0A100B0AE02000000000077
:105890000001780071A0800060FF2F000088B9002F
:1058A000000078000000410080A08800809E8000F9
:1058B000919E800002002000031224009CB102008F
:1058C0000000000001F0A100B0AE020000000000E6
:1058D0000001780081A0800060FF2F000088B900DF
:1058E0008001780071A08000C0F92F000088B90005
:1058F00000007800008041000000410090A0880076
:10590000809E8000919E800002002000832C240055
:105910009CB102000000000001F0A100B0AE020046
:10592000000000000001780081A08000C0F92F0075
:105930000088B9008001780071A0800080C12F002C
:105940000088B9000000780000804100000141009B
:1059500091A0800060FF2F000088B900000078004F
:1059600000004100A0A08800009E8000119E8000E1
:1059700018C0B30002002000C3282400E0AD0200DC
:10598000000000000000E00001003C000044EB00CB
:105990000804E0000C003A00009E8000119E800088
:1059A00018C0B3000200200003122C00DCAD02007E
:1059B000000000000000E000010035000044EB00A2
:1059C0000804E00003003200803E210011C0B30053
:1059D00001487800209E8000319E800018C0B300EE
:1059E00002002000C3282400E0AD020000000000F7
:1059F0000000E00001003C000044EB000804E0006F
:105A00000C003A00209E8000319E800018C0B30038
:105A10000200200003122C00DCAD02000000000098
:105A20000000E000010035000044EB000804E00045
:105A300003003200903E210011C0B30001487800FD
:105A40001080200010407800E34F50001B003A0007
:105A5000409E8000519E800018C0B30002002000CC
:105A6000C3282400E0AD0200000000000000E000B8
:105A700001003C000044EB000804E0000C003A0088
:105A8000409E8000519E800018C0B300020020009C
:105A900003122C00DCAD0200000000000000E0005A
:105AA000010035000044EB000804E0000300320070
:105AB000A03E210011C0B30001487800609E800024
:105AC000719E800018C0B30002002000C32824008B
:105AD000E0AD0200000000000000E00001003C001A
:105AE0000044EB000804E0000C003A00609E8000D7
:105AF000719E800018C0B3000200200003122C0029
:105B0000DCAD0200000000000000E00001003500F4
:105B10000044EB000804E00003003200B03E210026
:105B200011C0B30001487800809E8000919E8000E3
:105B300018C0B30002002000C3282400E0AD02001A
:105B4000000000000000E00001003C000044EB0009
:105B50000804E0000C003A00809E8000919E8000C6
:105B600018C0B3000200200003122C00DCAD0200BC
:105B7000000000000000E000010035000044EB00E0
:105B80000804E00003003200C03E210011C0B30051
:105B9000014878000080200010407800E14F50005C
:105BA00010003A006C3A020002000000D03A0200F5
:105BB000020000001080200010407800E34F5000E9
:105BC00002003A00343B020002000000983B020051
:105BD00002000000FC3B0200020000007C3F0200CB
:105BE000020000004F04BE000080FA000000060022
:105BF0005000FA004135800000FC2F00008060005A
:105C00001001B300403588005136800000FC2F00A1
:105C1000008060007000B30050368800F1368000CC
:105C200000FC2F00008060000030A000F0368800EB
:105C3000E8A2A800E882A900E842A900E902A900B8
:105C4000ED02A9004022EF00101280000020A10008
:105C50000030A1000040A100101288001012800046
:105C60000000A0000010A0001012880042A2A800AE
:105C70004422EF004822EF004342A9004302A9005A
:105C800042C2A8004322A90041E2A800F00F200070
:105C900010079800F00F200020079800F00F200058
:105CA00030079800F00F2000400798000001200006
:105CB0005007980050012000600798000001200064
:105CC00070079800F000470022602B0008000900D0
:105CD000B2187800210220008100470042612B00A9
:105CE00008000900B218780080002000201F9800EA
:105CF00000082000301F9800F0002000401F98008E
:105D000000072000501F980000082000601F980026
:105D100000082000701F980000082000002798004D
:105D20008000200010279800000A200020279800FB
:105D3000F0002000302798008007200040279800BE
:105D400000082000502798000008200060279800D5
:105D500000082000702798000040EB00004F7800FA
:105D6000070037001E00FB00000040000000470055
:105D700010009000AC890200020000001E4FE800F5
:105D80001E407800E34F5000F6FF3400903C0700BF
:105D90000040EB00004F7800070037001E00FB00BA
:105DA000000040000000470050009000AC89020055
:105DB000020000001E4FE8001E407800E24F500035
:105DC000F6FF34000040EB00004F7800070037007A
:105DD0001E00FB000000400000004700201890005B
:105DE000AC890200020000001E4FE8001E4078004F
:105DF000E24F5000F6FF3400000000005117800011
:105E000000022000008060000000E000FBFF3A007C
:105E10006F3C07000040EB00004F780007003700A0
:105E20001E00FB0000004000000047001020900012
:105E3000AC890200020000001E4FE8001E407800FE
:105E4000E24F5000F6FF34000000000051178000C0
:105E500000022000008060000000E000FBFF3A002C
:105E60000040EB00004F7800070037001E00FB00E9
:105E7000000040000000470010109000AC890200B4
:105E8000020000001E4FE8001E407800E84F50005E
:105E9000F6FF3400000000000080FA000000060059
:105EA0000200FA00D902A80017E2A900C1C2A900A5
:105EB000C1E2A800000000001116800000002800C8
:105EC000008060000000E00009003A00C5C2A9009F
:105ED000703C0700C5C2A8006E3C07001116800088
:105EE00000002800008060000000E000F7FF3200A2
:105EF000F00420002010880007E2A9000722A80073
:105F00008620A90007E2A8001C820200020000000F
:105F100020C1B300004F78001E00FB0000004000CD
:105F2000004F78001E00FB00D88202000200000033
:105F300000012000D8820200020000004001200081
:105F4000D882020002000000A00F2100104078005B
:105F50000000FB0069001000D8820200020000006F
:105F6000A00F2100104078000000FB006800100026
:105F7000D882020002000000A00F2100104078002B
:105F80000000FB0069001000D8820200020000003F
:105F900040012000D88202000200000040012000E1
:105FA000D88202000200000020002000D8820200F7
:105FB000020000000000EB00D88202000200000096
:105FC000E0002000D882020002000000E000200073
:105FD000D8820200020000000000EB00D88202001C
:105FE0000200000096830200020000004E820200C0
:105FF00002000000020007000080FA000000060016
:106000000200FA0020C1B300004F78000060FE00DB
:106010000060FE001C820200020000001E00FB0067
:1060200000004000004F78001E00FB00D8820200F4
:106030000200000040002000D882020002000000A0
:106040007A820200020000001E4078000040E80052
:10605000004F78001E00FB00D88202000200000002
:1060600062830200020000008040780060E52000AA
:1060700001487800348302000200000010479800B5
:1060800096830200020000004E820200020000001F
:1060900060E52000104078000080FA000000060053
:1060A0000000FA0000F9070008000700960007004A
:1060B000F043210010407800E14F500001003A0009
:1060C000240407000080FA00000006000200FA0025
:1060D000C022A80017E2A900C042A900C062A8001F
:1060E0000000000010168000680060000000E00062
:1060F00008003A00C442A900E63B0700C442A800D9
:10610000E43B070010168000680060000000E0001B
:10611000F8FF320040012000A01088001722A800DC
:106120008A40A90017E2A80000000000E2830200F4
:1061300002000000E00D20009E840200020000002A
:10614000300020009E84020002000000E283020072
:1061500002000000F00D20009E84020002000000FA
:10616000FA84020002000000004F78009E80FB00CD
:1061700000022000008060000000E0000B003A00F8
:10618000E283020002000000E00D20009E84020075
:10619000020000000000EB009E84020002000000EC
:1061A000000820009E840200020000001E80FB0008
:1061B000680060000000E0000B003A00E28302008B
:1061C00002000000E00D20009E840200020000009A
:1061D000300020009E8402000200000080002000A9
:1061E0009E84020002000000E28302000200000020
:1061F000E00A20009E84020002000000100120003E
:106200009E84020002000000E283020002000000FF
:10621000F00A20009E84020002000000FA840200BE
:10622000020000008040780000432100014878000F
:1062300014840200020000000080FA000000060042
:106240000000FA00C022A80017E2A900C042A9007D
:10625000C062A80000000000101680006800600006
:106260000000E00008003A00C442A900893B070092
:10627000C442A800873B0700101680006800600039
:106280000000E000F8FF320040012000A01088006C
:106290001722A8008A40A90017E2A8000000000009
:1062A000E283020002000000E00A20009E84020057
:1062B00002000000F00020009E84020002000000A6
:1062C000E283020002000000F00A20009E84020027
:1062D00002000000FA840200020000008040780002
:1062E000F0422100014878001484020002000000FE
:1062F000F042210090407800A00F21000148780072
:106300000080FA00000006000000FA00E2830200AC
:1063100002000000E00A20009E840200020000004B
:10632000800120009E84020002000000E28302003F
:1063300002000000F00A20009E840200020000001B
:106340002885020002000000D0A18800FA84020023
:106350000200000080407800C0432100014878001E
:106360001484020002000000D0A1800061006000DF
:106370000000E00003003200E043210011C0B30040
:1063800001487800D0A18000610060000000E000BA
:1063900003003A00E04321008040EB000148780010
:1063A000D0A18000620060000000E0000300320025
:1063B000F043210011C0B30001487800D0A1800053
:1063C000620060000000E00003003A00F04321009A
:1063D0008040EB0001487800D0A180007000600090
:1063E0000000E000030032000044210011C0B300AF
:1063F00001487800D0A18000700060000000E0003B
:1064000003003A00004421008040EB00014878007E
:106410000080FA00000006000400FA00E283020097
:1064200002000000E00A20009E840200020000003A
:106430000000EB009E84020002000000E2830200E4
:1064400002000000F00A20009E840200020000000A
:106450002885020002000000B0A088002885020004
:1064600002000000C0A08800288502000200000091
:10647000E0A088002885020002000000F0A088004B
:10648000288502000200000000A188002885020083
:106490000200000010A18800288502000200000010
:1064A0008040780050422100014878002885020091
:1064B000020000008040780040422100014878003E
:1064C000288502000200000030A188002885020013
:1064D0000200000040A188002885020002000000A0
:1064E00080407800A0422100014878002885020001
:1064F0000200000080407800B0422100014878008E
:10650000288502000200000080407800C04221007F
:1065100001487800288502000200000080407800D1
:10652000D0422100014878002885020002000000C6
:1065300080407800E0422100014878002885020070
:106540000200000080407800F042210001487800FD
:10655000288502000200000090A188002885020022
:1065600002000000A0A188002885020002000000AF
:10657000B0A188002885020002000000C0A18800A8
:1065800028850200020000002047980028850200AC
:106590000200000020479800288502000200000049
:1065A00020479800FA84020002000000204798006B
:1065B000B0A08000610060000000E0008A003200AE
:1065C000E283020002000000E00A20009E84020034
:1065D000020000000000EB009E84020002000000A8
:1065E000C00020009E840200020000000000EB00BA
:1065F0009E84020002000000800A20009E840200A7
:1066000002000000100620009E840200020000002C
:106610000000EB009E840200020000000000EB007E
:106620009E840200020000000000EB009E84020035
:1066300002000000300220009E84020002000000E0
:106640001484020002000000000000000000EB00C3
:10665000000F7800280037008E3A0700E28302001E
:1066600002000000E00A20009E84020002000000F8
:106670000000E0001F003A00800020009E8402001D
:1066800002000000100020009E84020002000000B2
:106690000000EB009E8402000200000010002000B9
:1066A0009E840200020000000000EB009E840200B5
:1066B00002000000100020009E8402000200000082
:1066C000100020009E840200020000000000EB0089
:1066D0009E84020002000000200020009E84020030
:1066E000020000001484020002000000000000000C
:1066F000050037001E0FE800300620009E007800DD
:10670000808F5000D4FF34000000EB00000F7800B1
:10671000280037005F3A0700E28302000200000011
:10672000E00A20009E840200020000000000E00059
:106730001F003A00000120009E84020002000000B9
:106740000000EB009E840200020000000000EB004D
:106750009E84020002000000500720009E84020078
:10676000020000000000EB009E8402000200000016
:106770000000EB009E840200020000000000EB001D
:106780009E840200020000000000EB009E840200D4
:10679000020000000000EB009E84020002000000E6
:1067A0001484020002000000000000000500370011
:1067B0001E0FE800300620009E007800808F5000F9
:1067C000D4FF3400400620009E007800808F5000E7
:1067D00009003A005C8502000200000014840200F7
:1067E00002000000040037005C8502000200000087
:1067F00014840200020000000080FA00000006007D
:106800000000FA00B0A080004200DE00614060009D
:1068100080407800800E210001487800B0A0800000
:106820004300DE006140600080407800A00E21003F
:1068300001487800B0A080004400DE0061406000A4
:1068400080407800C00E210001487800B0A0800090
:106850004600DE006140600080407800B00E2100FC
:1068600001487800F0A080004800DD008000EB00C7
